:020000040802F0
:1000000030A000103503020813560208F54F02080D
:10001000C355020811370208517B02080000000096
:100020000000000000000000000000001B6C02083F
:10003000BD44020800000000F3310208415C0208E0
:10004000897C02084F0302084F0302084F0302088D
:100050004F0302084F0302084F0302084F03020830
:100060004F0302084F0302084F0302084F03020820
:100070004F0302084F0302084F0302084F03020810
:100080004F0302084F0302084F03020845380208D5
:10009000093802084F0302084F030208C14402084E
:1000A0004F0302084F0302084F0302084F030208E0
:1000B0004F030208356F0208D56F02084F0302088C
:1000C0004F0302084F0302084F0302084F030208C0
:1000D0004F0302085972020851730208A9730208FB
:1000E0004F0302084F0302084F0302084F030208A0
:1000F0004F0302084F0302084F0302084F03020890
:100100004F0302084F030208097002084F03020858
:100110004F0302084F0302084F0302084170020810
:100120004F0302084F0302084F0302084F0302085F
:100130004F0302084F0302084F030208ED3902087B
:10014000B13902084F0302084F0302084F030208A7
:100150004F0302084F0302084F030208A17402086C
:100160004F0302084F0302084F0302084F0302081F
:100170004F0302084F0302084F0302084F0302080F
:100180004F0302084F03020800F002F800F0C0F825
:100190000AA090E8000C82448344AAF10107DA45E2
:1001A00001D100F0B5F8AFF2090EBAE80F0013F074
:1001B000010F18BFFB1A43F00103184798CC000049
:1001C000D8CC00000A444FF0000C10F8013B13F0AB
:1001D000070408BF10F8014B1D1108BF10F8015BA0
:1001E000641E05D010F8016B641E01F8016BF9D193
:1001F00013F0080F1EBF10F8014BAD1C0C1B09D1EA
:100200006D1E58BF01F801CBFAD505E014F8016B5B
:1002100001F8016B6D1EF9D59142D6D370470000ED
:10022000103A24BF78C878C1FAD8520724BF30C822
:1002300030C144BF04680C607047000000230024F4
:1002400000250026103A28BF78C1FBD8520728BFE6
:1002500030C148BF0B6070476E2900F04A85702995
:1002600000F0938166290CF0A98265290CF0A68222
:1002700067290CF0A38261290CF0A28203681B0A93
:1002800028BF41F08001692900F00481642900F051
:100290000181752900F0FE806F2900F030867829F1
:1002A00000F05F81E92900F0CB85E42900F0C885E2
:1002B000F52900F0C585EF2900F02D86F82900F01A
:1002C0005E810368DB0928BF41F08001632900F0EB
:1002D0004C85732900F05185E32901F09B85F329B2
:1002E00001F0A085002070471FB50CF05AFA01F00C
:1002F000A7F90400002000210BF0B0FB401C606057
:10030000002000210BF0C0FBE0601FBD10B510BD48
:1003100001F0FEFF1146FFF7E7FF0AF049FB02F08C
:1003200087FA03B4FFF7F2FF03BC09F0E7F8000017
:1003300040BA70470948804709480047FEE7FEE792
:10034000FEE7FEE7FEE7FEE7FEE7FEE7FEE7FEE785
:1003500004480549034A054B70470000D96E02085E
:10036000890102083091001030A000103091001077
:1003700072B6704762B67047EFF3108072B670477E
:1003800080F31088704730BF704720BF7047B0FAC5
:1003900080F0704790FAA0F0B0FA80F0704790FAC1
:1003A000A0F070471CB50C46064B7B446946009094
:1003B000204600F0B8FC04460020694600F0C6FC68
:1003C00020461CBD9F0900000FB41CB5084B06AAAF
:1003D0007B4469460090059800F0A5FC0446002087
:1003E000694600F0B3FC20461CBC5DF814FB00001D
:1003F0007909000070B5044685690068C10601D519
:10040000302600E02026C00707D070BDD4E90121C6
:1004100030469047206A401C20626D1EF6D570BDA4
:1004200070B5044685690078C00707D170BDD4E96E
:10043000012120209047206A401C20626D1EF6D5C5
:1004400070BD70B50C460546012A05D02878800697
:1004500000D5EA69002302E0012305E05B1C93421A
:1004600002D2E05C0028F9D1A869E618C01AA86198
:10047000286A184428622846FFF7BCFF04E0D5E943
:10048000012114F8010B9047B442F8D32846FFF736
:10049000C7FF70BD2DE9F04106460024106875299C
:1004A000314616A510D000F0B9FB002802DA404210
:1004B00013A507E031688A0701D512A502E04907B4
:1004C00004D511A5012401E000F0B1FB00210A22AE
:1004D00006F1240709E0B0FBF2FCB0FBF2F302FBEB
:1004E0001C00303078541846491C0028F3D12346AC
:1004F0002A463046BDE8F04100F0A2BB00000000F3
:100500002D0000002B00000020000000F0B40D467C
:100510000188090502D5214C7C4402E01F4C7C4433
:100520000E34002100F1240608E002F00F07120942
:10053000E75D42EA03721B097754491C52EA03073C
:10054000F3D102780023120704D5702D06D009B12B
:10055000022311342246F0BC00F072BB0123103498
:10056000F8E770B504460D462146106800F05FFBC1
:10057000024629462046BDE870400023C6E7D21D4A
:1005800022F00703D3E90023C0E70368126843F0B1
:10059000200303600823C3610023B7E7D2C500002E
:1005A0002DE9F05F894604464FF0000ADFF874B188
:1005B000FB44C0F820A02046E1688847002874D09A
:1005C000252806D0D4E901219047206A401C2062EA
:1005D000F1E700265F462046E16888472028054667
:1005E00007DB312D05D2781910F8200C08B106432D
:1005F000F1E7B00701D526F00406C4F81CA00027D7
:10060000C4F818A02A2D09D0284608F070FF38B386
:1006100004EB8708303DC8F8185019E059F8041B5E
:10062000204604EB87029161E1688847012F054667
:1006300018D1E069002820DA26F020061DE0D8F85D
:10064000180000EB800005EB40003038C8F81800B7
:100650002046E1688847054608F049FF0028EED1AA
:10066000012F0AD02E2D08D12046E16888477F1C33
:100670000546022F46F02006C4DBA069002803DAF5
:10068000404246F00106A061F00701D026F01006B6
:100690006C2D0BD0682D09D04C2D39D06A2D35D05A
:1006A000742D35D07A2D33D016E038E0E1682F462E
:1006B00020468847B842054609D16C2F26D04FF412
:1006C0008060E168064320468847054604E06C2FB9
:1006D0001AD04FF4807006430DB3A5F141001928DC
:1006E00002D8203546F400664A4629462046266050
:1006F0004E46FFF7B1FD80B101280BD0F61D26F064
:10070000070000F1080956E74020E4E78020D8E719
:100710000020D6E706F104094DE7284652E7206A93
:10072000BDE8F09F62C500000FB400B58DB010A900
:10073000099000910B904FF0FF300A9000200C9030
:10074000064878440690064878446A4607900F9910
:1007500009A800F07BFE0DB05DF814FB270D00002A
:100760003F0D00002DE9FF5F1D464FF0FF3B914616
:100770004FF000085F46D5E90146A96901987F1C42
:100780008847296A824688470028F6D1BAF1FF3F98
:100790000CD0002E24F4C06419DD600614D5BAF123
:1007A0002B0F09D0BAF12D0F0ED103E0584604B03B
:1007B000BDE8F09F44F48064A96901987F1C8847D4
:1007C000761E8246002E02DDBAF1300F03D0B9F159
:1007D000000F26D032E0A969761E01987F1C44F4F0
:1007E00000748847002E824605DDBAF1780F06D0E6
:1007F000BAF1580F03D0B9F1000F10D01EE0B9F1D3
:10080000000F02D0B9F1100F18D1A969761E019816
:100810007F1C24F4007488478246102002E00820E0
:1008200000E00A20814609E0A96908FB0908761E54
:1008300001987F1C44F4007488478246002E05DD31
:100840004946504600F072FB0028EDDAE96901984C
:100850008847A00502D46FF00100A8E7E00725D182
:10086000600613D5600502D5C8F1000000E04046DF
:1008700029680A1D2A600968220501D5087015E05B
:10088000220701D5088011E008600FE02868011DEB
:1008900029600068210502D580F8008006E0210764
:1008A00002D5A0F8008001E0C0F8008038467EE75D
:1008B00070B5064600F096F90468054630460A22EF
:1008C000002100F042FE2C6070BD2DE9F05F9346E0
:1008D0000F4680460446002600F084F9D0F80090C8
:1008E000824614F8015B2DB100F074F90068405D98
:1008F000C007F6D12B2D02D02D2D1AD0641E002159
:10090000CAF800105A463946204600F0CFFD01468D
:1009100027B13868A04201D1C7F80080DAF800009A
:10092000022809D0CAF80090700505D54842BDE8F4
:10093000F09F46F48066E2E70846F8E70EB5054604
:1009400014460E4613A000F043FE284600F040FE79
:1009500016A000F03DFE304600F03AFE15A000F073
:1009600037FE00218DF80B100A210DF10A008DF8D9
:100970000A1008E094FBF1F201FB124294FBF1F43F
:10098000303200F8012D002CF4DC00F021FE00F0E4
:1009900014FE00002A2A2A20617373657274696F3D
:1009A0006E206661696C65643A2000002C206669DF
:1009B0006C6520002C206C696E652000014A00F0F7
:1009C00011BE0000D407002040EA0103024630B502
:1009D0009B0710D14FF0013400E008C208C91D1B6D
:1009E0009D4315EAC41FF8D013F0FF0102F8011B64
:1009F0000DD01B0AF8E711F8013B002B02F8013B70
:100A000005D011F8013B002B02F8013BF3D130BDBA
:100A10002DE9F0410E460546002400E0641C285DE7
:100A200000F0EFF80746305D00F0EBF8381A02D11D
:100A3000295D0029F2D1BDE8F08110B5431C02E028
:100A400010F8011B71B18107FAD14FF0013202C8D1
:100A50008C1A8C4314EAC211F9D0C01A0A0603D0CA
:100A6000C01E10BDC01A10BD0A0401D0801E10BDEA
:100A70000902FCD0401E10BD421E12F8013F002B9F
:100A8000FBD111F8013B002B02F8013BF9D1704773
:100A9000032A40F2308010F0030C00F0158011F8AA
:100AA000013BBCF1020F624498BF11F801CB00F882
:100AB000013B38BF11F8013BA2F1040298BF00F8D6
:100AC00001CB38BF00F8013B11F0030300F0258093
:100AD000083AC0F0088051F8043B083A51F804CBBA
:100AE000A0E80810F5E7121D5CBF51F8043B40F880
:100AF000043BAFF30080D20724BF11F8013B11F88B
:100B000001CB48BF11F8012B24BF00F8013B00F8CE
:100B100001CB48BF00F8012B704710B5203AC0F058
:100B20000B80B1E81850203AA0E81850B1E81850EE
:100B3000A0E81850BFF4F5AF5FEA027C24BFB1E82B
:100B40001850A0E8185044BF18C918C0BDE810409C
:100B50005FEA827C24BF51F8043B40F8043B08BFA5
:100B60007047D20728BF31F8023B48BF11F8012B6C
:100B700028BF20F8023B48BF00F8012B70474FF018
:100B8000000200B5134694469646203922BFA0E8DD
:100B90000C50A0E80C50B1F12001BFF4F7AF0907E9
:100BA00028BFA0E80C5048BF0CC05DF804EB8900DA
:100BB00028BF40F8042B08BF704748BF20F8022B1D
:100BC00011F0804F18BF00F8012B70477047704735
:100BD0007047000010B500F033FD001D10BD00BFD0
:100BE0007DAE000000487047E81C012010B5FFF7FB
:100BF000F9FF006810BD10B50446FFF7F3FF04606D
:100C000010BD10B50446FFF7E5FF0068005DC006A3
:100C100002D504F1200010BD204610BD09684A0528
:100C200001D540B27047C905FCD500B270470968CC
:100C30004A0501D5C0B27047C905FCD580B27047DE
:100C40002DE9F0470D4699469246044600F12408E6
:100C50000168880604D5E06921F01001216000E0F8
:100C60000120A84201DD471B00E00027A1697A1995
:100C700002EB0900081AA0612078C00602D42046C1
:100C8000FFF7B8FB002608E0D4E901211AF80600B6
:100C90009047206A401C761C20624E45F4DB207889
:100CA000C0060AD52046FFF7A5FB06E0D4E90121DE
:100CB00030209047206A401C2062381EA7F10107AF
:100CC000F4DC07E0D4E9012118F805009047206A18
:100CD000401C2062281EA5F10105F3DC2046FFF729
:100CE0009FFB2078000602D50220BDE8F087012096
:100CF000FBE711680268006A530501D508700AE035
:100D0000D30501D5088006E0130603D5C217C1E953
:100D1000000200E0086001207047000001694A1CE1
:100D200002610878704700B58FB0CDE9013100212C
:100D3000059105497944CDE9031011466846FFF74E
:100D40002FFC0FB000BD0000E5FFFFFF0A6802F8AE
:100D5000010B0A60704710B5436913B1AFF300800F
:100D600001E0FFF76EFB012010BD127800F12401B5
:100D70000A7000224A700122EDE711684FF0FF323D
:100D8000E9E700002DE9FF5F15468A460446DFF8D3
:100D9000AC80F8440027D8E900103E46CDE90010A9
:100DA00010E03AF816106A4602A801F06BFA411CEE
:100DB00007D02178890603D5E269391891420DD808
:100DC0000744761C2078800602D5E069B84205DD2C
:100DD000AE42E6DB3AF816000028E2D1A069C01B5B
:100DE000A0612046FFF706FBD8E90010CDE900100E
:100DF000002017E03AF818106A4602A801F042FAFB
:100E0000B0F1FF3F81460BD000250DF1080B05E046
:100E1000D4E901211BF8050090476D1C4D45F7D31F
:100E200008F10100B0428046E4DB206A38442062C9
:100E30002046FFF7F5FABDE8FF9F0000B2BE0000B4
:100E40002DE9F0418046D21D22F007020025D2E9AB
:100E50000002F52915A614D0011E72F1000106DA70
:100E60000023D0EB030063EB020211A608E0D8F8E0
:100E700000108B0701D50FA602E0490701D50EA689
:100E800001251146002408F1240704E000F0DCFBF2
:100E900030323A55641C50EA0102F7D12B463246F3
:100EA00021464046BDE8F041FFF7CABE0000000001
:100EB0002D0000002B0000002000000030B40021B5
:100EC00000F1240408E002F00705D208303542EAB8
:100ED0004372DB086554491C52EA0305F3D10468E8
:100EE000002310A2250707D5A40600D421B1C469A8
:100EF00001230DA2641EC46130BCFFF7A1BE10B572
:100F0000044621461068FFF792FE02462046BDE8DF
:100F100010400023D2E7D21D22F00701D1E90023BF
:100F2000CCE7000000000000300000003A2800D2AA
:100F3000303820F02002412A01D3A2F13700884244
:100F400001D34FF0FF3070472DE9FF4F06468BB0BD
:100F50000878FF2806D0491C2D2805D000244FF022
:100F6000000908E000200CE00124F8E709EB890300
:100F7000491C00EB43090878FF28F7D114B1C9F1E7
:100F800000008146107800252C46AA4629462D28C7
:100F900001D02B2804D1521C2D2813D000208246CA
:100FA0008B461078FF280FD04FF0000C0A21521CFE
:100FB000A5FB017804FB018105FB0C11C5194BEB66
:100FC0000104EEE70120EAE7002108464FF00000A7
:100FD000BAF1000F02D000EB80004008C0F3815747
:100FE000012F01DD4FF0FF370E9955EA040009EBA0
:100FF00001080BD04FF0020918F5FA7F16DA4FEA14
:10100000CA70002F706008DD012007E04FEACA7047
:10101000C6E900B00FB0BDE8F08F00203060FFF7E8
:10102000E1FDC0F800901821084616E0B8F5FA7FF7
:1010300018DD002F02DAF748784401E0F6487844DA
:10104000D0E90010C6E9001040EACA707060FFF7EE
:10105000C9FDC0F80090142108460FB0BDE8F04F5C
:101060000BF0A9BB002108464FF00000B8F10001C9
:10107000099002DAC7F1000200E03A4601DAC8F14D
:10108000000106A801F08CF806AB93E8070003AB5B
:1010900083E8070044F23E005BEA040100905846F2
:1010A00004D144F21E012C465D460091210C090436
:1010B000014306D10099240444EA15442D04103953
:1010C000009104F07F41014306D10099240244EAD3
:1010D00015642D020839009104F07041014306D1D6
:1010E0000099240144EA15742D01091F009104F0B0
:1010F0004041014306D10099A40044EA9574AD0033
:10110000891E009104F00041084304D100986D1934
:101110006441401E00904FF001033A466846B8F122
:10112000000FCDE9014503A902DD01F010FF01E048
:1011300001F0E3FEBAF1000F04460D4601D084F041
:101140000044002108464FF00000099940F2FF7763
:10115000484010F00C0F07D124F00040284303D082
:10116000C4F30A50B84212D1FFF73CFDC0F800901A
:10117000C4F30A50B8420AD1A8487844D0E9001014
:10118000C6E9001004F000410843706042E7C6E978
:1011900000543FE72DE9FF4F1F464FF0000A4FF084
:1011A000FF38454691B0D7E90146CDF83CA000F0A4
:1011B00047FAC0680168405C1090B96912986D1CCC
:1011C0008847396A814688470028F6D1B9F1FF3F40
:1011D0000AD0002E24F4D06411DDB9F12B0F08D011
:1011E000B9F12D0F0BD102E0404615B013E744F4DE
:1011F0008064B96912986D1C8847761E8146600527
:1012000004A901D52D2000E02B20002E01F1010BB7
:101210000DF130088DF810003FDDB9F1690F08D0ED
:10122000B9F1490F05D0B9F16E0F02D0B9F14E0FE7
:101230001CD13B4601A8009580E85002DDE912125E
:101240006FF002000BF022FBC11CCED10EE0B96999
:1012500012986D1C884781461398761E44F40074DA
:1012600005600F98401C002E0F9016DDB9F1300F6D
:10127000EDD0B9F1780F02D0B9F1580F0DD10F9818
:1012800001280AD13B46CDE90054DDE91212001FC6
:1012900002960BF0F9FAC11CA7D1109989453ED1ED
:1012A00044F0800406E01399681CAAF1010A44F492
:1012B00000740860B9696D1C1298761E8847302842
:1012C0008146F0D02BE01099894505D1200603D442
:1012D000761E44F0800418E0484608F008F908B388
:1012E000761E0DF123018B4544F4007408D2A9F158
:1012F00030000BF8010B200607D5AAF1010003E02E
:10130000200602D40AF101008246A00502D51399F5
:10131000681C0860B96912986D1C88478146002EC8
:10132000D1DC53E0002E51DDB9F1650F02D0B9F1E7
:10133000450F4BD1A00549D5B9696D1C1298761E91
:1013400024F440748847002E81460CDD2B2804D0FD
:10135000B9F12D0F07D144F48074B96912986D1C4E
:101360008847761E8146E00501D52D2100E02B211E
:1013700008F8011BCDF8008021E0761E0DF139013F
:10138000884544F400740CD2A9F1300010F0FF003D
:1013900088F8000002D10099884509D908F10108B0
:1013A00006E0E00501D51E4801E042F20F708246DA
:1013B000B96912986D1C8847814613980560002E04
:1013C00004DD484608F093F80028D6D1F969129850
:1013D0008847FF2053468BF8000088F80000002063
:1013E0000A900B9004AA0CA90AA8FFF7ADFDA0056E
:1013F00002D46FF00100F8E614F0240F12D0E007D9
:101400001CD13868DDE90A12031D3B600068C0E9A1
:10141000001213E060BE000052BE000016BD0000C6
:10142000F1D8FFFF0AA9684608F04EF8E00705D199
:101430003868009A011D3960006802602846D4E6C9
:10144000026811441378016018467047D16005495D
:1014500079445161044979441162002111611146B6
:1014600000F0E4BCEDFFFFFF79020000426842B1EA
:10147000016811F8013B23B1521EC0E90012184661
:1014800070470121C160881E704742685AB1C36825
:10149000016843B983688B4205D0491E521CC0E9DC
:1014A0000012002070474FF0FF3070472DE9F05FC9
:1014B000824615468B4600270AF10104B94600789A
:1014C000302801D09DB113E014F8010B01277828D2
:1014D00003D0582801D045B10AE00DB1102D07D135
:1014E000002714F8010B102502E0082500E00A256A
:1014F0000026B0460EE005FB080005FB06F10127BB
:101500001FFA80F801EB1046B6F5803F00D3B946CC
:1015100014F8010B2946FFF709FD0028EBDABBF1AF
:10152000000F05D00FB1641E00E05446CBF8004018
:10153000B9F1000F06D0FFF755FB02210160C81E6C
:10154000BDE8F09F48EA0640FAE72DE9F0479146EA
:101550000F4680460446002614F8015B2DB1FFF7C4
:1015600039FB0068405DC007F6D12B2D02D02D2D30
:1015700018D0641E4A4639462046FFF797FF27B128
:101580003968A14201D1C7F800804FF0020471050B
:101590000BD54042002803DDFFF724FB0460A007C1
:1015A000BDE8F08746F48066E4E70028F8DAFFF744
:1015B00019FB04606FF00040F2E710B5002000F066
:1015C00081FEFEF7A3FEBDE81040012007F096BFA4
:1015D00010B5044602E0641C00F026F820780028CC
:1015E000F9D110BD2DE9F04115460E46040002D197
:1015F0002C6804B90BA4204600F07BFE044420783C
:1016000070B127463146384600F063FE0444207826
:1016100010B1002004F8010B38462C60BDE8F081C1
:101620000027F9E70000000008B569468DF80000C2
:101630000320ABBE08BD000000487047E81C012035
:1016400000487047081D012030B5B0F10A024FEA8A
:10165000900E71F100034EEA817EB0EB0E0061EB5B
:1016600091014FEA101E4EEA017E10EB0E0041EB95
:1016700011114FEA102E4EEA016E10EB0E0041EBF5
:1016800011214FEA104E4EEA014E10EB0E0041EBD5
:101690001141401841F100014FEAD00040EA417089
:1016A0004FEAD10110EB80054FEA810444EA9074BF
:1016B00044EB01046D1944EB0404521BA3414FF0A9
:1016C000000348BF0A3200D530BD401C41F1000183
:1016D00030BD10B50446FFF77DFA0068005D00F0EC
:1016E000010010BD70472DE9FF4F0C461E464FF01C
:1016F000FF378BB0D2E90001DDF860800A908A469E
:10170000C1F30A5505B93D46002108464FF00000D7
:10171000BAF1000F00F4400005DA00EB80004FF44E
:10172000400101EA50004FEA9059B9F1010F00DD84
:10173000B9460A9850EA4A000ED044F61050A5F275
:10174000FF3545432F14B8F1000F1ED07542291EF6
:101750001EDDC9F100021CE0B8F1010F4FF00000DE
:1017600001D0302103E0F24305E02154401CB04297
:10177000FBDB30460022002121540B99C1F8088080
:10178000C1E900200FB0BDE8F08FBD1B6D1CDEE786
:101790004A4600DA694206A800F002FD06AB93E86B
:1017A000070003AB83E8070050460A9901F0D2F81E
:1017B0008DE80700A0F500501F3800900398002D19
:1017C0000ADD42F21F014A460844002303A90390A0
:1017D000684601F07DFB09E0A0F500504A461F383D
:1017E000002303A90390684601F09CFB8DE80700E5
:1017F0000004000C03D04FF0FF30410800E0104619
:10180000B8F1000F03D00022009215461EE0751EAD
:1018100005D4FFF719FF303262556D1EF9D5B34676
:101820000122084302D000227F1C04E020783028E7
:1018300001D100227F1E002A099784D01DE0112DBE
:1018400007DAFFF701FF303262556D1C50EA0102E2
:10185000F5D1084302D00098C8B10EE00021681EFF
:1018600005E0235C625C63542254401E491C8142A3
:10187000F7DBAB46A81B401E0990002004F80B00C4
:101880000B98099AC0F80880C0E9002B7AE7112666
:101890004FF0000857E72DE9F04F88460446D21D67
:1018A00022F0070191B0D1E90001CDE90A0106F06B
:1018B0005DFB02460B98C00F01D02D2007E0206889
:1018C000810701D52B2002E0202101EAC000032A74
:1018D000099001D0072A05DB03464146204600F067
:1018E0003DFD0BE12078800601D5E06900E006208F
:1018F000B8F1650F814606D0B8F1660F18D0B8F17F
:10190000670F70D131E00020B9F1110F009001DBB9
:10191000112301E009F101030AAA01A90CA8FFF7AC
:10192000E2FEDDE90C70002609F10105834647E07F
:1019300001204B4600904FF000470AAA01A90CA8CD
:10194000FFF7D1FEDDE90DB00C995D46002610B918
:1019500009F101000D18B9EB050003D4C0F1FF3601
:1019600009F10105A5EB09002BE0B9F1010F01DA3E
:101970004FF001090020B9F1110F0090484601DD38
:10198000112300E003460AAA01A90CA8FFF7ABFE49
:10199000DDE90C704D4600268346207800070AD406
:1019A000AB4500DA5D4601A8012D04DD411911F8AF
:1019B000011C302907D04F4502DA17F1040F04DA71
:1019C000012082460FE06D1EEEE7002F02DCED1BCA
:1019D0003E4403E0781CA84200DD7D1CB81B00F1EA
:1019E000010A4FF000472078000703D4AA4501DB25
:1019F0004FF0FF3A0021B7F1004F0DF143088DF889
:101A0000431024D002202B23002F01DA7F422D2304
:101A10000A21021EA0F1010000DC5FB197FBF1FC7E
:101A200097FBF1F201FB1C7C17460CF1300C08F817
:101A300001CDEEE7A8F1010003702188090501D569
:101A4000452100E06521A0F1010800F8011C09987A
:101A50000FA9A1EB0807FF1D00B10120411901EBFF
:101A6000EA70A1693844081A401EA0612078C006B7
:101A700002D42046FEF7BEFC099828B1D4E9012122
:101A80009047206A401C20622078C00622D520465C
:101A9000FEF7B0FC1EE0002E04DBB34502DD01A81A
:101AA000805D00E03020D4E901219047206A401C8D
:101AB0002062761CAAF101005FEA000A0AD1FFF752
:101AC000BFFDC0680168405CD4E901219047206AED
:101AD000401C2062281EA5F10105DCDC07E0D4E9EA
:101AE000012118F8010B9047206A401C2062381E23
:101AF000A7F10107F3DC2046FEF792FC032011B0AA
:101B000041E600002DE9F04F04460D46D21D22F0BB
:101B1000070089B0D0E900974846394606F026FA12
:101B20000246F80F01D02D2307E02068810701D578
:101B30002B2302E0202101EAC0038DF820300BB1F5
:101B4000012000E00020032A824601D0072A04DB9E
:101B50002946204600F002FC3FE12078800601D4AF
:101B60000D2500E0E569C7F30A560D2D49DA00217D
:101B70004FEA175B08464FF00000002F00F44000CA
:101B800007DA00EB80004FF4400100EBD07001EA6F
:101B900060008115012901DD4FF0FF3100224FEA7D
:101BA000850CBCF1180F06D31346ACF118004FF0AA
:101BB0008052C24003E04FF4801323FA0CF30CF17F
:101BC0000C0CBCF1200F04D3ACF1200C09FA0CF082
:101BD00001E007FA0CF000294FF0004801DD18B9C8
:101BE0000FE00ED140450CD319EB02095F4121B93A
:101BF000404502D19F4329EA0209BBEB175F00D0A1
:101C0000761C2088000502D57B48784402E07A489B
:101C10007844193808AA302302F80A30037C0AF104
:101C20000101002E0AF1020A53546A4602DC4FF009
:101C3000300101E04FF031014FF001088DF8001044
:101C400002D0A6F2FF3603E059EA470100D06B4EFE
:101C5000002D02DC2178090704D54FF002082E215F
:101C60008DF80110C44600210BE0C7F303433F0188
:101C7000C35C491C6D1E02F80830052908F10108F3
:101C800001DA002DF1DC00210CE000EB1973491C96
:101C90001B786D1E082902F808304FEA091908F16F
:101CA000010801DA002DF0DC21688B0602D516E070
:101CB000A8F10108E04505DD02EB080313F8013C3B
:101CC000302BF5D0B8F1000F09DD02EB080313F853
:101CD000013C2E2B03D1090701D4A8F10108002DE6
:101CE00005DD3E2102F808106D1E08F10108407C58
:101CF000002E02F8080008F1010804DA2D207642CF
:101D000002F8080002E02B2002F808000A214FF434
:101D10007A70864208F101080BDB96FBF0F3303352
:101D200002F8083096FBF0F308F1010800FB136697
:101D300001E0642E0CDB642096FBF0F3303302F8F4
:101D4000083096FBF0F308F1010800FB136601E090
:101D50000A2E06DB96FBF1F0303002F8080008F19D
:101D6000010896FBF1F001FB1060303002F808002A
:101D7000A16908F1010808EB050202EB0A00081A44
:101D8000A0612078C00602D42046FEF733FB216A0A
:101D900008AE01EB0A00206204E0D4E9012116F844
:101DA000010B9047BAF1010AF7D22078C00602D59C
:101DB0002046FEF71FFB6E4609E016F8010B3E2891
:101DC0000FD0D4E901219047206A401C2062B8F16D
:101DD0000108F2D22046FEF723FB09B00320BDE83C
:101DE000F08F206A2844206203E0D4E901213020EA
:101DF00090476D1EEBD3F8E75DB0000002FCFFFFDB
:101E000010B5436913B1AFF3008001E0FEF7BAFFEC
:101E1000012010BD128800F1240182840022C284B6
:101E20000122EDE711684FF0FF32E9E72DE9F34FAA
:101E30004FF0000A0C4656468DB001200C9001F17F
:101E40000C000B9062690B9801219047051E2DD064
:101E5000252D2CD0216A8847C0B162690B980121D9
:101E60009047216A88470028F7D16269411E0B9884
:101E7000904700E0761CA1690D988847216A884741
:101E80000028F7D1E1690D988847DBE7A1690D9833
:101E90008847A842074601D1761CD3E7E1690D982F
:101EA00088477F1C02D1BAF1000F6FD06BE16269E5
:101EB0000B9800273D46394690472A2804D162698D
:101EC0000B98012190470125DFF8D08262690B98B9
:101ED00001219047A0F130010A290AD24745E5DCEB
:101EE00007EB870100EB4107303FDFD445F01005D9
:101EF000ECE7E90601D46FF000476C280AD04C28C3
:101F000014D0682815D06A280DD074281CD07A28DF
:101F10001AD01DE062690B98012190476C2802D00D
:101F200045F0040514E045F002050DE045F02005FC
:101F30000AE062690B9801219047682802D045F0B9
:101F4000080505E045F4006562690B98012190479A
:101F5000C4E9015765283DD019DC58287AD00CDC3B
:101F6000452837D004DC252826D041289ED131E0F1
:101F700046282FD0472899D12CE05B2877D06128BC
:101F800028D063287CD0642823D15AE0F6E06F285B
:101F900048D008DC66281DD067281BD0692821D0CE
:101FA0006E2816D127E0702845D0732868D0752890
:101FB00047D078280DD14DE0A1690D988847252894
:101FC00005463FF469AFE1690D9888476D1C3FF401
:101FD0006AAFD8E00D9923466A466FF001000AF017
:101FE00051FCC5E045F0400023464FF00002606020
:101FF000A80736D43EE0E8077FF447AF2068011D0C
:1020000021600068290501D506701BE7290701D565
:10201000068017E7A90703D5F117C0E9006111E7AA
:1020200006600FE745F0400023464FF0080260606D
:10203000A80716D41EE040F60E0125EA01006060F4
:1020400016E045F0400023464FF00A026060A80702
:1020500007D40FE045F040006060A80708D523468C
:1020600010220D996FF00100AFF3008080E007E0CF
:10207000102223460D996FF00100FEF773FB77E005
:102080004FF0000963284F46C8464B46CB4602D066
:102090005B2806D038E0E80601D40120A0600127C3
:1020A00032E06269D4F80CB00B98012190475E28A9
:1020B00007D14FF0010949466269D4F80CB00B987A
:1020C0009047216939B900210A4603AB43F8212022
:1020D000491C0829FADBD8B3216949B308F1010882
:1020E00062690B98012190475D28F4D1B9F1000F86
:1020F00009D0002003A951F82020D24341F8202024
:10210000401C0828F7DB03AB2069002820794FEA40
:1021100040701ED05B462246CDF80080CDE9019785
:102120000D9900286FF0010020DAAFF300801FE066
:10213000C11703AA00EBD1614B1121F01F0102EB83
:102140008302411A13680120884003431360C7E7E4
:1021500019E00D99224600286FF00100009702DA7D
:10216000AFF3008004E0AFF3008001E0AFF3008044
:1021700000280ADA401C06D10C9820B14FF0FF303D
:102180000FB0BDE8F08F5046FAE7E90701D10AF138
:10219000010A064400200C9054E60000CCCCCC0C84
:1021A0002DE9F047814616468AB0354878440DC877
:1021B0008DE80D0032487844801C03AC0DC884E8DB
:1021C0000D0041F69B300844372190FBF1F290FB63
:1021D000F1F5A5F1800501FB12041B3C02D5644218
:1021E000012000E00020DFF898A080460027FA4494
:1021F000AAF1BE0A0EE0E0070AD03246684607EBB5
:10220000470101230AEB810100F08CFE8DE80700F5
:1022100064107F1C002CEED1194F7F44AE3F19E0B3
:10222000E80715D007EB04100DF1180A90E80E002E
:102230008AE80E00C068F04201D198190890324631
:10224000012306A903A800F06DFE03AB83E8070095
:102250006D10641C002DE3D14FF001033246694636
:10226000B8F1000F03A802D000F032FE01E000F048
:1022700059FEC9E90001C9F808200AB0BDE8F08795
:102280004CAB000070B516460C460546FEF7A2FCA6
:10229000036893F80101012806D0FF2C0FD8185DC0
:1022A00068B101202C7070BDD3F807013246214679
:1022B00003F2071303442846BDE8704018474FF067
:1022C000FF3070BD10B500F0C1FABDE8104000F05D
:1022D000B8BA30B503461D781DB10A4603E0AC42DA
:1022E00001D1181A30BD12F8014B002CF7D15B1C3C
:1022F000F1E730B503461D783DB10A4612F8014BAF
:102300001CB1AC42FAD15B1CF5E7181A30BD70471E
:102310007546FFF791F9AE4605006946534620F031
:102320000700854618B020B5FEF712F8BDE820403A
:102330004FF000064FF000074FF000084FF0000B81
:1023400021F00701AC46ACE8C009ACE8C009ACE834
:10235000C009ACE8C0098D46704700002DE9F04186
:102360001F46044603260168072A01F4006004DBC7
:1023700008B116A505E016A503E008B115A500E013
:1023800015A521F010002060A069C01EA0610FB14A
:10239000401EA0612046FEF72DF84FB1D4E901217F
:1023A00038469047206A401C2062C01C206206E02C
:1023B000206AFAE7D4E9012115F8010B9047761E4F
:1023C000F8D22046FEF72CF8BDE8F0814E414E00D1
:1023D0006E616E00494E4600696E66002DE9FF4F42
:1023E0001F464FF03C0987B04FF00042DDE9141062
:1023F00001F10108DDF858A002EA405003900020E6
:1024000005908346054604460490B969461E08981F
:102410008847AAF1010A0290BAF1000F3BDD029849
:102420002E2815D01021FEF781FD00282EDB4FF05D
:10243000010B0599014317D0B9F1000F0BDB4A4698
:10244000C11700F05BFA05430C43A9F1040905E04C
:10245000012004900BE008B145F001050120059032
:10246000049820B9361D02E0049800B1361FB969FE
:10247000089808F101088847BBF1000FAAF1010A8A
:102480000290C9D00999C1F80080C5E70298702868
:1024900008D0502806D0F96908988847BBF1000F8A
:1024A00014D04FE0002002900120BBF1000F0490F7
:1024B00009D0B969089808F101088847AAF101090B
:1024C000B9F1000F07DCF969089888476FF001003F
:1024D0000BB0BDE8F08F2B2804D02D280CD14FF085
:1024E000FF300490B969089808F101088847A9F1FC
:1024F0000109B9F1000FE6DD411CE4D00A21FEF725
:1025000015FD0028DFDB029908F1010801EB8101CC
:1025100000EB41000290B969089888470A21FEF74C
:1025200005FD099AA9F10109B9F1000FC2F800806F
:1025300001DD0028E7DAF9690898884704990298CC
:1025400000FB016655EA040004D004F04041090094
:1025500002D006E0039898E0A40044EA9574AD0028
:10256000B61E04F00041080002D16D196441761EC8
:10257000159810F0240F03D04FF00B095C4803E0CE
:102580004FF028096FF07D008246564507DAAAEB26
:1025900006018944B9F1410F01DD4FF041090120E5
:1025A0000021A9F1010200F0A9F9024628400B46DA
:1025B0002140084301D0012100E00021501E02917A
:1025C00043F1FF3128402140084301D0012000E0C1
:1025D00000200299834651EA0B014FD000210846A2
:1025E0004FF00000039900F4400039B100EB800087
:1025F0004FF4400100EBD07001EA60008015012823
:1026000002DD4FF0FF3000E013D0401C36D00298BE
:1026100060B3BBF1000F0CD14A460120002100F04D
:102620006DF928402140084301D0012000E000203E
:10263000E0B101204A46002100F060F9034640194C
:102640000A4661412D1A8C4111D3B9F1400F09DDC1
:10265000159810F0240F02D0AAF1340603E0AAF175
:10266000170600E0761C00254FF0004406E05B1ED4
:1026700042F1FF3220EA030521EA0204CAF1010017
:10268000B04206DA1B4903980843019000200090ED
:102690000EE0039AC4F3D321E80A0A43164940EA3C
:1026A00044500A433146CDE90002684606F015FF62
:1026B000159810F0240F0BD01598C00715D1386865
:1026C000DDE90012031D3B600068C0E900120CE068
:1026D00002A8694606F0F8FE1598C00705D13868CB
:1026E000029A011D3960006802604046F0E6000071
:1026F00002FCFFFF0000F07F0000F03F2DE9FF4FDC
:1027000092461D4685B04FF00041DDE9124BDDE9F0
:1027100014727F1E01EA4B50414940F0FF4940EAE4
:102720000108002122F020004928049102D04E28FF
:1027300028D04CE03BA0012607C88DE80700A96916
:102740000698641C88477F1E014606D41DF80600C3
:1027500018B121F0200181420BD0E9690698884721
:10276000032E34D0082E32D06FF0010009B0BDE83E
:10277000F08F761C032E01D0082EE0D1601CCAF821
:102780000000DCE7A9690698641C88477F1E2AD4EC
:1027900020F02000412826D1A9690698641C8847AA
:1027A0007F1E20D420F020004E281CD1A969069855
:1027B000641C88477F1E48F4002849F48009CAF841
:1027C000004001D4282806D0E969069888475FEAC6
:1027D000CB7012D022E0A9690698641C88477F1E3E
:1027E00001D4002803DAE96906988847BCE729285C
:1027F000F1D1641CCAF80040E9E71BF0240F07D0B0
:1028000028680499031D2B600068C0E9001805E0E2
:102810002868021D2A600068C0F800902046A5E7DD
:102820000000F07F494E46494E49545900000000CF
:1028300010B50446AFF300802046BDE81040FDF718
:1028400070BD002801D006F059BE704710B50021B8
:1028500002A000F066F8012010BD00005349474176
:102860004252543A2041626E6F726D616C20746501
:10287000726D696E6174696F6E0000004FF0013C0B
:1028800050F8042B51F8043B9A4221D1A2EB0C03DF
:10289000934313EACC1317D150F8042B51F8043B9F
:1028A0009A4215D1A2EB0C03934313EACC130BD13C
:1028B00050F8042B51F8043B9A4209D1A2EB0C03C7
:1028C000934313EACC13DBD04FF00000704700BFF6
:1028D000D01A01BAB1FA81F101F0180122FA01F01F
:1028E000CB40C1F12001DBB2C0B2C01A2CFA01F317
:1028F000D11A914311EAC311E6D17047B2F1200316
:102900000AD5C2F1200301FA02F120FA03F300FA1A
:1029100002F041EA0301704700FA03F14FF00000B2
:10292000704770B505460C460A2000E06D1CFEF7A6
:102930007BFE35B128780028F8D102E0641CFEF750
:1029400073FE14B120780028F8D1BDE870400A2049
:10295000FEF76ABE5FEA400C08BF91F0000F4FEA35
:102960008C234FEAC12243EA51514FEA1C5018BF51
:1029700000F5F0404FEA300018BF41F000415FEA37
:102980006C5C00F02980BCF1FF3F08BF40F0804044
:102990007047130C06BF12044FF0100C4FF0000CE0
:1029A000130E04BF12020CF1080C130F04BF120126
:1029B0000CF1040C930F04BF92000CF1020CD30F26
:1029C00004BF52000CF1010C11464FF00002A0F1BF
:1029D0001F00A0EB0C00704711F0004F08BF7047BC
:1029E00031F000413FF4D5AF0B0C06BF09044FF0A6
:1029F000100C4FF0000C0B0E04BF09020CF1080C78
:102A00000B0F04BF09010CF1040C8B0F04BF8900EC
:102A10000CF1020CCB0F04BF49000CF1010CCCF1FE
:102A20002003A0EB0C0022FA03F302FA0CF241EAB5
:102A3000030100F10100704720F07F4C80EA0300A1
:102A400023F07F47ACEB070303F57C5300F0004015
:102A500003F1FF032DE980494FEA154B09B44FEA12
:102A6000144325EA0B4E24EA03480FF2042606EB32
:102A7000132749083E785FEA320203FB0667C7F571
:102A8000000707FB06F64FEA54374FEAD64606F131
:102A9000020607FB066CCCF1005C4FEA1C472CEAEF
:102AA000074C07FB06F40CFB06F504EB15464FEA52
:102AB000961634BF00204FF000404FEAD13706FB96
:102AC00007FC4FEA1C4C0CFB0BF7D21B03FB0CF76B
:102AD00061EB07010CFB0EF7B0EB074072EB1742FE
:102AE0000CFB08F734BFA2EB0742B2EB074261EBE5
:102AF00017414FEA0C444FEA910706FB07FC4FEAE7
:102B00001C4C0CFB0BF7B0EBC74072EB573203FBCE
:102B10000CF734BFA2EBC742B2EBC74261EB5731AF
:102B20000CFB0EF7B0EBC70072EB57720CFB08F70B
:102B300034BFA2EBC702B2EBC70261EB5771039F30
:102B40004FEA816141EA921104EBCC044FEAD1379C
:102B50004FEA826206FB07FC42EA90124FEA80606D
:102B60004FEA1C4C0CFB0BF7D21B03FB0CF761EB81
:102B700007010CFB0EF7B0EB074072EB17420CFBA2
:102B800008F734BFA2EB0742B2EB074261EB1741F3
:102B90004FEA8C554FEA910704EB9C2406FB07FC97
:102BA0004FEA1C4C0CFB0BF7B0EBC74072EB5732F3
:102BB00003FB0CF734BFA2EBC742B2EBC74261EB99
:102BC00057310CFB0EF7B0EBC70072EB57720CFBE2
:102BD00008F734BFA2EBC702B2EBC70261EB577133
:102BE00015EB4C254FEA816141EA92114FEA82626E
:102BF0004FEAD13742EA901206FB07FC44F1000489
:102C00004FEA80604FEA1C4C0CFB0BF7D21B03FB16
:102C10000CF761EB07010CFB0EF7B0EB074072EB12
:102C200017420CFB08F734BFA2EB0742B2EB074296
:102C300061EB174115EB1C154FEA813141EA9241D6
:102C40004FEA823242EA90424FEA80304FEA0C76F5
:102C500044F1000448EA03434EEA0B484FF0000EEB
:102C6000B2EB080C71EB030724BF624639464EEB0A
:102C70000E0E4FF0000B0018524149414BEB0B0B6D
:102C8000B2EB080C71EB03077BF1000B24BF62462B
:102C900039464EEB0E0E4FF0000B001852414941E1
:102CA0004BEB0B0BB2EB080C71EB03077BF1000B4A
:102CB00024BF624639464EEB0E0E51EA020718BF9A
:102CC00046F0010616EB0E7655F1000254F10001B4
:102CD00003D5BDE88901BDE80088BDE88901BDE8EC
:102CE0000048B619524141EB0101A3F101037047BD
:102CF00080807F7E7D7C7B7A797877767675747339
:102D0000727171706F6E6E6D6C6C6B6A6A696868F7
:102D1000676666656464636362616160605F5F5E8D
:102D20005E5D5D5C5C5B5B5A5A5959585857575603
:102D30005655555554545353525252515150505068
:102D40004F4F4F4E4E4D4D4D4C4C4C4B4B4B4A4ABA
:102D50004A494949484848474747474646464545FE
:102D60004544444444434343434242424241414137
:102D700046EA0646A3F570534FEA164646EA42561F
:102D80004FEAD22242EA415210B54FEAD121A3F1D3
:102D9000010300F02FF820F0004000F1020C00F0D9
:102DA000004701EB00501146BCF5006F40EA0700F8
:102DB00000D210BDBAF1000F0AD01CB503B44FF019
:102DC00004004FF004014FF000000FBCBDE81040BC
:102DD0004FF00001BBF1010FB9BF04484FF0FF31C4
:102DE0000348002140EA070010BD00BFFFFFEF7F4E
:102DF0000000F07F002B9C4630D477002BD01CB510
:102E00004FEA370703B44FF010004FF01001BAF14A
:102E1000000F06D0BCF1000FDCBF40F0080040F00E
:102E200008014FF000000FBCBDE810400BF1010B92
:102E3000BBF1010F08BF5FEA170722BF12F10102C1
:102E400011F101014FF0004143F1000300F0004097
:102E500043EA00007047F9D35708D0E746EA064630
:102E600013F1400F4FEA16461FDD13F1200FDFBFAD
:102E700016430A46002120335B42BED0C3F120072F
:102E800046EA064602FA07F74FEA164646EA0706FA
:102E9000C3F1200722FA03F201FA07F721FA03F13E
:102EA0004FF0000342EA0702A7E746EA020646EAB5
:102EB00006464FEA164646EA0106BCBF46EA064603
:102EC000360C4FF000034FF000024FF0000194E782
:102ED0002DE9804C9A46934670B491E8380007C8B3
:102EE00031EA400C48BF34EA430C03D5FFF7A4FD98
:102EF000FFF780FFF0BCBDE8008C2DE9804C9A46BE
:102F0000934670B491E8380007C831EA400C48BFD6
:102F100034EA430C03D5FFF78FFDFFF729FFF0BC20
:102F2000BDE8008C2DE9804C9A46934670B491E838
:102F3000380007C810F0804F08BF13F0804F03D14E
:102F400000F01AF8FFF756FFF0BCBDE8008C2DE941
:102F5000804C9A46934670B491E8380007C810F048
:102F6000804F08BF13F0804F03D100F005F8FFF742
:102F7000FFFEF0BCBDE8008C20F07F4780EA030034
:102F800023F07F4C07EB0C03A3F57C5300F00040CB
:102F9000A3F1FE0392F0000F00F0B38095F0000F54
:102FA00000F077802DE901494FEA11404FEA1446BD
:102FB00021EA004800FB06FC24EA064708FB06F667
:102FC00007FB08F800FB07F718EB06484CEB164C1C
:102FD0004FEA124B18EB07484FEA15464CEB1740E7
:102FE00022EA0B4E0BFB06FC25EA06470EFB06F613
:102FF00007FB0EFE0BFB07F71EEB064E4CEB164CC9
:103000004FF000061EEB074E4CEB174B18EB0B086E
:1030100040F1000018EB0E0B58EB000840F10000E7
:103020008F1A4FF000013CBFC943661B14BFB5EBBC
:10303000040C00213CBFC943F61B4FEA17444EEA7B
:103040008E0E27EA04454FEA1C4704FB07622CEA70
:10305000074C05FB07F70CFB05F604FB0CFC16EB15
:10306000074642EB174216EB0C4642EB1C421BEBA9
:10307000060658EB0202414146EA9E0601D5BDE82C
:103080000189B619524141EB0101A3F10103BDE8E9
:1030900001894FEA14454FEA114724EA054621EA1F
:1030A000074C05FB07F406FB07F70CFB06F105FBD5
:1030B0000CFC11EB074144EB17444FEA124711EBAC
:1030C0000C4144EB1C4422EA074C05FB07F206FBCB
:1030D00007F70CFB06F605FB0CFC16EB074642EB6C
:1030E000174216EB0C4642EB1C456A1854F10001DE
:1030F00048BF7047B619524141EB0101A3F10103EA
:10310000704795F0000F37D04FEA11424FEA14474D
:1031100021EA024624EA074C02FB07F106FB07F707
:103120000CFB06F402FB0CFC14EB074441EB1741CB
:103130004FEA154714EB0C4441EB1C4125EA074CC0
:1031400002FB07F506FB07F70CFB06F602FB0CFC7F
:1031500016EB074645EB174516EB0C4645EB1C42B4
:10316000121951F1000148BF7047B619524141EBA5
:103170000101A3F1010370474FEA14454FEA1147DB
:1031800024EA054621EA074C05FB07F106FB07F791
:103190000CFB06F24FF0000605FB0CFC12EB07429D
:1031A00041EB174112EB0C4251EB1C4148BF7047F9
:1031B000921841EB0101A3F10103704721484FF040
:1031C000FF010170002080F309881F48016881F326
:1031D00008881E484FF08051016062B6FEE71B4828
:1031E0004FF080510160704718484FF080510160E6
:1031F000704772B6EFF3098050B11EF0100F08BF90
:1032000020ED108A734620E9F80F1149096808601B
:1032100000B5104880475DF804EB0F480F490A7865
:1032200002700B480E490A6802601068B0E8F80F97
:103230009E461EF0100F08BFB0EC108A80F309887C
:1032400062B6704722ED00E04000001004ED00E09F
:1032500038000010815B02082200001023000010DB
:103260003C00001070B51E484BF68C1281684FF47C
:103270008040914202DA03F019FD01E003F08CFA7C
:10328000184C00252079E8B1D4F8800006F038F910
:1032900068B11548056004F11C0006F075FC07F0E4
:1032A000B9FB206807F0BAFA206006F033FAD4F8C8
:1032B0008000B0F5007F01D044280FD1BDE87040F8
:1032C00006F028BB4FF47A71022001F00FFF6572FF
:1032D00006F020FBBDE8704007F0A3BB70BD000006
:1032E000AC3900206C1B0120C0000020652802D0F2
:1032F000662802D003E000207047612902D06628CA
:1033000002D003E003207047632902D0662802D070
:1033100003E0042070476D2902D0622802D003E048
:1033200001207047612902D0622802D003E0052005
:103330007047632902D0622802D003E0062070475C
:103340006D2902D0662802D003E0022070476C2964
:1033500002D0622802D003E0072070476C2902D017
:10336000662802D003E009207047722902D0622843
:1033700002D003E008207047722902D04FF0FF30DE
:1033800070470A20704770B5054600234FF6FF705E
:103390004AF203040EE0EA5C50400022C60702D065
:1033A00084EA500000E04008521C92B2082AF5D38B
:1033B0005B1C9BB28B42EEDB70BD08B56A460821F0
:1033C0000A2002F0DFFBF9E72DE9F0478AB08146D9
:1033D00041480024032500780DF12408052815D163
:1033E00005944FF48070CDE90645CDF82080CDE9F5
:1033F00003041921394ACDE9012102200090374800
:103400000023374A37A1683802F092FACDE9064521
:1034100039480190059404204FF480666627CDF862
:1034200020800090CDE90276334804940023334A8B
:1034300033A1683802F07CFA05947000CDE90645A6
:10344000CDF82090CDE90304CC21334ACDE9012108
:103450000920009030480023304A31A1683802F03A
:1034600067FA07200594CDE90708334806944FF022
:10347000080ACDE900A0CDE9027600232F4A30A149
:103480000494683802F054FACDE9064530480190BA
:1034900005940520CDF820800090CDE902762C48D7
:1034A000049400232B4A2CA1683802F041FACDE99C
:1034B00006452F480594CDE900A0CDF82090CDE930
:1034C000027600232B4A2CA10494683802F030FACB
:1034D0000AB0BDE8F08700000000001008010010ED
:1034E000C3350208417070205461736B20466565D6
:1034F00064446F670000000070050010A9350208E1
:10350000417070205461736B2045746865726E65FC
:10351000742053657200000040260010D93502085F
:10352000417070205461736B204D6F74696F6E2011
:10353000436F6E74726F6C00A8460010BB330208B4
:10354000417070205461736B2043414E00000000B5
:10355000D81500108D350208417070205461736BCE
:103560002045746865726E657420436C69000000C4
:1035700010570010E7350208417070205461736BDA
:1035800020537065656420437472000008B5054CD3
:1035900006F078F8C4F8BC006A4608210A2002F058
:1035A000F1FAF5E76C1B012008B503F0F3FB06F018
:1035B000DFFC06F073FC6A4608210A2002F0E2FAFA
:1035C000F5E708B506F09FF800F0FEFF6A46002117
:1035D0000A2002F0D7FAF7E708B56A4608210A2060
:1035E00002F0D0FAF9E708B504F0A2FC6A46082117
:1035F0000A2002F0C7FAF7E71FB5684603F02EF875
:10360000019804B010BD000010B5FFF7F5FF09499F
:103610000968B0FBF1F0401EB0F1807F09D24FF095
:10362000E0214861044AF0201070002088610720E2
:10363000086110BDD8C8020823ED00E038B5304C51
:1036400004F51E6194F87E0B082843D00FDC012896
:103650000CD0022819D003281FD0042806D10091CD
:10366000002104230122084600F0A8FE38BD0B28E3
:1036700028D0212836D02728F8D1009100212723EF
:103680000122084600F09AFE38BD00910021022375
:103690000122084600F092FE38BD0091002103236C
:1036A0000122084600F08AFE1648D0F8801016A0C5
:1036B00002F040FF0022009006231146012000F096
:1036C0007DFE38BD012200910B231146002000F041
:1036D00075FE38BD0091082301220221002000F070
:1036E0006DFE38BD0091002121230122084600F023
:1036F00065FE04F5386403CCBDE8384006F0D0BA66
:10370000680901206C1B012025303478000000007E
:10371000FEE70000F0B58BB006460121084602F036
:1037200073FF0121480602F07DFF4FF4C05009905D
:1037300002208DF8280000248DF82A4003208DF8FF
:10374000290001258DF82B502C4F09A9384600F08F
:103750004DFF09220B21384600F086FF09220C217B
:10376000384600F081FF8DF81E408DF81F408DF81F
:1037700020408DF821508DF822408DF823408DF89F
:103780001A408DF81B4006208DF81C0005208DF88E
:103790001D00ADF818601A4E06A9304600F07EFAFA
:1037A0008DF812408DF813408DF81450ADF8084094
:1037B000ADF80A40ADF80C40ADF80E40ADF8104041
:1037C0008DF8155002A800F08FF901220221304631
:1037D00000F05AFA14208DF8040008208DF8050036
:1037E0008DF806408DF8075001A801F013FF054839
:1037F000048044808480C4800BB0F0BD000002408F
:1038000000640040D890001010B586B0FCF7B4FDFD
:10381000044601F0C3FF2046FCF7B2FD084C02212C
:10382000204600F0CBF920B101AA0021204600F08B
:10383000B7FA00200190029001F0C0FF06B010BD61
:103840000064004010B5FCF797FD044601F0A6FFA8
:103850002046FCF795FD174C0121204600F000F9A9
:103860000121204600F0AAF901280CD001212046B0
:1038700000F0A4F901280BD00121204600F09EF9A8
:1038800001280AD00DE00121204600F0E9F808E007
:103890000121204600F0E4F803E00121204600F079
:1038A000DFF800220121204600F0EEF9BDE81040CB
:1038B00001F084BF00640040F0B58BB006460121E2
:1038C000022002F0A1FE01214FF0C06002F0AAFE2A
:1038D0006020099002208DF8280000248DF82A40ED
:1038E00003208DF8290001258DF82B502D4F09A9B3
:1038F000384600F07BFE09220521384600F0B4FE70
:1039000009220621384600F0AFFE8DF81E408DF8E2
:103910001F408DF820408DF821508DF822408DF801
:1039200023408DF81A408DF81B4006208DF81C00AE
:1039300005208DF81D00ADF818601B4E06A9304615
:1039400000F0ACF90E208DF812008DF813408DF8C0
:103950001450ADF80840ADF80A40ADF80C40ADF891
:103960000E40ADF810408DF8155002A800F0BCF8DC
:1039700001220221304600F087F940208DF8040032
:1039800007208DF805008DF806408DF8075001A836
:1039900001F040FE0548048044808480C4800BB060
:1039A000F0BD0000000402400068004028910010B3
:1039B00010B586B0FCF7E0FC044601F0EFFE2046AF
:1039C000FCF7DEFC084C0221204600F0F7F820B19D
:1039D00001AA0021204600F0E3F9002001900290A6
:1039E00001F0ECFE06B010BD0068004010B5FCF719
:1039F000C3FC044601F0D2FE2046FCF7C1FC174C84
:103A00000121204600F02CF80121204600F0D6F8D4
:103A100001280CD00121204600F0D0F801280BD05D
:103A20000121204600F0CAF801280AD00DE001214A
:103A3000204600F015F808E00121204600F010F8BB
:103A400003E00121204600F00BF80022012120466E
:103A500000F01AF9BDE8104001F0B0BE0068004067
:103A600030B5082310240422B1F5007F33D011DCD7
:103A700020292AD007DC012922D0042923D00829B3
:103A800000D1C46030BD402921D0B1F5807FF9D18B
:103A9000426030BD0025B1F5004F20D008DCB1F503
:103AA000806F1AD0B1F5006FF3D18561426030BDEF
:103AB000B1F5803F0DD0B1F5003FF8D1446030BD85
:103AC0000849816030BDC36030BD036130BD046111
:103AD00030BD436030BD426030BD426030BD856165
:103AE000426030BD01010100F0B5827A01219140B0
:103AF000304C226842F0010222602E4D1C352A68AB
:103B00008A432A602B4A067B0C322B4B002E14D1A1
:103B100016688E4316604688C78846EA0746877A45
:103B200003EBC707C7F840660688878846EA07465A
:103B3000877A03EBC707C7F84466067B012E14D1CA
:103B400016680E4316604288068842EA0642867A64
:103B500003EBC606C6F84026C288868842EA0642BB
:103B6000867A03EBC603C3F84426124AC37A121DB1
:103B70003BB113680B4313600E4A0389143223B11F
:103B800006E013688B431360F6E713688B431360FA
:103B90000389012B02D113680B431360407B01287A
:103BA00002D1286808432860206820F001002060C6
:103BB000F0BD0000006600400060004002460020AA
:103BC00053690B425DD0B1F5807F4AD016DC0829DD
:103BD00037D009DC01292CD002292ED0042950D15C
:103BE000D068082100F084BB10292ED0202930D0C5
:103BF000402946D11069102100F07ABBB1F5004F81
:103C00003BD00CDCB1F5007F2FD0B1F5806F30D008
:103C1000B1F5006F35D19069702100F069BBB1F545
:103C2000803F1AD0B1F5003F2BD15068102100F031
:103C30005FBB9068134900F05BBBD068032100F0C4
:103C400057BBD068102100F053BB1069032100F06E
:103C50004FBB1069082100F04BBB5068082100F0F1
:103C600047BB9069012100F043BB9069022100F03D
:103C70003FBB9069042100F03BBB5068042100F079
:103C800037BB704701010100002A03D042690A4393
:103C90004261704742698A434261704710B5002211
:103CA000036823F002030360036843F00103036029
:103CB0004FF6FF7300E0521C4468E40701D19A42BA
:103CC000F9D14268D2073ED08A79012A3DD00268F4
:103CD00022F080020260CA79012A3BD0026822F0F9
:103CE000400202600A7A012A39D0026822F02002DA
:103CF00002604A7A012A37D0026822F0100202607C
:103D00008A7A012A35D0026822F008020260CA7A53
:103D1000012A33D0026822F0040202608A78CC784B
:103D2000920742EA04620C7942EA04424C7909881B
:103D300042EA0452491E0A43C261016821F00101AE
:103D40000160002120E0002010BD026842F08002E6
:103D50000260C0E7026842F040020260C2E7026807
:103D600042F020020260C4E7026842F010020260E2
:103D7000C6E7026842F008020260C8E7026842F043
:103D800004020260CAE7491C4268D20701D0994286
:103D9000F9D14068C00701D0002010BD012010BD3E
:103DA00010B500EB0113D3F8B04104F00404147211
:103DB000002C2CD0D3F8B041E408546003F5D8733C
:103DC0001C6804F0020454725C6804F00F049472DE
:103DD0005C68240AD4749C68D4729C68240A1473A6
:103DE0009C68240C54739C68240E9473DC68D47310
:103DF000DC68240A1474DC68240C5474DB681B0E21
:103E0000937449B1016941F02001016110BDD3F8FB
:103E1000B041640D1460D1E7C16841F02001C16078
:103E200010BD10B500F016F8BDE8104000F010B855
:103E300010B5FCF7A1FA04461021044801F0C2FBBA
:103E40002046BDE81040FCF79BBA00001067001048
:103E5000FFF7EEBF02490020086000F009B800003B
:103E600014000010014908607047000014000010A1
:103E700010B5FFF7C1FB08490A6842F080720A607A
:103E8000064900224A600A6842F001020A60BDE861
:103E90001040FFF7E7BF0000FCED00E0001000E07D
:103EA00070B52DED088BB0EE408A4FF0FF369FEDD8
:103EB000890A894D78EE40BA9FED889B38EE00BAAA
:103EC0000124DFED888AE86908F0FAFB41EC1A0B5F
:103ED00018EE100A08F0F4FB41EC100B04F040FB64
:103EE00053EC1A2B51EC100B08F0B8F823D2B5EEB6
:103EF000C08AF1EE10FA0EDD18EE100A08F0E0FBB1
:103F000041EC100B04F02CFB51EC100B07F0DEFD24
:103F100008EE900AD4E0344618EE100A08F0D0FB00
:103F200041EC100B04F01CFB51EC100B07F0CEFD24
:103F300008EE900AC4E0E86908F0C2FB41EC1A0BF5
:103F40001BEE900A08F0BCFB41EC100B04F008FBE0
:103F500053EC1A2B51EC100B08F080F823D218EE1A
:103F6000100A614988420EDD1BEE900A08F0A8FB9A
:103F700041EC100B04F0F4FA51EC100B07F0A6FD25
:103F800008EE900A9CE034461BEE900A08F098FB7D
:103F900041EC100B04F0E4FA51EC100B07F096FD25
:103FA00008EE900A8CE0E86908F08AFB41EC1A0BF5
:103FB00018EE100A08F084FB41EC100B04F0D0FA64
:103FC00053EC192B51EC100B08F090FA41EC100B4C
:103FD00004F0C6FA53EC1A2B51EC100B08F03EF823
:103FE00037D2B5EEC08AF1EE10FA19DD344618EE7C
:103FF000100A08F065FB41EC100B04F0B1FA53EC29
:10400000192B51EC100B08F071FA41EC100B04F075
:10401000A7FA51EC100B07F059FD08EE900A4FE09B
:1040200018EE100A08F04CFB41EC100B04F098FA63
:1040300053EC192B51EC100B08F058FA41EC100B13
:1040400004F08EFA51EC100B07F040FD08EE900AD8
:1040500036E0E86908F034FB41EC190B1BEE100A5E
:1040600008F02EFB41EC100B04F07AFA53EC192BFC
:1040700051EC100B07F0F2FF22D218EE100A1B4988
:1040800088420ED21BEE100A08F01AFB41EC100B0E
:1040900004F066FA51EC100B07F018FD08EE900AD8
:1040A0000EE034461BEE100A08F00AFB41EC100B40
:1040B00004F056FA51EC100B07F008FD08EE900AD8
:1040C00000EE104AB8EEC00A20EE280ABDEC088BBC
:1040D00070BD00000000B442BC02002000000000DF
:1040E00000806640000000000000B4420000B4C23E
:1040F00030EE600A0849DFED090A10EE100A884226
:1041000001D330EE200A064910EE100A884201DB86
:1041100030EE600A70470000DA0F49C0DA0FC9407C
:10412000DA0F494010B52DED060B2DED048B9FEDF8
:104130001D0A9DED041ADDED070A9DED089ADDEDDF
:10414000059AB4EE601AF1EE10FA0ED1B4EEE99AC7
:10415000F1EE10FA05DD9FED140ABDEC048B06B0FC
:1041600010BDFAD29FED110AF7E730EEC10A10EE4A
:10417000100A08F0A5FA39EE690A41EC180B10EEA6
:10418000100A08F09DFA41EC100BB0EE481AF0EE60
:10419000681A04F0EDF851EC100B07F097FC00EEF4
:1041A000100ADAE700000000DA0FC93FDA0FC9BFD2
:1041B0002DE9F84F044600250095464EDFF818A17A
:1041C0004FF0010830784FF4C877002807D13946FE
:1041D0005046FCF7D4FC757086F80080B580232C1F
:1041E0000CD035817078DFF8F4904FF0020B052881
:1041F0006ED2DFE800F06A140D280D0086F8018009
:104200003089401C80B230810128EBD1B580E9E7CC
:1042100039465046FCF7B3FC86F80180B580202C67
:1042200009D0B088B84206D2411C484400F500507D
:10423000B18080F8504D5A2C23D0F580B088B84218
:1042400043D386F801B0B08842F648514844084448
:104250006A4623A1FCF768FAB088083801B25046D4
:10426000FFF791F801460098814213D090B139468A
:104270005046FCF784FCB58086F801B0232C1FD093
:1042800023E0F088401C80B2F08002281DD103207A
:104290007070D8E739461448FCF771FC5146124853
:1042A000FCF792FB39465046FCF769FC0E48FCF7D8
:1042B000C4FB0E49C1F8780BB5800420707004E08F
:1042C00039465046FCF75BFCB5807078BDE8F88F46
:1042D000FEE70000F4020020B8C600206899002024
:1042E0002530347800000000D897002068090120AC
:1042F000024600200A4200D0012070472DE9F0411B
:104300002A4D022085F87C0B302085F87E0B28484A
:1043100000F0F0F90024274E274F04EB840006EB51
:1043200080013846FCF774FB80B3022C32D0641C49
:10433000E4B2032CF1D300241E4E1F4F3C36283F1D
:1043400004EB840006EB80013846FCF761FB18B3F0
:10435000032C24D0641CE4B2042CF1D30024154EA9
:10436000154F8C36283704EB440000EBC40006EBF5
:1043700040013846FCF74CFB98B1302C14D0641C3B
:10438000E4B2312CEFD30020BDE8F081FFE785F8DF
:104390007C4BD0E70220F7E785F87D4BDEE7032072
:1043A000F2E785F87E4BEEE70720EDE7680901208C
:1043B000B8C600200403002098C800202DE9FE4361
:1043C000DDF8288007460E4615461C464FF4C87196
:1043D0002B48FCF7D4FB2B48828E1AB12AA12C481B
:1043E000FBF7F2FF2A4904EB440000EBC400503114
:1043F00001EB4000CDE9000805EB85008C3901EBAD
:10440000800306EB86003C3101EB800221A11C48B1
:10441000FBF7DAFF1A48FCF710FB01B21848FEF769
:10442000B2FF024621A102A8FBF7CEFF02A9144861
:10443000FCF722FB1248FCF700FB0246104906205D
:1044400003F0C6FC0E48FCF7F8FA024604EBC40081
:10445000194D00EB041005EB001000F5F56008495C
:10446000FCF75BFB281900F5A04080F8387405EBD9
:10447000840000F5A0400021C0F86C14BDE8FE8364
:10448000349600206C1B01202530345800000000B9
:104490004003002023232C2C25732C2C25732C2C3B
:1044A00025732C2C25732C2C00000000253034782B
:1044B0002C2C5A5A00000000343A002070470000AB
:1044C00010B505A1012003F0CBFABDE810404FF470
:1044D000807000F039B800003C2A2A2A2A2A2A2AA9
:1044E0002A2A2A2A2A2A2A2A2A2ABFAAC6F4B1A3B1
:1044F000B4E60D0A000000003EB502F029F80121E3
:10450000880302F09DF80821012002F087FB4FF498
:104510008070009000258DF804500C208DF8050067
:1045200001248DF80640684600F014F817208DF835
:1045300008008DF8095002208DF80A008DF80B4014
:1045400002A801F067F83EBD01490860704700000D
:10455000143C014030B51B4A83790168002B2AD0F6
:1045600013688B431360111D0B680468A3430B6031
:10457000017911440B68046823430B60114C083423
:104580002168036899432160231D19680568A943C0
:1045900019604179102905D011440A680068024366
:1045A0000A6030BD21680268114321601968006803
:1045B0000143196030BD0079104402688A430260EB
:1045C00030BD0000003C014007480068064900F08B
:1045D0007F00091D096801F07F01884202D27F2017
:1045E00003F0D4BB70470000002C00402DE9F041DF
:1045F000002201274FF0030C07FA02F50B682B404D
:10460000AB422CD1066853000CFA03F4A6430660B3
:104610000E79D0F800809E4046EA080606600E79C2
:10462000012E01D0022E12D18668A64386604E79F3
:10463000D0F808809E4046EA080686604668AE4389
:10464000466045688E799640B6B235434560C56888
:10465000A543C560CC799C40C3681C43C460521C10
:10466000102AC9D3BDE8F08110B54B07DB0E9A4084
:10467000C90800EB8100016A0F249C40A14301623C
:10468000016A1143016210BD0246002012690A420C
:1046900000D001207047000010B51C280CD207493B
:1046A000064AA03A31F8101052F82000FFF7ECFF4C
:1046B000002800D0012010BD002010BD64010020A2
:1046C000418370470183704714280FD2084AA2F132
:1046D000700329B132F8101053F82000FFF7F2BF31
:1046E00032F8101053F82000FFF7EABF70470000BF
:1046F000240200202DE9F041044604F58045002005
:10470000C5F8200E24A12548FCF758F9064617E005
:10471000D5F8200E042818D000EB800004EBC00070
:1047200000F5C87032461EA1FBF74EFED5F8200EEC
:10473000401CC5F8200E18A10020FCF73FF90646E2
:10474000002EE5D10020BDE8F0814FF4C87704F5D4
:10475000486039468046FCF712FA324610A14046BE
:10476000FBF732FED5F8200E0EA200EB800004EB22
:10477000C00000F5C8700AA1FBF726FE44F6904081
:10478000204439460646FCF7FAF93A464146304697
:10479000FCF7C3F9CAE700002C2C0000D8970020D2
:1047A000257300003000000070B58EB004460E4640
:1047B0001546342101A8FCF7E2F93046FCF73DF933
:1047C0000246314601A8FCF763F900202070294613
:1047D00001A8FCF7F3F8024610E020780AA1C0EB2C
:1047E000001004EB4000401CFBF7EEFD2078401C5D
:1047F000207029460020FCF7E1F80246002AECD19F
:104800000EB0002070BD0000257300002DE9F84FA8
:1048100081460024002644F62461002041F8090066
:104820004FF4C87504EB840009EBC00000F561602B
:104830002821FCF7A4F9641CA4B2AC42F2D37DA1F8
:1048400009F54860FCF7BAF802460FE006EB86006F
:1048500009EBC00000F5616077A1FBF7B5FD75A11C
:104860000020FCF7ABF80246761CB6B2002AEDD168
:10487000754872A10546FCF7CBF8DFF8D0A170B9F6
:1048800000240AE004EB4400C0EB44100AEBC00033
:10489000E821FCF774F9641CA4B2B442F2D36C486A
:1048A0000090C0F8C06165A12846FCF7B1F808B1D6
:1048B0000024A8E0674890F8930001287ED105F015
:1048C0009FF9654846604FF0000870E00098C0F816
:1048D000C46108EB880009EBC00108EB4800C0EB9D
:1048E000481B0AEBCB0401F561615CA22046FFF78F
:1048F0005BFF0025584808EB480100EBC107C5EBFA
:10490000051004EB4000401C0A220021FBF7DDFFEC
:1049100004EB8501C1F8D80000EE100A07EB850012
:10492000B8EEC00A80ED030A6D1CADB2022DE6D3CD
:104930001AF83B00401EC0EB001004EB4000401C86
:10494000FBF7B6FF38761AF83B00801EC0EB00106C
:1049500004EB4000401CFBF7ABFFF8611AF83B008A
:1049600004F180010246001FC0EB001004EB400080
:10497000B0F80100A4F8D300D01EC0EB001004EB87
:104980004000B0F80100A1F8550094F8D510702946
:104990001AD071291CD0002087F8200094F8D30089
:1049A000FEF7A4FC788308F101081FFA88F8B045E7
:1049B0008CD32849002081F8930000E025E04FF4D3
:1049C000127001F0E9FE20E0012087F82000E5E701
:1049D000022087F82000E1E721A12846FCF718F81B
:1049E000B0B104EB840009EBC00000F561600A225D
:1049F0000021FBF76AFF0AEB840101F5E041C1F8F1
:104A0000800B641CA4B2B442E6D30020BDE8F88F4A
:104A100004EB840009EBC00000F561601022002166
:104A2000FBF753FF0AEB840101F5E041C1F8800B6D
:104A3000E7E700003A3A0000257300007365746CE4
:104A4000726F757400000000C0C8002068990020D3
:104A5000681901206C1B0120988F00205F00000066
:104A600073657474697073002DE9F05F2DED028B2E
:104A700001258B4EDFF82C82DFF82CA23078DFF88E
:104A80002C92DFF82CB200279FED8A8B8B4C0028EC
:104A900002D0012857D0E5E08948D0ED022A90EDF8
:104AA000012AD0ED001A874890ED021AD0ED010AD4
:104AB00090ED000AFFF736FB88ED090A9AED021A1D
:104AC000F0EE400AB0EE410AFFF712FB10EE100ABA
:104AD00007F0F6FD41EC100B03F042FD9FED7A1B51
:104AE00051EC100B53EC112B07F0F4FA06F0EEFF2B
:104AF000206227607770D9F8040007F0E1FD41ECEF
:104B0000100B03F02DFD53EC182B51EC100B07F09C
:104B1000A5FA17D2DBF8040007F0D2FD41EC100B28
:104B200003F01EFD53EC182B51EC100B07F096FA16
:104B300008D267490868421C0A60B0F57A7F01DD37
:104B400035700F608EE0207F032801D004281AD131
:104B5000D8ED090A9AED020AFFF7CAFA86ED080AAB
:104B6000D8ED090A9AED020AFFF7C2FA10EE100A10
:104B700007F0A6FD41EC100B03F0F2FC51EC100B1A
:104B800006F0A4FFF06196ED070A524910EE100AF4
:104B9000884205DBDFED500A30EE600A86ED070A39
:104BA00096ED070A4D4910EE100A884202DB642098
:104BB000206027E010EE100A49490844494988421C
:104BC0000ED29FED492AF3EE0E1A9FED481ADFED43
:104BD000480A05F004FFBDEEC00A84ED000A11E0AA
:104BE00010EE100A3E49C94388420ADD96ED080AD4
:104BF000D6ED090A20EE200AB5EEC00AF1EE10FA51
:104C000000D2757096ED080A86ED090A70780128C1
:104C100028D19FED380A86ED090A2760D9F80400EB
:104C200007F04EFD41EC100B03F09AFC53EC182BEF
:104C300051EC100B07F012FA11D2DBF8040007F068
:104C40003FFD41EC100B03F08BFC53EC182B51ECA7
:104C5000100B07F003FA02D22748807D50B1D4F838
:104C6000BC00B062B7EE080ABDEC028BBDE8F05F95
:104C700006F072BAD4F8BC00B16A401AB0F5FA7FF7
:104C8000F0D9207F032801D00428EBD1A07D1B4957
:104C9000401E00EB400001EBC00045833770E1E7A8
:104CA0008C0200202C1C0120DC1C0120AC390020CF
:104CB000C039002000000000000014406C1B0120DF
:104CC000D01C0120C41C01206666666666A64C40A6
:104CD000C0020020DA0FC940DA0FC9409A99993E04
:104CE000703D0AC30AD7A3010000C8429A99993EB1
:104CF0008FC2F53C00000000EC390020988F0020A6
:104D000070B5204D204C206807F0DAFC41EC100B08
:104D100003F026FC9FED1D1B51EC100B53EC112BE7
:104D200007F0D6FA08D8B5F918002860BDE8704039
:104D3000B6EE000A06F010BA206807F0C1FC41EC9C
:104D4000100B03F00DFC51EC100B06F0BFFE00EE53
:104D5000100AB5F91800DFED0F1A00EE900A9FED6A
:104D60000E1AB8EEE02ADFED0D0A05F038FEBDEEB2
:104D7000C00A85ED000ABDE870409FED090A06F003
:104D8000EBB900006C1B01202C1C012033333333A2
:104D90003333D33F0000C8429A99993E0000000087
:104DA000CDCC4C3E70B52DED048B8148D0ED022A60
:104DB00090ED012AD0ED001A7E4890ED021AD0ED58
:104DC000010A90ED000A02F0FFF9B0EE408A18EEF9
:104DD000100A7949794C88421CDDE06807F070FCC4
:104DE00041EC100B03F0BCFBB0EE409AF0EE609A81
:104DF00018EE100A07F064FC53EC192B07F076FB51
:104E00009FED6F1B53EC112B07F070FB06F05EFE5D
:104E1000206115E0E06807F053FC41EC100B03F053
:104E20009FFBB0EE409AF0EE609A18EE100A07F081
:104E300047FC53EC192B07F059FB06F047FE2061A5
:104E4000614D297F687F814203D1B5F91800286040
:104E500068E0072815D0082813D0092811D00A289F
:104E60000FD0288F94ED040A00EE900AF8EE600A45
:104E7000B4EEE00AF1EE10FA2CDBB5F91800286068
:104E800050E0288F94ED040A00EE900AF8EE600AD4
:104E9000B4EEE00AF1EE10FA03DBB5F91800286071
:104EA00040E0B5F9181000EE901AB5F91A10B8EEF6
:104EB000E02A00EE901AF8EEE01A00EE900AB8EE42
:104EC000601ADFED420A05F08AFDBDEEC00A85EDED
:104ED000000A27E000EE900AF8EE600AB4EEE00A5D
:104EE000F1EE10FA1CD810EE101A394A914217DD73
:104EF000B5F9181000EE901AE98EB8EEE02A00EE2F
:104F0000901AF8EE601A00EE900AB8EE601AF3EE0E
:104F10000E0A05F064FDBDEEC00A85ED000A01E051
:104F2000E88E28602B49E0682B4E2C4C884237DAFB
:104F300096ED010AD4ED010A30EE600A10EE100A77
:104F400007F0BEFB41EC100B03F00AFB9FED241BA6
:104F500051EC100B53EC112B07F0BAF918D296ED67
:104F6000010AD4ED010A30EE200A10EE100A07F013
:104F7000A7FB41EC100B03F0F3FA9FED1B1B51EC68
:104F8000100B53EC112B07F0A5F807F021F828605F
:104F90009FED170ABDEC048BBDE8704006F0DCB84D
:104FA000BDEC048BB7EE080ABDE8704006F0D4B83B
:104FB000D01C0120C41C012000401C462C1C0120D8
:104FC00000000000000079406C1B01200000000080
:104FD0000000F04100009643AC390020C0390020A9
:104FE0000000000000003440000000000000E03F2E
:104FF0009A99993E2DE9F0412AA30021344C585C3E
:10500000A08022885206FCD5491CC9B22A29F6D3B1
:105010007F2002F0BBFE02F023FE2E490878401CE0
:10502000C0B2087001283AD82B4F40F22556002212
:105030003146384602F0F7FA40F227750022294639
:10504000384602F0F0FA00223146204602F0EBFA30
:1050500000222946204602F0E6FA204C0022314682
:10506000204602F0E0FA00222946204602F0DBFA50
:105070001B4C00223146204602F0D5FA0022294678
:10508000204602F0D0FABFF34F8F16490868164A3F
:1050900000F4E06010430860BFF34F8FFEE7BDE807
:1050A000F08100000D0A456E7465722048617264DB
:1050B0004661756C745F48616E646C65722C205338
:1050C000797374656D2048616C742E0D0A000000C0
:1050D0000010014011000010001401400044004085
:1050E000004800400CED00E00400FA0510B504464D
:1050F0000846002803D000F0D5FA604300E02046BF
:10510000C0B2082875D2DFE800F00412202E3C4A15
:10511000586600210420FFF7D7FA00210620FFF788
:10512000D3FA0021BDE810400520FFF7CDBA0021D9
:105130000420FFF7C9FA01210620FFF7C5FA002174
:10514000BDE810400520FFF7BFBA00210420FFF79B
:10515000BBFA00210620FFF7B7FA0121BDE8104095
:105160000520FFF7B1BA01210420FFF7ADFA0021B5
:105170000620FFF7A9FA0021BDE810400520FFF73F
:10518000A3BA01210420FFF79FFA01210620FFF7AF
:105190009BFA0121BDE810400520FFF795BA0121D7
:1051A0000420FFF791FA00210620FFF78DFA012174
:1051B000BDE810400520FFF787BA01210420FFF762
:1051C00083FA01210620FFF77FFA0021BDE8104095
:1051D0000520FFF779BA00210420FFF775FA0121B5
:1051E0000620FFF771FA0121BDE810400520FFF706
:1051F0006BBA00210420FFF767FA00210620FFF7B1
:1052000063FA0021BDE810400520FFF75DBA10B534
:1052100020287ED2DFE800F07D101E2C3A4856642C
:105220007282909EACBAC8D6E4FDFCFBFAF9F8F79E
:10523000F6F5F4F3F2F1F0EF00210846FFF744FA37
:1052400001210846FFF740FA0121BDE81040022085
:10525000FFF73ABA01210020FFF736FA00210120BA
:10526000FFF732FA0121BDE810400220FFF72CBA07
:1052700000210846FFF728FA00210120FFF724FA51
:105280000121BDE810400220FFF71EBA01210020D5
:10529000FFF71AFA01210846FFF716FA0021BDE8C8
:1052A00010400220FFF710BA00210846FFF70CFA61
:1052B00001210846FFF708FA0021BDE8104002204E
:1052C000FFF702BA01210020FFF7FEF900210120BB
:1052D000FFF7FAF90021BDE810400220FFF7F4B90A
:1052E00000210846FFF7F0F900210120FFF7ECF953
:1052F0000021BDE810400220FFF7E6B9012100209F
:10530000FFF7E2F901210846FFF7DEF9012102204B
:1053100000E055E1BDE81040FFF7D6B901210020BB
:10532000FFF7D2F900210120FFF7CEF90121BDE8F6
:1053300010400220FFF7C8B900210846FFF7C4F962
:1053400001210846FFF7C0F90121BDE81040022005
:10535000FFF7BAB901210020FFF7B6F9012108468D
:10536000FFF7B2F90121BDE810400220FFF7ACB908
:1053700001210020FFF7A8F901210846FFF7A4F951
:105380000021BDE810400220FFF79EB90021084629
:10539000FFF79AF900210120FFF796F90121BDE8F6
:1053A00010400220FFF790B901210020FFF78CF98F
:1053B00000210120FFF788F90121BDE810400220FB
:1053C000FFF782B900210846FFF77EF90121084660
:1053D000FFF77AF90121BDE810400220FFF774B908
:1053E00001210020FFF770F901210846FFF76CF951
:1053F000012102200EE0D5E0C6E0B7E0A8E099E088
:105400008AE07BE06CE05DE04EE03FE030E021E0F0
:1054100012E003E0BDE81040FFF756B9012100207B
:10542000FFF752F901210846FFF74EF90021BDE8C8
:1054300010400220FFF748B900210846FFF744F961
:1054400000210120FFF740F90121BDE810400220B2
:10545000FFF73AB901210020FFF736F900210120BA
:10546000FFF732F90121BDE810400220FFF72CB907
:1054700000210846FFF728F901210846FFF724F923
:105480000121BDE810400220FFF71EB901210020D4
:10549000FFF71AF901210846FFF716F90121BDE8C7
:1054A00010400220FFF710B901210020FFF70CF98E
:1054B00001210846FFF708F90021BDE8104002204D
:1054C000FFF702B900210846FFF7FEF8002101208E
:1054D000FFF7FAF80121BDE810400220FFF7F4B809
:1054E00001210020FFF7F0F801210846FFF7ECF852
:1054F0000121BDE810400220FFF7E6B80021084670
:10550000FFF7E2F801210846FFF7DEF80121BDE8C8
:1055100010400220FFF7D8B801210020FFF7D4F88F
:1055200000210120FFF7D0F80121BDE81040022042
:10553000FFF7CAB800210846FFF7C6F8002101208E
:10554000FFF7C2F80121BDE810400220FFF7BCB808
:1055500001210020FFF7B8F801210846FFF7B4F851
:105560000021BDE810400220FFF7AEB80021084638
:10557000FFF7AAF801210846FFF7A6F80021BDE8C9
:1055800010400220FFF7A0B801210020FFF79CF88F
:1055900000210120FFF798F80021BDE8104002200B
:1055A000FFF792B800210846FFF78EF8002101208E
:1055B000FFF78AF80021BDE810400220FFF784B809
:1055C00010BDFEE70A460021AFF3008010B5002AA7
:1055D0001ED000281CD0002300241B020B43641C97
:1055E000042CFAD300F0030424B909E000F8011BED
:1055F000521E641C22B1042CF8D301E008C0121F13
:10560000042AFBD202E000F8011B521E002AFAD144
:1056100010BD704730B50F23C27801250178002AEC
:105620001FD0154A126802F4E062C2F5E062C2F3CC
:105630000722C2F10404D3404278A24084781C407F
:105640001443220101F1E02181F80024007800F0E8
:105650001F018D404009800000F1E020C0F800519A
:1056600030BD01F01F0085404809800000F1E020B6
:10567000C0F8805130BD00000CED00E00249084345
:1056800002490860704700000000FA050CED00E0D8
:10569000024A1140014302480160704780FFFF1F2A
:1056A00008ED00E00749084AD1F8BC105368CB1A4E
:1056B000834204D95160107880F001001070107896
:1056C000704700006C1B01205C020020704770478F
:1056D00010B5044600F050F81C48002303701C4825
:1056E00003701C4803701C4803601C4803601C487E
:1056F00003701C4803701C4803701C48016841B1CA
:105700001B49096829B1026801E0521E08C1002A3C
:10571000FBD11848037000F0DDFB00F007FC2046C9
:1057200000F0ACFC208800280FD1204600F0A8FA39
:105730002088002809D1204600F0A0FE20880028FB
:1057400003D1BDE81040FFF7C1BF10BD200000101D
:105750002100001025000010380000103C0000104F
:10576000220000102300001024000010D0C80208FE
:10577000CCC802082E0000100548064900680968D8
:1057800000EB8100044920F007000860704700002A
:10579000CCC80208D0C802084000001005480078B4
:1057A000012805D104490878FA2801D2401C087064
:1057B00070470000210000102000001010B52048A4
:1057C000007801283AD1FAF7D7FD04461D49087838
:1057D00040B1401EC0B2087048B12046BDE810403C
:1057E000FAF7CEBD2046BDE81040FAF7C9BD16480D
:1057F000007820B12046BDE81040FAF7C1BD00F0A6
:1058000057FB12490870124900EB400051F8200084
:105810001049086010490968884204D12046BDE853
:105820001040FAF7ADBD0D480168491C0160FDF755
:10583000DBFC2046BDE81040FAF7A2BD10BD000019
:10584000210000102000001025000010230000108F
:10585000087000103C0000103800001028000010F4
:1058600010B515480078002825D114480078002884
:1058700021D1FAF781FD044600F01AFB10490870A7
:10588000104900EB400051F820000F4908600F4913
:105890000968884204D12046BDE81040FAF770BD7F
:1058A0000B480168491C0160FDF799FC2046BDE8E2
:1058B0001040FAF765BD10BD200000102500001053
:1058C00023000010087000103C0000103800001089
:1058D0002800001070B504460F4D2878002803D02A
:1058E00045F68A60208070BD00F0E2FA0B4908702E
:1058F0000B4908700B4900EB400051F820000A49A1
:1059000008600A49086001202870FDF757FC43F63B
:105910009920208070BD000021000010230000109D
:1059200022000010087000103C0000103800001029
:105930002DE9FF4F83B00446DDE910A8DDE91765C6
:10594000139F9346BAF10F0F08D13348844205D014
:1059500046F27320288007B0BDE8F08F204600F0A3
:1059600099FB4FF00009A5F80090F0070AD0B007A6
:1059700008D54546002003E0C5F800902D1D401CC9
:10598000B842F9D3129808EB8005CDE900762B4692
:1059900042465846069900F0BBF8C4F828B006996C
:1059A000E1620499216284F837A02060A56015980F
:1059B000606516986060C4F82480A763A6870020FD
:1059C00004EB8001C1F85C90401CC0B20028F7D005
:1059D000204600F027F8FAF7CFFC054694F8370088
:1059E00000F084FA204600F0E9FA0C490888401CCF
:1059F00008800B480078012805D007B02846BDE88C
:105A0000F04FFAF7BDBC2846FAF7BAFC07B0BDE87C
:105A1000F04FFFF725BF0000A06F00102C00001012
:105A200021000010704770472DE9F05F83468A46D9
:105A300014461D464FF00008002C01D0C4F8008029
:105A4000FAF79AFC0646DFF8B890D9F80000476CE0
:105A500067B17F1E47640CB1006C20603046FAF7D6
:105A60008FFCA5F800803846BDE8F09F5FEA0A4049
:105A700007D53046FAF784FC46F2B01028800020A3
:105A8000F2E72048007838B13046FAF779FC46F65C
:105A9000635028800020E7E700215B460722084684
:105AA00000F022F93046FAF76BFCFFF7D9FEFAF75F
:105AB00063FCD9F8002092F8351069B1012911D0A2
:105AC000032916D046F62E612980D9F800104C6CB7
:105AD000FAF756FC2046C7E70CB1116C2160A5F817
:105AE0000080F2E70CB1116C216046F2A911298007
:105AF000EBE70CB1C4F8008047F2D9212980E4E734
:105B000038000010250000101346002200F010BBE2
:105B100010B5029C02EB840222F007024FF0807461
:105B200042F8044C42F8080C0C3A14481060A2F1F8
:105B300034004FF0123404634FF00332C2624FF06E
:105B400002328262436201624FF01131C161D100C1
:105B5000816161104161910001614FF00731C160C5
:105B60004FF0063181604FF005314160510040F83F
:105B700004196FF00201016010BD000011610208FC
:105B8000704700002DE9F04107460D4614461C48B9
:105B90000078002804D046F663502080BDE8F081EC
:105BA0004DB1022D07D0042D06D0082D03D045F6A7
:105BB00025602080F2E79FB1FAF7DEFB8046114EA8
:105BC0000121306880F8361023462A46394600F015
:105BD00021FB208840B14046BDE8F041FAF7D0BB38
:105BE00047F27E202080D9E7306800F003FA404673
:105BF000FAF7C6FBFFF734FE00202080CEE7000056
:105C0000250000103800001070B50546FAF7B4FB07
:105C100003490C68FAF7B4FB00202880204670BDC9
:105C20003000001008B500F009F86A46002102486B
:105C3000FFF76AFF08BD0000C87000107047000041
:105C400010B5FAF799FB064A1178491C1170FAF75A
:105C500097FBFFF7E7FFBDE81040FFF7AFBD00007F
:105C600020000010054CFAF787FB2168491C2160D1
:105C7000FAF786FBFFF72BFDF5E700001C0000108C
:105C800000B589B00D4A002111600B22CDE9061242
:105C900008900C4A05910A480B4B126800681B6873
:105CA000CDE90132CDE903010F2000900023074A1E
:105CB00007A10C48FFF73CFE09B000BD1C00001016
:105CC000C8C80208C4C80208C0C80208655C020847
:105CD00075432F4F532D4949492049646C65205421
:105CE00061736B00A06F00102DE9F0410C46074670
:105CF00019460E4D286880F83420002680F835605B
:105D000000F0A2F96CB104F10806FC6001223946EA
:105D1000286800F00DF839463046BDE8F04100F043
:105D20001AB82868C6870663BDE8F08138000010FD
:105D300010B5C28701630024002309E04B600B60AB
:105D40000B614B610B83CB6188602031641CA4B272
:105D50009442F3D310BD30B58A6892F83740028977
:105D60000025002A03D0521C028102680CE00122A7
:105D700002814D600D600160416030BD936893F811
:105D80003730A34202D85268002AF7D132B11368E3
:105D900053B10B604A605960116030BD4D6042687C
:105DA0000A605160416030BD11600D604A60016061
:105DB00030BD70B50646356BF48F07E0E8680830F3
:105DC000294600F009F82035641EA4B2002CF5D154
:105DD0000020F087306370BD10B502890024012ACD
:105DE0000BD00A6862B14B6873B153601A600289C4
:105DF000521E02814C600C6010BD04604460F6E7E6
:105E00004A6814600260F2E754604260EFE7F8B558
:105E1000064606980C46002594F83610082915D237
:105E2000DFE801F01414040414141B1B94F834105C
:105E300003290CD0206416B12046FFF7BAFF204694
:105E400000F056F93434A57065702570F8BD0090E7
:105E50002146304600F019F8EDE794F83410032994
:105E60000DD02064204600F04DFA16B12046FFF711
:105E7000A0FF04203434A07065702570F8BD009038
:105E80002146304600F001F8ECE770B5049D0C6B3C
:105E9000C98F0AE0E668864204D1206162612383EB
:105EA000E56170BD2034491E89B20029F2D170BD70
:105EB00010B50024064802E02034E4B2001D016859
:105EC0000029F9D00068FAF762FA2044C0B210BD88
:105ED000180000100020044A002142F82010401C45
:105EE0000028FAD07047000018000010410900F0A7
:105EF0001F020120C2F11F029040034B53F82120E2
:105F0000024343F82120704718000010410900F0B7
:105F10001F020120C2F11F029040034B53F82120C1
:105F2000824343F821207047180000100020074BDF
:105F3000002200EB400103EB81010A810A604A6004
:105F4000401CC0B21028F4D3704700000870001045
:105F500010B5044694F83700FFF7C8FF074994F8D6
:105F600037000978884204D12046BDE8104000F08F
:105F700025B82046BDE8104000F002B8220000100D
:105F800090F837100C4A01EB410102EB810100232C
:105F90000A89002A08D0521C0A810A68C26003617B
:105FA0000A6810610860704701220A81C3600361BA
:105FB00008604860704700000870001090F83710C3
:105FC0000B4A01EB410102EB810100230A89002AFF
:105FD00007D0521C0A81C3604A680261D0604860E1
:105FE000704701220A81C3600361086048607047FE
:105FF0000870001070B50446124994F8370000EBA1
:10600000400001EB80012069E2680025002808D0EB
:106010000B895B1E0B81C26092B110612561E56046
:1060200070BD2AB10889401E088115610A60F5E734
:106030000D810D604D6094F83700FFF767FFEDE7C5
:106040004860EBE70870001038B5044602250029C7
:106050000ED06B460222204600F0DCF8BDF80000AE
:1060600010B184F8365005E0032084F8360001E0D2
:1060700084F836502046FFF7BDFF38BD034A0021A3
:106080001180034A11600180704700002C0000104D
:10609000280000100022026082604260C26002613B
:1060A00042618261C26110A1016242628262C26287
:1060B0000264002100EB8103DA65491CC9B20029A2
:1060C000F8D03430026142600263C26202814FF054
:1060D000004141618261C2610262426202704270AB
:1060E00082701021C17070473F5461736B000000D3
:1060F00010B50446204600F005F994F8361049071B
:1061000004D42046BDE81040FFF722BF10BD0000B8
:1061100008B505480068FFF786FC044C6A46002174
:106120002068FFF72FFDF9E738000010D8C80208F3
:106130002DE9F8430446894615461E46FAF71CF930
:1061400007460CB92748046825640020308094F87D
:10615000360046F6C55808283BD2DFE800F00404B4
:10616000151504041515656C681C05D06D1C656457
:106170003846FAF705F933E03846FAF701F9A6F898
:1061800000800020BDE8F88394F83400072808D088
:10619000656C681C16D06D1C65643846FAF7F0F81B
:1061A0001EE000231A46214618460095FFF72FFEF1
:1061B000656C3846FAF7E4F85FEA094010D4FFF757
:1061C0004FFB0DE03846FAF7DBF8A6F80080002018
:1061D000D8E73846FAF7D4F846F62D603080002527
:1061E0002846CFE73800001010B500200022074BEA
:1061F000074C06E003EBC0010A608A80CA80401C9D
:1062000080B221888842F5D310BD0000206F0010B5
:10621000ECC80208F0B5384E002547F27E273468F6
:10622000042A08D099B33746082A3F680F4410D093
:10623000C76401651CE00A1B521E12F5803F04D999
:10624000C5640565C5611F80F0BDC164521C02654F
:106250000EE0826C0A44A2EB040CACF1010C8C45FC
:1062600001D2C26400E0C764C16C0A1B026581648C
:10627000224AC16C1288B1FBF2F402FB141189B2FC
:106280001F4A02EBC102918839B1116822E0FFE791
:10629000C5640565C5611F80F0BD456185611060FD
:1062A000012191801BE0CC6C3768E41B0C65076D05
:1062B000A74208D94C690CB121460BE045618161C8
:1062C0004861002106E08C698CB1846141616061A4
:1062D000886100210029E6D19188491C9180D488E9
:1062E00091888C4200D2D180C2611D80F0BD856151
:1062F000416188611060ECE730000010ECC80208D2
:10630000206F001010B5C169002915D00024046564
:106310000A68824204D142690A6032B1946104E0A1
:10632000836942695A6102B1936144618461C461C5
:10633000C4648888401E888010BD00002DE9F84F95
:10634000FAF71AF800904FF0000B3E4E3068401CF0
:1063500030603D490988B0FBF1F201FB120080B2C8
:106360003A4901EBC00004680025A8464FF0030934
:106370004FF0040A7CB3676994F8360008284FD2BE
:10638000DFE800F04E044E124E2A4E38E06C3168C1
:10639000421A2265884205D184F836802046FFF7EC
:1063A000A7FE3DE001253BE0E06C3168421A226522
:1063B00088420ED1C4F840802046FFF7FAFC204600
:1063C000FFF796FE84F8368084F8359084F83480A0
:1063D00026E0012524E025E0E06C3168421A2265C0
:1063E000884205D184F836A02046FFF78BFF17E0DE
:1063F000012515E0E06C3168421A226588420ED111
:10640000C4F840802046FFF7D4FC2046FFF77AFF0F
:1064100084F836A084F8359084F8348000E00125B3
:106420003C4600E00125002DA4D0CBF10000084936
:106430000A68824200D208600098BDE8F84FF9F778
:106440009FBF000030000010ECC80208206F001051
:10645000340000101CB5084C002101AB6A46084608
:10646000FFF7E2FABDF804000028F5D120780128F2
:10647000F2D1FFF763FFEFE72100001030B589B0DC
:1064800004461B48002505601A480560FFF7ACFE6E
:106490001948016851B11949194B0A681B689A4299
:1064A00008D247F21320208009B030BD47F21220F5
:1064B0002080F9E7134A13780F2B03D347F21120FA
:1064C0002080F1E70B23CDE90653059508940E4B88
:1064D000096800681B68CDE90315CDE90103107850
:1064E00000900023094A0AA10E48FFF721FADBE7D2
:1064F0003000001034000010E0C80208E8C80208AC
:10650000D4C80208DCC80208E4C8020855640208BE
:1065100075432F4F532D494949205469636B2054CB
:1065200061736B00C8700010014908627047000079
:1065300000000E420FB410B503AA04480299F9F7FF
:1065400031FF10BC01485DF814FB00000C3A00203C
:106550001CB50121022000F057F84FF48070009024
:1065600000208DF8040003208DF8050002208DF82E
:10657000070069460148FEF739F81CBD00040240D7
:1065800010B590B09FED160A8DED0F0A8DED0E0A35
:106590008DED0D0A00210C910B910A910991089142
:1065A0000AAB0BACCDE9034308A909AACDE9052143
:1065B0000DAA0EABCDE900320CA902910FAB094A2E
:1065C00009A1FAF7B1F80A98012807D105489DED0D
:1065D0000D0A1C3880ED040A0121017610B010BDAF
:1065E00000000000A83900203C256440282566787A
:1065F00025662925664025784025784025642D2587
:10660000642D25643E000000054A002903D011686E
:1066100001431160704711688143116070470000A9
:1066200030380240054A002903D011680143116047
:106630007047116881431160704700004038024084
:10664000054A002903D011680143116070471168A1
:1066500081431160704700004438024070B5244BFC
:10666000196801F00C01234C00291ED06610042982
:106670001DD008291DD00460196801F0F001090936
:106680001D4A545C0168E14041601C6804F4E05418
:10669000A40A145D21FA04F484601B6803F46043C7
:1066A0005B0BD25CD140C16070BD0460E4E7066062
:1066B000E2E70F4A121F1168C1F38055116801F01B
:1066C0003F0135B1B6FBF1F11468C4F3881461439E
:1066D00005E0B4FBF1F11468C4F388146143126857
:1066E000C2F30142521C5200B1FBF2F10160C3E758
:1066F000083802400024F4000100001070B5034681
:1067000000240020012B06D0022B06D0032B06D03C
:10671000062B06D070BD0F4B18E00F4B16E00F4B49
:1067200014E00F4B12E0B3F80058B3F80268B5421A
:10673000F0D0401CB3F802585D5D0D55B3F8025817
:106740006D1CC5F30905A3F80258641C9442EAD3F2
:1067500070BD00001E190020262100202E290020D7
:106760003631002070B50024094D002604EB84006A
:1067700005EBC0010748FAF74BF920B9281900F5D5
:10678000A04080F83864641CE4B2312CEED370BDB4
:10679000343A0020C497002002490A6882430A6004
:1067A00070470000EC1B01202DE9F0412DED048B1A
:1067B000EF4CB4F8420000EE100AF8EE400A9FEDEC
:1067C000ED1AED4D80EE810AD5ED020A30EE209AE9
:1067D000DFF8A88398F81600002805D198ED030A81
:1067E000FDF75EFB85ED060A98F8160000260128E5
:1067F00031D002282FD0A97809B130B32BE06079CD
:106800000121052809D006280DD0207F4FF47A7287
:1068100003280ED0042812D01DE0062088F81600A8
:10682000A9702E6317E0052088F81600A9702E6362
:1068300011E0042088F81600A9702A630BE00320F9
:1068400088F81600A9702A6305E0207F042802D08A
:10685000032800D0AE7098ED030AD5ED080A30EE9B
:10686000600A85ED0A0AD8ED010AF5EEC00AF1EEDC
:1068700010FA12D2B5EEC00AF1EE10FA06DDD5ED2F
:10688000060A30EE200A85ED0A0A1DE0D5ED060A5B
:1068900030EE600A85ED0A0A16E0F5EEC00AF1EE68
:1068A00010FA11DDB5EEC00AF1EE10FA06DDD5EDF5
:1068B000060A30EE600A85ED0A0A05E0D5ED060A03
:1068C00030EE200A85ED0A0A95ED0A0AAC4910EE71
:1068D000100ADFEDAC0A884203DD30EE600A85ED78
:1068E0000A0A95ED0A0AA84910EE100A884203D94F
:1068F00030EE200A85ED0A0A206A05F0E1FE41EC3F
:10690000180BA86A05F0DCFE41EC100B01F028FE24
:1069100053EC182B51EC100B05F0E8FD41EC100B7B
:1069200001F01EFE51EC100B05F0D0F800EE100A3D
:1069300085ED090A98F81600032805D0042803D02D
:10694000052801D006281DD110EE100A8F49884273
:1069500002DD85ED059A15E010EE100A8C4988429B
:106960000CDDB0EE492AD5ED031AB3EE0E1AF0EEA7
:10697000080A04F034F885ED050A03E095ED030AF2
:1069800085ED050A9FED838A2F6B6C68BC4232DB74
:10699000D5ED050A95ED0B0AF4EEC00AF1EE10FAFA
:1069A0000DDD10EE100A05F08BFE9FED7B1B53EC06
:1069B000112B05F0BDF805F089F868610DE00CD2E7
:1069C00010EE100A05F07CFE9FED751B53EC112BA9
:1069D00005F08CFD05F07AF8686195ED050AB5EED5
:1069E000C00AF1EE10FA01D285ED058A95ED050A8F
:1069F00085ED0B0A03E085ED0B8A85ED058A98F895
:106A00001600B3EE0E0ADFED680AFEEE002A9FEDD7
:106A1000671AF3EE0D1AB6EE002A07280BD2DFE84C
:106A200000F0040A0E2A4B6C890088ED018A98ED6B
:106A3000030A85ED080ABDEC048BBDE8F0819FEDEB
:106A40005C0A88ED010A286905F03AFE41EC190B51
:106A5000686A05F035FE41EC100B01F081FD53EC46
:106A6000192B51EC100B05F0F9FAE4D888ED018AE6
:106A700088F81660DFE7601C6860BC42DBDB95EDE0
:106A8000052A62EE200A60EEA20A80EE812A62EEFA
:106A9000210A80EE801A88ED011A95ED090AD5EDDC
:106AA000040AB4EEE00AF1EE10FAC4D26E6088ED8A
:106AB000018A88F81660BEE7601C6860BC42BADBD9
:106AC000D5ED052A62EEA00A60EE820A80EE812AE8
:106AD00062EE210A80EE801A88ED011A95ED090A0E
:106AE000D5ED040AB4EEE00AF1EE10FAA3D26E601E
:106AF00088ED018A88F816609DE795ED052A62EE1B
:106B0000200A60EEA20A80EE812A62EE210A80EE5F
:106B1000801A88ED011A95ED090AD5ED040AB4EE44
:106B2000E00AF1EE10FA86D26E6088ED018A88F8EC
:106B3000166080E7D5ED052A62EEA00A60EE820AB3
:106B400080EE812A62EE210A80EE801A88ED011A19
:106B500095ED090AD5ED040AB4EEE00AF1EE10FA5B
:106B600088D26E6088ED018A88F8166063E70000BD
:106B70006C1B012000006643BC020020EC390020A1
:106B8000000034430000B443000034C30000F0416F
:106B900000004040000000007B14AE47E17A743FE3
:106BA0007B14AE47E17A843F4095134ADA0F49409F
:106BB000005043C7002904D0018841F04001018002
:106BC0007047018821F04001018070470246002093
:106BD00012890A4200D00120704780897047818164
:106BE000704730B5028802F441530A884C88CD883A
:106BF00022438C882C4322430C8922434C89224314
:106C00008C892243CC8922431A430280828B22F44E
:106C100000628283098A018230BD704710B58A07FD
:106C2000120F0F23934021F003040649214401F67B
:106C300008010C689C430C600B68904003430B6098
:106C400010BD00000030014010B5124890F87C1BC8
:106C50001148002910D001291AD1FDF7D7FD0028CD
:106C600016D114210D48F9F78AFFBDE810400C4AEF
:106C70000CA10A48F9F7A8BBFDF7C8FD002807D109
:106C800009480079002803D0BDE81040FCF7D6BCC5
:106C900010BD000068090120B8C60020C49700207C
:106CA000C0C80020257300006C1B012002490A683F
:106CB00002430A6070470000EC1B01204FF4807112
:106CC0000148FDF7FDBC0000000802404FF4807150
:106CD0000148FDF7F7BC0000000802400CB5002297
:106CE000019200922749086840F4803008604FF410
:106CF000A043086800F4003000900198401C019007
:106D0000009810B901989842F3D10868800302D521
:106D10000120009000E000920098012831D119482C
:106D20004030026842F0805202601748026842F424
:106D3000404202601348083002680260026842F470
:106D400000420260026842F4A0520260021F0F4B30
:106D500013600A6842F080720A600A689201FCD5EA
:106D60000B4A40F205711160016821F003010160D6
:106D7000016841F0020101600168C1F3810102294B
:106D8000FAD10CBD003802400070004008544007A2
:106D9000003C024010B504F025F904F06DFA04F04F
:106DA000D1FA0549054803F0C3FFBDE81040044986
:106DB000044803F0ABBF000011B30208DDB20208C3
:106DC000859E0208919E020808489FED070A80ED03
:106DD000000A074880ED000A064880ED010A0648CF
:106DE00080ED010A7047000000000000AC3900206F
:106DF000C0390020D4390020EC39002005489FED2F
:106E0000040A80ED000A044880ED000A7047000083
:106E100000000000AC390020C03900202DE9F04707
:106E2000294F0026294DB878002819D0BE700024BB
:106E300004EB840005EBC0002821F9F7A0FE281917
:106E400000F5A04080F8386405EB840000F5A04010
:106E5000C0F86C64641CE4B2312CE9D3BDE8F0875F
:106E60000024DFF86C80281900F5A04090F8380461
:106E700028B3D8F8BC00F96840F2DC52411A9142BC
:106E80001DD3F8604FF4C87949461248F9F777FEE8
:106E900004EBC40000EB041005EB001101F5F561F3
:106EA0004A460C48F9F739FE4A460A49062000F0DE
:106EB0008FFF05EB840000F5A040C0F86C64641CF3
:106EC000E4B2312CCFD3C9E7F4020020343A0020D9
:106ED0006C1B01203496002010B51248016841F463
:106EE000700101601048016841F0010101600E4A23
:106EF00000210832116002680C4B1A400260031D29
:106F00000B4A1A60026822F48022026006480C30A4
:106F10000160FFF7E3FE03494FF00060803908602D
:106F200010BD000088ED00E000380240FFFFF6FED3
:106F30001030002410B5F9F71FFA0446FEF72EFCB6
:106F40002046F9F71DFA074C0121204600F0E5F82C
:106F500018B10121204600F0CFF8BDE81040FEF73F
:106F60002DBC0000000400407FB504460D46012101
:106F70000220FFF757FB0294ADF804500024ADF84F
:106F80000640ADF80C40124D01A9284600F0DEF88D
:106F90000121284600F0A4F801221146284600F0FD
:106FA000C8F81D218DF800100E218DF801108DF804
:106FB000024001218DF803106846FEF72BFB0121EA
:106FC000284600F09CF80021284600F0BCF87FBD60
:106FD0000004004010B5F9F7CFF90446FEF7DEFBD8
:106FE0002046F9F7CDF9074C0121204600F095F82D
:106FF00018B10121204600F07FF8BDE81040FEF7EF
:10700000DDBB00000008004010B5F9F7B5F90446F3
:10701000FEF7C4FB2046F9F7B3F9084C01212046DE
:1070200000F07BF828B10121204600F065F803F05C
:10703000D9FDBDE81040FEF7C1BB0000000C0040C8
:1070400010B5F9F799F90446FEF7A8FB2046F9F7C1
:1070500097F9074C0121204600F05FF818B1012193
:10706000204600F049F8BDE81040FEF7A7BB00003D
:10707000001400407FB504460D4601212020FFF793
:10708000D1FA0294ADF804500024ADF80640ADF8F2
:107090000C40124D01A9284600F058F8012128465D
:1070A00000F01EF801221146284600F042F8372170
:1070B0008DF800100E218DF801108DF8024001218D
:1070C0008DF803106846FEF7A5FA0121284600F066
:1070D00016F80021284600F036F87FBD0014004065
:1070E000002904D0018841F08001018070470188A7
:1070F00021F0800101807047C94301827047002957
:1071000004D0018841F0010101807047018821F01D
:10711000010101807047406A704702460020138ACF
:107120000B4092890A40002B02D0002A00D0012097
:107130007047002A03D082890A438281704782897E
:107140008A438281704741627047000030B50288EF
:10715000164C174DA0420DD0A8420BD0B0F1804F75
:1071600008D0144B984205D0134B984202D0134BD1
:10717000984203D122F070034A881A43104B984278
:1071800006D0104B984203D022F440730A891A4368
:1071900002804A68C2620A880285A04201D0A842E1
:1071A00001D1897A01860121818230BD0000014030
:1071B000000401400004004000080040000C0040B2
:1071C000001000400014004010B52DED060B2DED11
:1071D000048B9DED050ADDED080A30EE600A10EE25
:1071E000100A05F06DFA9FED1A9B41EC100BB0EE02
:1071F000491AF0EE691A01F027FAB0EE408AF0EE73
:10720000608A9DED040ADDED070A30EE600A10EE9B
:10721000100A05F055FA41EC100BB0EE491AF0EEE9
:10722000691A01F011FA53EC182B51EC100B04F011
:107230007FFC41EC100B02F02FF851EC100B04F026
:1072400045FCBDEC048B06B000EE100A10BD00003A
:1072500000000000000000402DE9F041F9F78CF833
:107260000446FEF79BFA2046F9F78AF8364D40F2BD
:107270002551284600F0B7F9344CB0B1284600F04B
:107280004BFAC1B2B4F80028521CC2F30900B4F89A
:107290000228904209D0B4F800082154B4F800083C
:1072A000401CC0F30900A4F8000840F227763146DC
:1072B000284600F098F940F2266700B3B4F80408B5
:1072C000B4F8061888420FD0B4F80618B4F80608C7
:1072D000401CC0F30900A4F80608601890F80014D8
:1072E000284600F01DFA2AE000223146284600F028
:1072F0009AF901223946284600F095F91FE03946EF
:10730000284600F070F9D0B1B4F80408B4F80618B3
:1073100088420FD0B4F80618B4F80608401CC0F331
:107320000900A4F80608601890F80014284600F038
:10733000F7F904E000223946284600F074F9BDE868
:10734000F041FEF73BBA0000001001401E1900207A
:1073500070B5F9F711F80446FEF720FA2046F9F760
:107360000FF8104C40F225552946204600F03BF915
:10737000012805D103F03CFC2946204600F018F90D
:1073800040F227752946204600F02DF9012805D145
:1073900003F034FC2946204600F00AF9BDE87040AD
:1073A000FEF70CBA004400402DE9F041F8F7E4FF85
:1073B0000446FEF7F3F92046F8F7E2FF364D40F2B7
:1073C0002551284600F00FF9344CB0B1284600F0A2
:1073D000A3F9C1B2B4F80028521CC2F30900B4F8F2
:1073E0000228904209D0B4F800082154B4F80008EB
:1073F000401CC0F30900A4F8000840F2277631468B
:10740000284600F0F0F840F2266700B3B4F804080C
:10741000B4F8061888420FD0B4F80618B4F8060875
:10742000401CC0F30900A4F80608601890F8001486
:10743000284600F075F92AE000223146284600F07F
:10744000F2F801223946284600F0EDF81FE03946EF
:10745000284600F0C8F8D0B1B4F80408B4F806180B
:1074600088420FD0B4F80618B4F80608401CC0F3E0
:107470000900A4F80608601890F80014284600F0E7
:107480004FF904E000223946284600F0CCF8BDE868
:10749000F041FEF793B90000004800402E2900207B
:1074A0002DE9F041F8F768FF0446FEF777F920462A
:1074B000F8F766FF3A4D40F22551284600F093F860
:1074C000384CB0B1284600F027F9C1B2B4F8002812
:1074D000521CC2F30900B4F80228904209D0B4F853
:1074E00000082154B4F80008401CC0F30900A4F8B7
:1074F000000840F227763146284600F074F840F242
:10750000266718B3B4F80408B4F80618884212D0F5
:10751000B4F80618B4F80608401CC0F30900A4F833
:107520000608601890F80044FFF7D0FB2146284673
:1075300000F0F6F82FE000223146284600F073F8FC
:1075400001223946284600F06EF824E039462846E4
:1075500000F049F8F8B1B4F80408B4F80618884205
:1075600012D0B4F80618B4F80608401CC0F309009D
:10757000A4F80608601890F80044FFF7A7FB21461E
:10758000284600F0CDF806E000223946284600F0F3
:107590004AF8FFF793FBBDE8F041FEF70FB9000092
:1075A00000140140363100208A05C943018070472C
:1075B00040F66A120A0A01219140C94301807047CE
:1075C000002904D0818941F400518181704781896B
:1075D00021F40051818170470246002012880A423E
:1075E00000D00120704770B5002440F66A12C1F344
:1075F000421301F01F05012606FA05F2012B0CD0FB
:10760000022B0DD0838A1340090A8E400088304037
:107610000BB100B10124204670BD83891340F3E70C
:10762000038A1340F0E710B540F66A13C1F3421322
:1076300001F01F040121A140012B07D0022B07D02C
:1076400014303AB102680A43026010BD0C30F8E70A
:107650001030F6E702688A43026010BD7FB5044629
:107660000D46208A20F44051E88808432082A089F2
:1076700041F20C618843A9882A8911436A8902432F
:107680001143A181A08A20F44071A8890843A082F7
:107690006846FEF7E3FF1E48844202D01D4884423C
:1076A00001D1039800E00298A189090408D500EBF4
:1076B000C00101EB001029684900B0FBF1F007E0C0
:1076C00000EBC00101EB001029688900B0FBF1F06C
:1076D0006422B0FBF2F109010B096FF018056B434E
:1076E00000EB8300A3891D044FF0320307D503EBA1
:1076F000C000B0FBF2F000F00700084306E003EB27
:107700000010B0FBF2F000F00F00084320817FBDB5
:1077100000100140001401408088C0F30800704749
:10772000C1F30801818070472DE9F04188B0074618
:1077300001212020FEF768FFDFF8F080202140467D
:10774000FCF7BEFF2020069001258DF81C50002478
:107750008DF81E4003208DF81D0002268DF81F6055
:1077600006A94046FCF742FF01210846FEF74CFF00
:1077700001211020FEF764FFDFF8B4800722092101
:107780004046FCF771FF07220A214046FCF76CFFD8
:107790004FF4C06006908DF81C608DF81D608DF868
:1077A0001E408DF81F5006A94046FCF71FFF2520FC
:1077B0008DF804008DF805408DF806408DF80750CF
:1077C00001A8FDF727FF0297ADF80C40ADF80E4079
:1077D000ADF81040ADF814400C20ADF81200154D76
:1077E00002A92846FFF73AFF012240F22551284618
:1077F000FFF719FF40F22776012231462846FFF7AE
:1078000012FF31462846FFF7CFFE40212846FFF7FA
:10781000CBFE09490C804C808C80CC80012128460D
:10782000FFF7CEFE08B0BDE8F08100000014024072
:1078300000000240001001401E210020F0B587B07A
:10784000064601210420FEF7DFFE01218804FEF731
:10785000E9FE234F07220A213846FCF705FF0722DD
:107860000B213846FCF700FF4FF4406005900221E1
:107870008DF818108DF8191000248DF81A40012584
:107880008DF81B5005A93846FCF7B0FE27208DF86F
:10789000000003218DF801108DF802108DF80350BF
:1078A0006846FDF7B7FE0196ADF80840ADF80A400E
:1078B000ADF80C40ADF810400C20ADF80E00094CAE
:1078C00001A92046FFF7CAFE012240F225512046B9
:1078D000FFF7A9FE01212046FFF772FE07B0F0BDB9
:1078E0000008024000480040F0B587B001210420A4
:1078F000FEF78AFE3A4F4FF4807421463846FCF773
:10790000DFFE059401258DF8185000248DF81A40EB
:1079100003208DF8190002268DF81B6005A9384652
:10792000FCF764FE01212020FEF78AFE08220621D2
:107930003846FCF799FE082207213846FCF794FEEA
:10794000C02005908DF818608DF819608DF81A40E8
:107950008DF81B5005A93846FCF748FE47208DF8E6
:1079600000008DF801408DF802408DF80350684604
:10797000FDF750FE4FF4E13001902803ADF8080008
:10798000ADF80A408010ADF80C00ADF810400C20A6
:10799000ADF80E00134D01A92846FFF75FFE012246
:1079A00040F225512846FFF73EFE40F2277601229D
:1079B00031462846FFF737FE31462846FFF7F4FDEB
:1079C00040212846FFF7F0FD07490C804C808C8051
:1079D000CC8001212846FFF7F3FD07B0F0BD000081
:1079E00000080240001401403639002070B5E4B0B0
:1079F0004FF4C87269460620FEF780FE0646300046
:107A000024D00025134C1FE094F8D00148B91DF88C
:107A100005001149FCF7CCFB042802D1012084F8B1
:107A2000D00194F8D00170B1FCF768FC08B9FFF7F9
:107A30000BF9002084F8D001084890F87C0B01284D
:107A400001D1FEF78FFE6D1CB542DDD3FFF7E6F9DD
:107A500064B070BD68190120B8C600206809012013
:107A60000FB410B5ADF5806D04460DF58262684621
:107A7000DDF80C14F8F796FC6846F8F7DEFF0246CE
:107A80006946204600F0A4F90DF5806D10BC5DF844
:107A900014FB00002DE9F04FBDB078221FA904208F
:107AA000FEF72CFE0746DFF89CA0274DDFF89CB0C0
:107AB00038004FF0000637D000240DF104084FF0D5
:107AC000010929E01FA8005D3C2802D03E2804D00F
:107AD00005E0EE61C5F8189001E00221A961E969AD
:107AE000642901DDAE61EE61A969012902D0022994
:107AF00006D010E0E9694A1CEA6108F801000AE0D2
:107B0000EA69511CE96108F8020001A8FEF738FD96
:107B1000AE618AF81990641CBC42D3D3DBF8BC0078
:107B200028623DB0BDE8F08FDBF8BC00296A411A3D
:107B3000B1F5FA7FF5D928628AF81960CAF81C6095
:107B4000EFE700008C390020640200206C1B01204C
:107B5000FEE7000070B505460B4CE06880476069A1
:107B60008047216A0F208847216AC5F3072088478C
:107B7000216AE8B28847E06980470546A1698847DD
:107B800021698847284670BD700000102DE9F0413A
:107B900080460E46174600240E4DE8688047686907
:107BA0008047296A0F208847296AC8F30720884739
:107BB000296A08F0FF00884704E0E86980473055EB
:107BC000641CA4B2BC42F8D3A86980472869BDE808
:107BD000F04100477000001070B505460E460C4C91
:107BE000E068804760698047226AF0209047226AF7
:107BF000C5F307209047226AE8B29047216A3046D1
:107C00008847A06980472069BDE8704000470000B0
:107C1000700000102DE9F04180460E461746002402
:107C20000E4DE868804768698047296AF0208847D8
:107C3000296AC8F307208847296A08F0FF008847A7
:107C400004E02B6A305D9847641CA4B2BC42F8D3B0
:107C5000A86980472869BDE8F0410047700000101E
:107C60000149002008607047082C0040024940F09C
:107C70008000086070470000002C0040014901208E
:107C800008607047A480054270B57F2000F07EF840
:107C9000FFF7E6FF21494878401CC0B24870012830
:107CA0003BD81F4E40F22555002229463046FFF7AB
:107CB000BAFC40F22774002221463046FFF7B3FC9D
:107CC000184E002229463046FFF7ADFC002221461F
:107CD0003046FFF7A8FC144E002229463046FFF735
:107CE000A2FC002221463046FFF79DFC29460F4D9D
:107CF00000222846FFF797FC002221462846FFF77E
:107D000092FCBFF34F8F0A4801680A4A01F4E06110
:107D100011430160BFF34F8FFEE770BD9C00001060
:107D200000140140001001400044004000480040A1
:107D30000CED00E00400FA05F8B505460E461746BE
:107D40000121C802FEF76EFC0F4C2078054025701B
:107D5000384600F023F8304600F02AF82078FFF784
:107D600085FF00208DF800008DF801008DF80200DD
:107D700001208DF803006846FDF74CFCFFF770FF0B
:107D8000FFF77CFFF8BD00009C000010024900F0E6
:107D90007F00086070470000002C0040034A116813
:107DA00021F4C0710143116070470000042C0040B1
:107DB00008B506490A6822F07F020092009A00F096
:107DC0007F00104300900098086008BD042C00401C
:107DD000F0B401280FD0022810D0032811D00628B3
:107DE00037D11D4B1D48B3F80448B3F80658AC42D0
:107DF0000AD1012709E01A4B1A48F4E71A4B1B482D
:107E0000F1E71B4B1B48EEE70027002403F58066D3
:107E100015E0B3F80458B3F806C86D1CC5F309059E
:107E200065450ED00D5DB3F804C80CF80650B3F8E4
:107E300004586D1CC5F30905A3F80458641C94424A
:107E4000E7D3002F05D0F0BC012240F22771FFF7E5
:107E5000EABBF0BC7047000036310020001401403E
:107E60001E1900200010014026210020004400407F
:107E70002E2900200048004070B50020FCF70CFCC3
:107E8000264D274C80F00100287020710120FCF75E
:107E900003FC80F00100687060710220FCF7FCFBBD
:107EA00080F00100A870A0710620FCF7F5FB80F0BF
:107EB0000100A87120700720FCF7EEFBE871E0706C
:107EC0000820FCF7E9FB287260700920FCF7E4FB4E
:107ED0006872A0700A20FCF7DFFB6873E0726278BA
:107EE000603C01210AB184F8841020B10E489FED56
:107EF0000D0A80ED030A94F862200C484AB1D4F8C8
:107F0000BC20436BD21A40F6B8339A4200D30170BA
:107F100070BDD4F8BC10416370BD0000441B01204B
:107F2000CC1B012000000000D4390020BC0200203E
:107F300010B5FFF7AFFD02F07BFD4FF47A7002F051
:107F40000DFF0949487920B9087F032801D004288A
:107F500001D107208882087DFDF759F9FFF746FD1A
:107F6000BDE81040FBF77EB96C1B012003B40198FB
:107F70004100009850EAC12018BF04204A0D18BFE4
:107F800040F0010040F2FF72B2EB515F08BF40F0D9
:107F90000200012808BF052002B070470000000061
:107FA00030B52DED048B81B0B0EE408AF0EE608AE2
:107FB0006A4651EC180B02F067FB00989FED329B6C
:107FC0007E300090002821DC53EC192B51EC180B6B
:107FD00003F0C2FF1AD0002140F608004FF0000065
:107FE000044651EC180B03F071FD08EE100A40F640
:107FF000080004EA00014FF00000B5EEC08AF1EE7F
:1080000010FA04BF0220F8F7F6FD2DE00098FF28D3
:1080100030DB002108464FF0000000F4400553EC2F
:10802000192B51EC180B04F053F98CBF00240124D8
:108030000220F8F7E0FD9FED168A4DB1002C0CBF31
:108040004FF400004FF48000A84218BF9FED118A42
:10805000042108464FF00000002C01BFB1EE480A91
:1080600001B0BDEC048B30BDB0EE480A01B0BDECF0
:10807000048B30BD51EC180B03F028FD01B000EE6D
:10808000100ABDEC048B30BD0000000000000000B1
:108090000000807FFFFF7F7F70B59B482DED020BB6
:1080A0002DED068B079D25F00044A04218DC974873
:1080B000844202DC0AD1069840B19DED060BBDEC6E
:1080C000068B02B0BDE8704001F0BAB9002DCCBFFC
:1080D0009FED8F0B9FED900BBDEC068B02B070BD3A
:1080E0008F48A04215DD8F48A042D8BF4FF0FF3423
:1080F00058DD9DED060B51EC100BFFF737FF042800
:1081000008BF01F0D1F99DED060BBDEC068B02B066
:1081100070BD9DED060B51EC100B02F0A9FACDE9F4
:10812000060181489FED828BA0423CDD8248A0423F
:108130001FDD00249FED82AB9DED060B53EC1A2B47
:1081400051EC100B03F0F4FC9DED060B41EC190B08
:1081500053EC1A2B51EC100B03F0BCFF53EC182B13
:1081600004F0C4F953EC192B03F09EFDCDE9060190
:1081700049E09DED060B012453EC182B51EC100B3C
:1081800003F0D6FC9DED060B41EC190B53EC182BBC
:1081900051EC100B04F0AAF953EC192B03F084FDF9
:1081A000CDE906012FE06848A0421FDD02249FEDC3
:1081B000689B9DED060B53EC192B51EC100B03F053
:1081C00089FF53EC182B03F0B3FC9DED060B41EC3B
:1081D000180B53EC192B51EC100B04F087F953ECEE
:1081E000182B03F061FDCDE906010CE09DED060BB7
:1081F000032453EC102B9FED580B51EC100B03F0A4
:1082000053FDCDE906019DED060B53EC102B51EC0F
:10821000100B03F05FFF41EC180B53EC182B03F02D
:1082200059FF41EC190B4E480621B0EE490AF0EE19
:10823000690A784401F06DF853EC182B51EC100BDF
:1082400003F048FF41EC180B4648B0EE490AF0EE47
:10825000690A0521784401F05CF853EC192B51ECC4
:10826000100B03F037FF41EC100B51EC180B53ECE3
:10827000102B002C0EDA03F05BFC9DED061B53EC7B
:10828000112B03F027FF9DED061B53EC112B04F07F
:1082900055F835E003F04CFC9DED061B53EC112B1B
:1082A00003F018FF41EC100B2F48784400EBC4009A
:1082B00090ED001B51EC100B53EC112B04F016F950
:1082C0009DED061B53EC112B04F010F941EC100B43
:1082D0002648784400EBC40090ED001B51EC100BD5
:1082E00053EC112B04F02AF841EC100B002DA2BF27
:1082F000BDEC068B02B070BD51EC100B03F0DAFB45
:1083000041EC100B01E70000000010440000F07F7A
:10831000182D4454FB21F93F182D4454FB21F9BF7B
:108320000000DC3F0000203E0000F33F00000000A2
:10833000000000000000F03F0000E63F00000000E9
:10834000000000000000004000800340000000002A
:10835000000000000000F83F000000000000F0BF37
:108360005A490000104900009A4800005248000095
:1083700070B56B4E2DED040B2DED028B82B0DDF848
:108380001CC0DDE905235C422CF000411C4341EA9E
:10839000D474049D22F00040B44205D86C422C43B2
:1083A00040EAD474B4420BD99DED061B9DED040B3D
:1083B00002B0BDEC028B04B0BDE8704001F04AB8D9
:1083C000ACF14054A4F17F641C430BD0022404EAB6
:1083D000AC7444EAD27405439FED538B9FED542B4C
:1083E00007D015E09DED040B51EC100B01F042F9A4
:1083F00042E0002C11BF012C9DED040B02B0BDEC3E
:10840000028B04BF04B070BD022C38D0032C3BD0CB
:108410000B439FED491B9FED4A0B0AD0B14218D187
:10842000B04209D121F0804120F0804007910590B1
:108430000FE0002A15DA10E0434B7B44002C08BF04
:1084400093ED000B0DD0012C10D0022C17D0032C73
:108450001AD0B0421DD1002A03DAB0EE410AF0EE84
:10846000610A02B0BDEC028B04B070BD93ED000B4D
:1084700051EC100B03F01EFB41EC100BF1E7B0EEDA
:10848000480AF0EE680AECE7B0EE420AF0EE620A43
:10849000E7E7401A00153C28C8BF8DED000B19DC3A
:1084A000BCF1000FBEBF10F13C0F9FED290B8DED0D
:1084B000000B0FDB9DED060B53EC102B9DED040B19
:1084C00051EC100B03F0F0FB02F0D2F801F0D2F8FF
:1084D000CDE90001002C08BF9DED000BC1D0012C9F
:1084E00010D0022C9FED1C0B53EC102B9DED000BBC
:1084F00051EC100B0DD003F0F9FF53EC182B03F0E7
:10850000F5FFB9E7019880F0004001909DED000B68
:10851000A7E703F0EBFF53EC182B03F00FFFABE7DB
:108520000000F07F00000000182D4454FB2109409A
:10853000182D4454FB2109C0182D4454FB21F9BFC8
:10854000182D4454FB21F93F1248000000000000A0
:108550000000000000000000075C143326A6A13CC8
:108560002DED020B019820F0004001909DED000BD5
:1085700002B070470000000030B540F2FF742DEDEE
:10858000048BF0EE608A18EE901A85B0B0EE408A47
:108590009FED2B9B05468DED008B34EA115147D0A2
:1085A00053EC192B51EC180B03F0D6FC40D02A46A3
:1085B00051EC180B04F038F941EC180B18EE900A46
:1085C0008DED008B34EA10501CD053EC192B51EC7C
:1085D000180B03F0C1FC2BD10220F8F70CFB00F0C4
:1085E00063FF10EE901A18EE900A8DED020B8DEDE0
:1085F000008B61F31E0003909DED020B05B0BDECF6
:10860000048B30BD0220F8F7F6FA00F03DFF10EEC3
:10861000901A18EE900A8DED020B8DED008B61F330
:108620001E0003909DED020B05B0BDEC048B30BD28
:1086300005B0B0EE480AF0EE680ABDEC048B30BD20
:1086400000000000000000002DE9F04D2DED040BAE
:108650002DED0E8B96B0DDE92550279CDDF890A01E
:1086600025F0004624F00048BAF1000F14BF0121A4
:10867000002101EB4502FC4953184A1093422AD3CA
:10868000002814BF0123002303EB44030B44F749E4
:108690008B4220D358EA00019FEDF59B76D0DFF89E
:1086A000D8B35D4503D1BAF1000F05D188E0BAF126
:1086B000000F08BF002100D0012101EB450111F599
:1086C000001F08D8002814BF0121002101EB44013C
:1086D00011F5001F0BD99DED261B9DED240B16B047
:1086E000BDEC0E8B04B0BDE8F04D00F0B3BE00272A
:1086F000002DBCBFE149884521DAE1498845A8BF82
:1087000002271CDAC3451ADCDE4901EB2851142983
:1087100008DDC1F1340220FA02F101FA02F28242CC
:108720000DD108E058B9C1F1140228FA02F101FA9A
:1087300002F2424503D101F00101C1F1020756EAFC
:108740000A0124D1002C22DA002D18BF022F01D0FB
:10875000012F0AD00220F8F74EFA16B0BDEC0E8BAE
:1087600004B0BDE8F04D00F053BE0220F8F743FA24
:1087700000F04EFE51EC100B03F09CF941EC100B95
:1087800016B0BDEC0E8B04B0BDE8F08D18E09FED87
:10879000BEAB9FEDBF8B002871D1B848804522D178
:1087A00005F1804010F5801008BFBAF1000F07D026
:1087B000B3450ADC002CA8BF9DED260BE0DA0DE0E6
:1087C000B0EE490AF0EE690ADAE7002C06DA9DED10
:1087D000260B51EC100B03F06DF96FE0AE487844B6
:1087E00090ED000BCCE7D8454DD1002C48DA2EB1E6
:1087F00086423AD1BAF1000F42D126E0BAF1000F19
:1088000013D00220F8F7F7F900F03EFE8DED020BD1
:108810009DED240B8DED000B10EE900A039961F392
:108820001E0003909DED020BAAE78DED02AB9DEDBE
:10883000240B1AEE901A10EE900A8DED000B61F3E6
:108840001E0003909DED020B9AE78DED028B9DEDCE
:10885000240B18EE901A10EE900A8DED000B61F3C8
:108860001E0003909DED020B8AE709DA9DED240BB3
:1088700051EC190B53EC102B03F016FA1EE020E01C
:108880009DED240B7CE786421BDAB4F1804F0DD0BE
:10889000A4F10050B0F1FF5013D1002D11DB9DED7C
:1088A000240B51EC100B02F07BFD07E09DED240B37
:1088B00053EC102B51EC100B00F0C2BC41EC100B30
:1088C0005EE79DED240B51EC100B01F0D1FEBAF1E7
:1088D000000FCDE90E0142D19FED710B46B3A6F119
:1088E000E040B0F17F600CD05E4538D1002D00DA59
:1088F000A7B3022F0CBF01204FF0FF3003F097FB0E
:10890000DCE7002D01DD002C0DDA002D01DD002C4F
:108910001FDB002D16DA002C14DB012F08BF9FEDA2
:10892000620B3FF42DAFB0EE4A0AF0EE6A0A27E779
:10893000022F18BF002D0CD0012F0AD1002DFFF6F9
:108940001FAF06E0002DB8BF002C08DA012F3FF45E
:1089500017AFB0EE480AF0EE680A11E71BE00120FD
:1089600000EBE57050EA070115D0791EB0EE498A98
:10897000F0EE698A084308BF9FED4D8B4E480025F5
:10898000804570DD4D494E48884514DDB0420DDB11
:10899000002C19DB2FE00120F8F72DF916B0BDEC03
:1089A0000E8B04B0BDE8F04D00F05EBDB34502DCB7
:1089B000002C09DC1FE0864202DA002C1BDA03E0FF
:1089C0005E452BDD002C16DD0220F8F714F900F0CF
:1089D0005BFD8DED020B53EC1A2B51EC180B03F0E1
:1089E00079FBCDE900010399019861F31E00039022
:1089F0009DED020BC4E60220F8F7FDF800F054FDEF
:108A000010EE901A18EE900A8DED020B8DED008B92
:108A100061F31E0003909DED020BB1E69DED0E0B80
:108A200053EC192B51EC100B03F060FD9FED260B5E
:108A3000CDE9080153EC102B9DED080B51EC100B08
:108A400003F048FB9FED221B53EC112B03F076FC47
:108A50009DED081B53EC112B03F03CFB9FED1E1BFF
:108A600053EC112B3CE08CE0FFFF1F00FFFF0F00D9
:108A7000000000000000F03F0000F03F0000F07F29
:108A80000000404301FCFFFF000000000000F07FF9
:108A900000000000000000006E4400000000000024
:108AA0000000000000000080000000000000F0FF57
:108AB000000000000000F0BF0000E0410000F043B3
:108AC000FFFFEF3F00000000000000000000D03F6B
:108AD000555555555555D53F000000000000E03F65
:108AE00003F02CFC9DED080B41EC1A0B53EC102B02
:108AF00051EC100B03F0EEFA53EC1A2B03F0EAFAE8
:108B000041EC1A0B9FEDFE0B53EC102B9DED080B67
:108B100051EC100B03F0DEFA41EC1B0B9FEDFA0B4E
:108B200051EC1A0B53EC102B03F0D4FA41EC1A0B56
:108B30009FEDF70B53EC102B9DED080B51EC100B38
:108B400003F0C8FA53EC1A2B03F0D0FC41EC1A0BDB
:108B500051EC1B0B53EC1A2B02F0EAFF0690CDE907
:108B600006519DED060B53EC1B2B51EC100B03F043
:108B7000BDFC53EC1A2B03F0E1FB41EC100B00F0B1
:108B8000A1B90020B6F5801F0EDA9FEDE30B53EC80
:108B9000102B9DED0E0B51EC100B03F09BFACDE961
:108BA0000E016FF034000E4600EB2650A0F2FF37A6
:108BB000C6F31300DA4940F07F6646F0405688421B
:108BC000D8BF002408DDD7498142C8BF012403DC97
:108BD0000024A6F580167F1CD348784400EBC4001F
:108BE0000F9690ED00CB9DED0E0B53EC1C2B51EC32
:108BF000100B03F07BFC9DED0E0B41EC1B0B53ECBB
:108C00001C2B51EC100B02F093FF41EC100B51ECBC
:108C1000190B53EC102B03F047F841EC1D0B51ECF2
:108C20001B0B53EC1D2B03F055FA41EC1A0BBF48FC
:108C30008DED10AB7844109590ED000B4FF0005087
:108C400040EA660000EB84408DED080B00F5002043
:108C500009909DED080B53EC1C2B51EC100B03F00D
:108C600045FC9DED0E1B53EC112B03F067FB41EC13
:108C7000100B53EC102B9DED100B51EC100B03F06F
:108C800029FA9DED080B41EC1C0B53EC102B9DEDCC
:108C9000100B51EC100B03F01DFA53EC1B2B03F0DF
:108CA0004DFB53EC1C2B03F021FC53EC1D2B03F06C
:108CB00011FA41EC1C0B53EC1A2B51EC1A0B03F07C
:108CC00009FA41EC1B0B9A480621B0EE4B0AF0EE74
:108CD0006B0A784400F01DFBB0EE401AF0EE601A0B
:108CE000B0EE41DAF0EE61DA53EC1B2B51EC1B0BCA
:108CF00003F0F0F953EC1D2B03F0ECF99DED100B94
:108D000041EC1B0B53EC1A2B51EC100B02F010FF33
:108D100053EC1C2B03F0DEF953EC1B2B02F008FF85
:108D20009DED100B41EC1B0B53EC102B51EC100B79
:108D300003F0D0F941EC1D0B9FED7FEB53EC1E2BA4
:108D400002F0F6FE53EC1B2B02F0F2FE0890CDE988
:108D500008519DED080B53EC1E2B51EC100B03F04A
:108D6000C5FB53EC1D2B03F0C1FB53EC1B2B03F095
:108D7000E5FA9DED080B41EC1D0B53EC102B9DED1E
:108D8000100B51EC100B03F0A5F941EC1B0B53EC4D
:108D90001A2B51EC1D0B03F09DF99DED080B41ECD6
:108DA0001A0B53EC102B51EC1C0B03F093F953EC02
:108DB0001A2B02F0BDFE41EC1A0B51EC1B0B53ECCD
:108DC0001A2B02F0B5FE0C90CDE90C519DED0C0B69
:108DD00053EC1B2B51EC100B03F088FB53EC1A2BBC
:108DE00003F0ACFA41EC1B0B9FED550B53EC102B31
:108DF0009DED0C0B51EC100B03F06CF941EC1A0BD0
:108E00009FED510B51EC1B0B53EC102B03F062F94F
:108E100041EC1B0B9FED4E0B53EC102B9DED0C0BFF
:108E200051EC100B03F056F953EC1B2B02F080FEB3
:108E300041EC100B4848784400EBC40090ED001B57
:108E400051EC100B53EC112B02F072FE41EC1B0B9A
:108E5000384603F0ECF8CDE9080153EC1B2B51EC3C
:108E60001A0B02F065FE41EC100B3C48784400EB15
:108E7000C40090ED00CB51EC100B53EC1C2B02F016
:108E800057FE9DED081B53EC112B02F051FE06908E
:108E9000CDE906519DED080B53EC102B9DED060B13
:108EA00051EC100B03F022FB53EC1C2B03F01EFBC8
:108EB00053EC1A2B03F01AFB53EC1B2B03F03EFA76
:108EC00041EC100B9DED261B53EC102B8DED001B80
:108ED00000959DED260B51EC100B03F0FBF89DED7A
:108EE000000B41EC1A0B53EC102B9DED260B51ECB3
:108EF000100B03F0FBFA9DED061B53EC112B2FE03A
:108F0000000000604715F73FFE822B654715F73FCD
:108F100044DF5DF80BAE543E00000000000040430B
:108F20008E9803007AB60B00E23F00001840000064
:108F30001A3F000000000000000000000000084090
:108F4000000000E009C7EE3FFD033ADC09C7EE3F31
:108F5000F5015B14E02F3EBEA63D0000603D000021
:108F600003F0B8F853EC1A2B02F0E2FD9DED060B6E
:108F700041EC1A0B53EC102B9DED000B51EC100B38
:108F800003F0A8F8CDE90C019DED0C0B51EC1A0B88
:108F900053EC102B02F0CCFDCDE902010C46AA499E
:108FA0008C422FDB611A084318D19DED0C0B53EC5A
:108FB000102B9DED020B51EC100B03F097FA41ECD6
:108FC0001B0B9FEDA30B51EC1A0B53EC102B02F073
:108FD000AFFD53EC1B2B03F07BF92DD20220F7F7EA
:108FE0000AFE00F051FA10EE901A18EE900A8DED7C
:108FF000020B8DED008B61F31E0003909DED020BC3
:10900000FFF7BEBB944A24F00041914214D3934928
:10901000214408437FF4EFAC9DED0C0B53EC102B77
:109020009DED020B51EC100B03F060FA53EC1A2B80
:1090300003F04EF97FF6DFAC24F000408849894AFE
:10904000002601EB205182422BDA481C4FF480119C
:1090500021FA00F02044844AC0F30A517A44A1F274
:10906000FF3192ED000B814A8DED080BCA4020EADA
:109070000202C0F3130040F48010C1F1140120FA81
:1090800001F60992002CB8BF76429DED080B53EC17
:10909000102B9DED0C0B51EC100B03F027FACDE9D2
:1090A0000C019DED0C0B51EC1A0B53EC102B02F044
:1090B0003FFD9FED6F0B0890CDE9085153EC102B4D
:1090C0009DED080B51EC100B03F004F841EC1B0B69
:1090D0009FED690B53EC102B9DED080B51EC100B21
:1090E00002F0F8FF9DED0C0B41EC1C0B53EC102B28
:1090F0009DED080B51EC100B03F0F8F953EC1A2B13
:1091000003F01CF99FED5E1B53EC112B02F0E2FF04
:1091100053EC1C2B02F00CFD41EC1A0B51EC1B0B19
:1091200053EC1A2B02F004FDCDE902019DED020B78
:1091300053EC1B2B51EC100B03F0D8F953EC1A2B0A
:1091400003F0FCF89DED020B41EC1A0B53EC102BD5
:1091500051EC100B02F0BEFFCDE908014A489DED2D
:10916000080B0521784400F0D4F89DED081B51EC64
:10917000100B53EC112B02F0ADFF9DED021B53ECD5
:10918000112B03F0DBF8CDE906019DED020B53EC4A
:109190001A2B51EC100B02F09DFF53EC1A2B02F02E
:1091A000C7FC9FED3B0B41EC1A0B53EC102B9DEDD4
:1091B000060B51EC100B03F099F99DED060B41ECF9
:1091C0001B0B53EC102B9DED020B51EC100B02F01E
:1091D00081FF53EC1B2B02F067FD53EC1A2B03F0BD
:1091E00085F99DED021B53EC112B03F07FF953EC35
:1091F000192B03F0A3F8CDE9020101EB065001158C
:109200000029C8BF039015DC9DED020B324651ECDE
:10921000100B03F009FBFEF7A9FE042808BF00F0BD
:1092200043F932469DED020B51EC100B03F0FCFAB2
:10923000CDE902019DED020B51EC180B53EC102B04
:1092400002F048FFFFF73ABB00009040000000002A
:10925000FE822B654715973C00CC904000346F3F51
:1092600001FCFFFF0000E03FF03B0000FFFF0F00AC
:1092700000000000432EE63F396CA80C615C20BE64
:10928000EF39FAFE422EE63FB83A00000000000037
:10929000000000000000004000B52DED048BB0EE92
:1092A000409AF0EE609A83B051EC190B03F052F83B
:1092B00041EC180B18EE100A18EE901A8DED008B89
:1092C000002818BF0120084320F00040C0F17F6053
:1092D00000F1E040C00F14D019EE101A19EE900AF8
:1092E0008DED009B002918BF0121084320F00040AC
:1092F000C0F17F6000F1E040C00F04BF0120F7F72C
:109300007AFCB0EE480A03B0F0EE680ABDEC048BBC
:1093100000BD70B504462DED028B4D1E00EBC5005F
:10932000B0EE408AF0EE608A90ED000B35F006005A
:1093300017D053EC182B51EC100B02F0CBFE41EC84
:10934000100B6D1E04EBC50090ED001B51EC100BD3
:1093500053EC112B02F0ECFB41EC100B35F0060046
:10936000E7D1022D36D0042D1CD0062D1CBFBDEC3C
:10937000028B70BD53EC182B51EC100B02F0AAFEBF
:1093800094ED0A1B53EC112B02F0D2FB53EC182B7B
:1093900002F0A0FE94ED081B53EC112B02F0C8FB69
:1093A00041EC100B53EC182B51EC100B02F092FE19
:1093B00094ED061B53EC112B02F0BAFB53EC182B67
:1093C00002F088FE94ED040B53EC102B02F0B0FB7E
:1093D00041EC100B53EC182B51EC100B02F07AFE01
:1093E00094ED021B53EC112B02F0A2FB53EC182B53
:1093F00002F070FE94ED001B53EC112B02F098FB71
:10940000BDEC028B41EC100B70BD000000000000B1
:109410009FED070B10B553EC102B9FED070B51EC94
:10942000100B02F041FC41EC100B10BD00000000DD
:109430000000000000000000000000000000F03FFD
:1094400010B553EC102B51EC100B02F071FB41ECFA
:10945000100B10BD10B553EC112B51EC100B02F09A
:1094600067FB41EC100B10BD9FED050B10B553ECE5
:10947000102B51EC100B02F017FC41EC100B10BD3F
:1094800000000000000000009FED050B10B553EC3C
:10949000102B51EC100B02F01DFE41EC100B10BD17
:1094A00000000000000000709FED050B10B553ECAC
:1094B000102B51EC100B02F00DFE41EC100B10BD07
:1094C000000000000000001010B5044691ED000BF4
:1094D000FEF766FD84ED000A10BD10B5044690ED60
:1094E000000B0846FFF748F884ED000B10BD30383C
:1094F0000A2801D201207047002070477047000001
:109500002DE9F041044641F69A30584D04424FF49B
:10951000FA774FF47A784AD0E00405D54146032023
:10952000FBF7E4FD10206872A0050CD54146012030
:10953000FBF7DCFD0B206872B2EE040AFDF75EFC5F
:109540000120BDE8F081200706D541460420FBF745
:10955000CDFD0420687225E0200604D54146042094
:10956000FBF7C4FD1EE0200506D541460320FBF7AE
:10957000BDFD0720687215E0A00706D50021062072
:10958000FBF7B4FD0A2068720CE0E00506D5002167
:109590000320FBF7ABFD0320687203E0394603208C
:1095A000FBF7A4FD3220FDF70FFC0020C9E744F2D1
:1095B000670004422E48407E4AD0610406D54146E9
:1095C0000720FBF793FD062068723CE0A10604D556
:1095D00041460620FBF78AFD35E061064FF00006A4
:1095E0000DD500210220FBF781FD6E72012085F868
:1095F0009300B2EE040AFDF701FC0120A1E7610728
:109600000CD520B164210220FBF770FD03E0414638
:109610000220FBF76BFD0220687214E0E00706D021
:1096200000210520FBF762FD052068720BE0A00415
:1096300005D541460420FBF759FD6E7203E039461B
:109640000320FBF753FD0520FDF7BEFB002078E764
:1096500020B164210120FBF749FD03E041460120D0
:10966000FBF744FD0820687201206AE76C1B0120AB
:109670006C39002010B541EC100BFEF70DFD51ECDC
:10968000100B10BD08B56846FCF7BEFA08BD000017
:1096900038B51549012008604FF44070FBF7EEFF24
:1096A00000F024F801F0CAFEFAF726FF0C20FAF7C2
:1096B00031F80C20FAF700F94AF20F444FF6FF7523
:1096C00021462846FDF750FC21462846FDF7D2FCEE
:1096D000002001224FF4E1331146009000F07AFEA1
:1096E000BDE8384000F088BCC000002010B54FF441
:1096F000E1342046FEF718F82046FEF79FF8BDE853
:109700001040FEF7F1B87E214FF4C0727F20FEF7C3
:1097100013BB000030B57849086800EE100AB8EEB7
:10972000C00ADFED760A764A60EE200A92ED081A4A
:10973000744A80EE810AF6EE000A60EE200AC2ED5D
:109740000B0A0C7F9FED701A6D4D43426F49704AB2
:1097500095ED0A0A0B2C70D2DFE804F0060B223BD1
:1097600048556270859AB10081ED001A82ED001AA9
:1097700030BD80B100EE900AF8EEE00A70EE800A8B
:10978000C1ED000A00EE900AF8EEE00A30EEC00AE1
:1097900082ED000A30BD81ED001A82ED001A30BD65
:1097A00090B100EE900AF8EEE00A70EE600AC1EDAA
:1097B000000A00EE900AF8EEE00A30EE800AB1EE00
:1097C000400A82ED000A30BD81ED001A82ED001AD8
:1097D00030BD00EE103AB8EEC00A81ED000A00EE8E
:1097E000100AB8EEC00A82ED000A30BD00EE100A81
:1097F000B8EEC00A81ED000A00EE103AB8EEC00AD9
:1098000082ED000A30BD00EE100AB8EEC00A81ED0C
:10981000000A00EE103AB8EEC00A82ED000A30BD30
:1098200000EE103AB8EEC00A81ED000A00EE100A10
:10983000B8EEC00A82ED000A30BD57E001EE100A12
:10984000B8EEC11A31EE601A31EE401A81ED001AFD
:1098500001EE100AB8EEC11A71EE200A30EE800A4D
:1098600082ED000AE8E701EE100AB8EEC11A31EE07
:10987000201A31EE001A81ED001A01EE100AB8EE3E
:10988000C11A71EE600A30EEC00A82ED000AD3E719
:1098900001EE100AB8EEC11A31EE201A31EE001AAC
:1098A000B1EE411A81ED001A01EE100AB8EEC11AAC
:1098B00071EE600A30EE600A82ED000ABCE701EE4C
:1098C000100AB8EEC11A31EE601A30EE411A81ED7D
:1098D000001A01EE100AB8EEC11A71EE200A30EE3D
:1098E000800AB1EE400A82ED000AA5E781ED001A78
:1098F00082ED001AA0E700006C1B01200000B943B4
:109900002C1C01208C02002000000000AC3900203B
:10991000C03900202DE9F0412DED048B8F48904C8B
:1099200090ED029A94ED020A39EE400A84ED040AA1
:1099300010EE100A8B49DFED8C0A884203DD30EE11
:10994000600A84ED040A94ED040A884910EE100AB6
:10995000884203D930EE200A84ED040A844F786AE5
:1099600002F0AEFE41EC180B206902F0A9FE41ECBA
:10997000100BFEF7F5FD53EC182B51EC100B02F019
:10998000B5FD41EC100BFEF7EBFD51EC100B02F0B6
:109990009DF800EE100A84ED030A97F805C0002236
:1099A0009FED741A744D754E4FF07C539FED748B80
:1099B0003946DFF8AC81B1F84200898FD8ED010A51
:1099C000BCF1070F0BD2DFE80CF0040B18B9B92675
:1099D000700085ED001A86ED001A84ED029AADE064
:1099E00000EE101AB8EE400A85ED000A00EE101ADB
:1099F000B8EE400A86ED000AA0E0484200EE100AE8
:109A0000B8EEC00A85ED000A00EE100AB8EEC00AF2
:109A100086ED000A92E010EE101A994206DB00EE85
:109A2000100AB8EE400A84ED050A14E0B4EEE00A2C
:109A3000F1EE10FA0CDD01EE100AF3EE0E1AB8EE9C
:109A4000412AB6EE001A00F0CAFF84ED050A02E0D2
:109A50007A7184ED051AD4ED050A94ED060AF4EE48
:109A6000C00AF1EE10FA0BDD10EE100A02F028FE2B
:109A700053EC182B02F05CF802F028F860610BE060
:109A80000AD210EE100A02F01BFE53EC182B02F063
:109A90002DFD02F01BF8606194ED050AF1EE400A1D
:109AA000C5ED000A86ED000A48E010EE101A994252
:109AB00006DB00EE100AB8EE400A84ED050A14E059
:109AC000B4EEE00AF1EE10FA0CDD01EE100AF3EE4E
:109AD0000E1AB8EE412AB6EE001A00F080FF84EDAF
:109AE000050A02E07A7184ED051AD4ED050A94EDB9
:109AF000060AF4EEC00AF1EE10FA0BDD10EE100AC1
:109B000002F0DEFD53EC182B02F012F801F0DEFF3C
:109B100060610BE00AD210EE100A02F0D1FD53ECA6
:109B2000182B02F0E3FC01F0D1FF606194ED050A0F
:109B300085ED000AB1EE400A86ED000A94ED050AB3
:109B400084ED060AF88FBDEC048B00EE100ABDE828
:109B5000F041B8EE400A01F0FFBA0000DC1C012021
:109B60008C020020DA0F4940DA0FC940DA0F49C0F1
:109B70006C1B012000000000AC390020C03900201F
:109B8000333333333333D33F0078012813D00228E3
:109B900011D0032811D004280FD005280DD0062895
:109BA0000BD0072805D0082803D0092801D00A289F
:109BB00005D1FBF7A5B8FBF7F5B8FAF755BF704725
:109BC0000E4A104692F8711090F87200002904D0E5
:109BD00018B1012082F88900704731B928B992F88C
:109BE0006E0010B992F86F0018B1022082F8890057
:109BF0007047002082F88900704700006C1B01202C
:109C000010B509480121817580F893104FF4027056
:109C1000FCF7C2FD40F29C610448F6F7B0FFBDE8D6
:109C200010404020FDF742B86C1B0120988F0020A7
:109C300070B50446042C02D94FF0FF3070BD40F2DD
:109C4000014000EB042510212846FDF7C5FF2846FA
:109C5000FDF780FF0028FAD140F2024000EB04201B
:109C6000FF21FDF7B9FF0D490120A0404A8882433A
:109C70004A808A8882438A8000200A3121F81400B1
:109C8000091F085540F2034000EB04242046FDF76D
:109C900061FF0028FAD1012070BD00004A000010C9
:109CA00070B506462DED028B0C462F482F4D9FEDCB
:109CB000308B072E07D2DFE806F0060409121B28B6
:109CC0003F002D480474BDEC028B70BD02218175EC
:109CD00000EE104AB8EEC00A85ED080AF3E703214A
:109CE000817500EE104AB8EEC00A85ED080AEAE771
:109CF00014B1012C09D104E001210920FAF7E4FC98
:109D000003E000210920FAF7DFFC6E7100EE104A33
:109D1000B8EEC00A10EE100A02F0D2FC53EC182B79
:109D200001F0C2FF01F0D2FE686200EE104AB8EE08
:109D3000C00A85ED080AC6E70620687100EE104AE1
:109D4000B8EEC00A10EE100A02F0BAFC53EC182B61
:109D500001F0AAFF01F0BAFE686200EE104AB8EE08
:109D6000C00A85ED080AAEE7EC3900206C1B012023
:109D70006666666666A64C40D43900202DE9F0413F
:109D800004460E461746042C03D94FF0FF30BDE8B9
:109D9000F0814FF4806000EB0420FDF7DBFE00F063
:109DA0000F00012802D06FF00400F0E740F20340FA
:109DB00000EB04252846FDF7CDFE132802D06FF0F6
:109DC0000200E4E73078717801EB0020B17801EB14
:109DD0000020F17801EB0020411C2CD058B36FB368
:109DE00040F20C4000EB042004223146FDF712FF44
:109DF0004FF48260390A00EB0420FDF7EDFE40F2DB
:109E00001140F9B200EB0420FDF7E6FE40F20140FC
:109E100000EB042604213046FDF7DEFE3046FDF758
:109E200099FE0028FAD116490120A040498808422D
:109E300007D00020ABE76FF00B00A8E76FF00A0037
:109E4000A5E740F2024000EB04240FE02046FDF7B6
:109E500081FE000706D520460821FDF7BDFE6FF004
:109E60000C0094E72846FDF775FE30B12846FDF753
:109E700071FE1728EAD1012089E76FF0030086E719
:109E80004A00001010210148FAF71CBC00000240F3
:109E900010210148FAF714BC0000024010B540F24E
:109EA0000350FDF757FE50B1132811D0172817D0D3
:109EB0001C2842D1BDE810400120FFF7B9BE1F4861
:109EC000202301210288BDE81040084601F050B966
:109ED0001B481C490288BDE810400120FFF74EBF17
:109EE00040F202542046FDF735FEC00703D00121A1
:109EF0002046FDF771FE012000F00CFC0446002C0A
:109F00001BD022461049012000F07EFE0E490020A1
:109F100008550A460DA10120FDF7A2FD104811A128
:109F20000A6802604A684260098901810A22014682
:109F3000BDE81040012001F075B810BD5E000010B2
:109F40006400001060000010D8080020C0B4D7D40E
:109F5000B7FECEF1C6F7CAFDBEDD25730D0A0000BF
:109F6000D810002061626364656667650D0A0000B1
:109F700010B540F20340FDF7EDFD50B1132815D0A8
:109F800017281CD01C282AD1BDE810400020FFF75C
:109F90004FBE13A10120FDF763FD134820230121CB
:109FA0000288BDE81040002001F0E2B80FA10120B6
:109FB000FDF756FDBDE81040002000F0BFBC40F2A8
:109FC00002442046FDF7C6FDC00703D0012120460C
:109FD000FDF702FEBDE81040002000F09BBB10BD65
:109FE00043726561740D0A005C0000104C495354C3
:109FF000454E0D0A0000000070B50024054D28787C
:10A00000012802D00624204670BD28698047002020
:10A010002870F8E7140000202DE9F0410C460026D6
:10A020002188052903D003263046BDE8F081417818
:10A030000A0281781143491C8FB2C1780902027962
:10A040000A43511E40F2CF73994221D20021218050
:10A05000012100F8011B23885B1C2380530703D0D8
:10A0600001EBD201CDB201E0C2F3C70500F8015BFC
:10A070002188491C21800023394600F09CFA18B140
:10A0800000F0A2FD0646CFE7208828442080CBE7D9
:10A090000326C9E770B50C4600262188052902D0A1
:10A0A0000326304670BD4178090282780A43521C6B
:10A0B00093B2C178090202790A43511E40F2CF756A
:10A0C000A94221D200212180022100F8011B218810
:10A0D000491C2180510704D0012101EBD201CDB2EE
:10A0E00001E0C2F3C70500F8015B2188491C21800B
:10A0F000194600F062FA18B100F066FD0646D0E796
:10A10000208828442080CCE70326CAE770B50C4697
:10A1100000262188052902D00326304670BD4178EB
:10A120000A0281781143491C89B205796A1E7C2A8A
:10A130001AD800222280032202702288521C228018
:10A140006A004270801C2288521C228000232A460A
:10A1500000F036FA18B100F037FD0646DDE720883A
:10A1600000EB45002080D8E70326D6E770B50C4603
:10A1700000262188052902D00326304670BD41788B
:10A180000A0281781143491C89B2C278120205790A
:10A1900015436A1E7C2A19D20022228004220270F2
:10A1A0002288521C22806A004270801C2288521C25
:10A1B00022802A4600F038FA18B100F005FD064664
:10A1C000DBE7208800EB45002080D6E70326D4E7B4
:10A1D0002DE9F04104460D46002728880A2842D37D
:10A1E00060780102A0780843401C1FFA80F8E078EC
:10A1F00000022679064360790102A0790843401CD9
:10A2000081B2E0790002227A0243607A731E7C2BCD
:10A2100028D83AB3792A25D8B0EB420F22D10123AE
:10A2200004F10A0000F0CCF9B8B9204600212980D9
:10A23000172101702988491C298071004170801CF8
:10A240002988491C298000233246414600F0B8F98C
:10A2500018B9298801EB4601298020B100F0B4FC2F
:10A26000074600E003273846BDE8F08170B50C468C
:10A27000054D0649401C2A88F6F70AFC2888401C30
:10A280002080002070BD0000480000107090001079
:10A2900038B500240988052902D00324204638BD9A
:10A2A0004178090282780A43521C91B202791AB9A4
:10A2B000C278FF2A02D00AB10324EFE700228DF80A
:10A2C0000120C078FF280CD08DF8002001231A4609
:10A2D000684600F070F90028E0D000F075FC0446F4
:10A2E000DCE701208DF80000F0E710B500240988B4
:10A2F000052902D00324204610BD41780A02817846
:10A300001143491C89B201231A46C01C00F058F9B8
:10A310000028F0D000F058FC0446ECE72DE9F041AD
:10A320000D4600242988052927D941780902827819
:10A330000A43521C91B2C278130202791A43467939
:10A34000530704D0012303EBD203DBB201E0C2F3D5
:10A35000C703571EB7F5F66F0DD2B3420BD10123D9
:10A36000801D00F028F918B100F02EFC044605E02D
:10A370000520288002E0032400E003242046BDE8F5
:10A38000F08170B50D460024298806291FD3417835
:10A39000090282780A43521C91B2C27813020279F0
:10A3A0001A434379561E772E0FD85606360E9E4214
:10A3B0000BD10123801D00F003F918B100F004FC5B
:10A3C000044605E00520288002E0032400E0032481
:10A3D000204670BD70B514461A46049B06460029F7
:10A3E00001D0F72901D9022421E0134D0846297133
:10A3F00016B10224ACB11AE0104929611049696113
:10A400001049E9601049A9610021E9610F492962F9
:10A410000F4969620F49A962214600F01DF8044600
:10A42000E8E701F053F920B16E7101202870204651
:10A4300070BD0324FBE700001400002089A502087A
:10A44000A5A5020835A5020899A4020889B8020842
:10A45000BDB9020845B9020870B508461546002482
:10A460000822294601F04CF9012801D003240EE00E
:10A47000B5F5964F01D9232003E006496800B1FBEA
:10A48000F0F080B201F0C6F9012800D00324204684
:10A4900070BD0000A07F17002DE9F04180460E46F8
:10A4A000174600240F4DA888FF280BD8A888042839
:10A4B00004D3A9880C4800F0ABFF40B10524204626
:10A4C000BDE8F081A12209A110A0F6F737FA0648ED
:10A4D000007888F80000A888C01E38800248401C18
:10A4E0003060ECE708000020D80700202E2E5C2EFC
:10A4F0002E5C4D4F444255535C6D6F646275735CC6
:10A500007274755C6D627274752E6300757352633C
:10A5100076427566666572506F73203C204D425FCF
:10A520005345525F5044555F53495A455F4D41581A
:10A530000000000070B5034608460025104C667800
:10A54000012E02D00525284670BD401EA0600126C0
:10A5500066800370618811446180618800F058FF53
:10A5600061884A1C6280074A5054030A6088411C73
:10A570006180135426700121002000F073FFE2E790
:10A5800008000020D807002010B5054900204870B9
:10A590000021012000F066FFBDE8104000F0A0BFE0
:10A5A0000800002010B50021084600F05BFFBDE860
:10A5B000104000F085BF0020704701207047000068
:10A5C0002DE9F0410546144600270819B0F57A6FC9
:10A5D00022D8134840880E1ADFF8488063B1012B57
:10A5E0001BD116E03046761C38F81000F5F7A0FEB7
:10A5F00025F8020B641EA4B2002CF3D10DE035F84F
:10A60000020BF5F795FE3146761C28F81100641E02
:10A61000A4B2002CF3D100E001273846BDE8F08158
:10A6200044000010307100102DE9F0410546144639
:10A6300000270819322812D80B4800880E1ADFF8B4
:10A640002C8009E03046761C38F81000F5F770FED3
:10A6500025F8020B641EA4B2002CF3D100E0012700
:10A660003846BDE8F0810000440000103071001051
:10A6700082B0CDE9000121F0004001909DED000B7A
:10A6800002B051EC100B704710B582B01446CDE902
:10A6900000010023009A2360194B21F000409842EA
:10A6A0002ADA024328D0B0F5801FA8BF226810DA4A
:10A6B0009FED150B53EC102B9DED000B51EC100B87
:10A6C00001F008FDCDE900016FF0350221F00040F6
:10A6D00022600F4B6FF31E5103EB2050104420609B
:10A6E00041F0FF5040F0005001909DED000B00BF85
:10A6F00002B051EC100B10BD9DED000BF8E700000F
:10A700000000F07F00000000000000000000504347
:10A7100002FCFFFF2DE9F041002740F2264101EB4A
:10A720000025491C01EB00262846FDF713FA0446D4
:10A730003046FDF70FFA00EB042084B24CB12846F6
:10A74000FDF708FA07463046FDF704FA00EB07204C
:10A7500087B2A742E8D13846BDE8F0812DE9F04143
:10A7600007464FF4C045002403264FF001080EE0D1
:10A770001A20FDF7EFF9610006FA01F21040C84017
:10A7800008FA00F080B205EB8025641C64B2BC427C
:10A79000EEDB2846BDE8F0812DE9F04100274FF4BB
:10A7A000846101EB0025491C01EB00262846FDF7DA
:10A7B000D1F904463046FDF7CDF900EB042084B210
:10A7C0004CB12846FDF7C6F907463046FDF7C2F9F9
:10A7D00000EB072087B2A742E8D13846BDE8F081F8
:10A7E0002DE9F04107464FF48045002403264FF041
:10A7F00001080EE01B20FDF7ADF9610006FA01F239
:10A800001040C84008FA00F080B205EB8025641CB7
:10A8100064B2BC42EEDB2846BDE8F081084991F8FD
:10A820007F20002A03D0322801DD3220704791F8C2
:10A830007E100029FAD06428F8DD642070470000FB
:10A840006C1B012070B5344C9FED340ADFED340AE7
:10A85000207C03280DD2DFE800F002050A00C4EDD9
:10A86000010A06E09FED2F1A84ED011A01E084ED44
:10A87000010A2D49487840B194ED011AB5EEC01A8D
:10A88000F1EE10FA01DDC4ED010A284A10B192F888
:10A89000840008B9087808B184ED010A92F86B00C9
:10A8A0001D4A002592ED030A30B194ED011AB5EE70
:10A8B000C01AF1EE10FA0BD310EE102A1C4B9A427C
:10A8C0000BDD94ED011AB5EEC01AF1EE10FA04DDBD
:10A8D0000D704D70C4ED010A257418B14FF0FF30B2
:10A8E000606170BDF3EE0E0A30EE600A10EE100AE1
:10A8F00001F0E6FE41EC100BFDF732FE9FED0D1B63
:10A9000051EC100B53EC112B01F0A8FB01D2656147
:10A9100070BD0120606170BDD43900200024F4C8EE
:10A92000000000000024F448BC0200206C1B012041
:10A9300000002C42000000000000F03F70B504460B
:10A94000042C02D94FF0FF3070BD4FF4806000EB53
:10A950000420FDF7FFF800F00F00012802D06FF08F
:10A96000040070BD40F2034000EB04200646FDF7F2
:10A97000F1F8132802D06FF0020070BD40F20140E0
:10A9800000EB042502212846FDF726F92846FDF7AD
:10A99000E1F80028FAD13046FDF7DCF8142805D09C
:10A9A0002046FFF745F96FF0030070BD012070BD30
:10A9B00008B54FF400318802FAF76AFEF9F731FA68
:10A9C000FEF766FEF8F720FE6846FAF781FE684655
:10A9D000F8F7FAFC6846FAF77DFF002008BDB4EEF0
:10A9E000E00AF1EE10FA01D2B0EE600AB4EEC10A4C
:10A9F000F1EE10FA01DDB0EE410A32EE612A30EEDE
:10AA0000600A31EE601A20EE020AC0EE010A30EE52
:10AA1000A10A704710B5FFF715FFBDE81040FBF71E
:10AA2000C3BE10B5FFF70EFFBDE81040FBF7BCBE7C
:10AA300070B5FDF721FA5D4C0025207908B3A07AA6
:10AA4000F8B1207F08B9607910B394F8660018B1A6
:10AA50000120FCF72BF902E00120FBF79DFE94F8A2
:10AA60006510012011B184F87F0001E084F87F5067
:10AA700094F8641011B184F87E0009E084F87E50E7
:10AA800006E00120FBF788FE84F87E5084F87F50B2
:10AA900094F8630018B10620FCF708F902E00220E0
:10AAA000FBF77AFE94F8600020B14FF48270FCF757
:10AAB000FDF803E04FF48070FBF76EFE94F8610040
:10AAC00010B10420FBF768FE94F8620010B1042076
:10AAD000FCF7ECF894F86B10354D19B100212846BD
:10AAE000FCF731FB217911B1D4F88010C9B30021F2
:10AAF0000720F9F7E9FD01210820F9F7E5FD2846CF
:10AB0000FCF709FB5434E0864FF08040FCF703FB70
:10AB100020872848FCF7FFFA60872748FCF7FBFAF4
:10AB2000A087B4F93600C11700EB91708010206443
:10AB3000FFF746F814F8500C543C002835D0207F1D
:10AB4000012817D0022815D0072813D0082811D0C3
:10AB500009280FD00A280DD0BDE870400820FBF767
:10AB60001BBE01210720F9F7AFFD00210820F9F7EE
:10AB7000ABFDC4E71148406801F0A2FD41EC100BA9
:10AB8000FDF7EEFC9FED0E1B51EC100B53EC112B5F
:10AB900001F09EFB04D2BDE870400820FCF786B8A7
:10ABA000BDE870400820FBF7F7BD70BD6C1B0120AD
:10ABB0000000014000040040000800402C1C01205F
:10ABC0000000000000005940002805D0012805D0F1
:10ABD000072805D0042070470020704702207047E6
:10ABE0000620704701480068004700003C00002034
:10ABF0000148006800470000340000200148006858
:10AC000000470000380000202DE9F74F05461646A2
:10AC1000042D03D94FF0FF30BDE8FE8F4FF4806064
:10AC200000EB0520FCF796FF00F00F00012802D092
:10AC30006FF00400F0E7D6B11A20FCF78BFF6F002D
:10AC40004FF0030909FA07F900EA0900F8404FF04C
:10AC5000010808FA00F04FF6FF7101EA8020B042C7
:10AC600000D2064640F2034000EB052A42E06FF0B6
:10AC70000D00D1E71C2805D02846FEF7D9FF6FF05C
:10AC80000600C9E7ECB92846FFF786FD83461B207E
:10AC9000FCF760FF00EA0900F84008FA00F080B213
:10ACA000BBEB802F05D12846FEF7C2FF6FF00600F0
:10ACB000B2E7154908FA05F04988084200D0BCB14E
:10ACC000C4B1B44200D2264632462846019900F06B
:10ACD0001BFC40F2014000EB052440212046FCF71C
:10ACE0007BFF2046FCF736FF0028FAD1304693E779
:10ACF000002091E72846FFF70DFD04465046FCF77B
:10AD000029FF1728D5D0B5E74A000010054A0028CA
:10AD100003D011B1506191617047034850610348FD
:10AD20009061704770000010C3B60208C1B60208F7
:10AD300010B5074C22889305FDD518B111B1E0611B
:10AD4000216210BD0348E0610348206210BD00008D
:10AD500070000010C5B60208C9B602082DE9F04F10
:10AD60002DED028BAFB0904B904AD3F880102D910F
:10AD7000890502D50121916001E000219160D3F89D
:10AD8000BC1054680C1B84427ED3516093F81C8025
:10AD9000B8F1010F1BD0B8F1030F18D0B8F1040FB0
:10ADA00015D0B8F1070F12D0B8F1080F0FD0B8F1D5
:10ADB000020F0FD0B8F1050F0CD0B8F1060F09D073
:10ADC000B8F1090F06D0B8F10A0F03D004E06620ED
:10ADD000107001E06220107074487649774C027858
:10ADE000754809682C9190ED000A754D6E48BDEECE
:10ADF000C08A94ED000A817DD5F804B02B91744986
:10AE0000DFF8C0C1DFF8C091497E2A91DCF8181044
:10AE10002991D9F814102891A16827916978269171
:10AE200001796A4E259100682490614F3068239023
:10AE300070682290A7F10C03FDEEC08AD3E900A947
:10AE40003E68662A58D0304601F03AFC04460D466A
:10AE5000304601F035FC06460F46484601F030FC0E
:10AE6000CDE92001504601F02BFC81468A462C9802
:10AE700001F026FC02462B98CDE9190BCDED1B8A7B
:10AE80000B468DED1C8A00E031E0CDE91758169491
:10AE9000DDE92001CDE91467CDE91201CDE9109A71
:10AEA0004248DDE9281485682A98CDE90D05CDE9E9
:10AEB0000B14DDE925452799CDE907450120CDE9AA
:10AEC000091044A5249C2D99CDE90450CDE9002317
:10AED000CDE902040691DDE922213F48FBF72AFB78
:10AEE00000220090142311461046F9F767FA2FB09C
:10AEF000BDEC028BBDE8F08F304601F0E1FB04466B
:10AF00000D46304601F0DCFBCDE92001484601F05A
:10AF1000D7FB06460F46504601F0D2FB81468A46D3
:10AF20002C9801F0CDFB2A4A92ED040AD269CDEDAE
:10AF30001B8ABDEEC00A8DED1C8A1D928DED1E0A86
:10AF40002B9ACDE9192BCDE917581694DDE920236A
:10AF5000CDE9109ACDE91423CDE91267134ADDE952
:10AF600029439568289ACDE90D35CDE90B24DDE913
:10AF70002654CDE908540122259B07930A9217A570
:10AF80002D9BCDE90452249C8DE81700DDE9222198
:10AF900006931348FBF7CEFA0022009014231146C3
:10AFA0001046F9F70BFAA2E76C1B0120C807002036
:10AFB000D01C012088020020C0390020AC390020BC
:10AFC000988F0020EC390020D43900206C39002003
:10AFD0008C39002062000000E8CD02086600000005
:10AFE00078CD02081CB501210846FBF70DFB0820AF
:10AFF000009001208DF804008DF8070002208DF8E4
:10B000000500074C69462046F9F7F0FA0421009143
:10B0100000218DF8041069462046F9F7E7FA1CBDB7
:10B02000000002402DE9F74F05461446042D03D9D0
:10B030004FF0FF30BDE8FE8F4FF4806000EB05203D
:10B04000FCF788FD00F00F00012802D06FF004002B
:10B05000F0E774B140F2034000EB052A5046FCF7DC
:10B0600079FD6FF00609172806D01C2804D0484641
:10B07000E0E76FF00D00DDE7DFF8D8804FF0010B5F
:10B080000BFA05F6B8F80400064211D040F202406F
:10B0900000EB05273846FCF75DFDC1061BD5384699
:10B0A0001021FCF799FDB8F80400B043A8F804009B
:10B0B0001B20FCF74FFD014668000322824011402F
:10B0C000C1400BFA01FB4FF6FF7000EA8B2084426F
:10B0D00035D9044633E0000705D52846FEF7A8FD1C
:10B0E0006FF00C00A6E70020A4E71C2804D0284637
:10B0F000FEF79EFD48469DE7B8F80200064203D0E1
:10B10000BC4201D9002095E7BC4218D82246284607
:10B11000019900F064FA40F2014000EB052520217E
:10B120002846FCF759FD2846FCF714FD0028FAD103
:10B13000B8F804000643A8F8046020467AE72846D9
:10B14000FFF72AFB07465046FCF704FD1728D3D02B
:10B15000CBE700004A000010034880ED040A0348D2
:10B1600080ED040A70470000AC390020C03900208F
:10B17000F8B504460F4616461D46042C02D94FF07A
:10B18000FF30F8BD062F18D2DFE807F017030A0AD0
:10B190000A0A042269460F20FCF7F8FC009848B11F
:10B1A00069076FF00500ECD495B1012F08D0022F8C
:10B1B0000ED109E06FF00200F8BD6FF00400F8BD99
:10B1C00015F0210FFBD003E0A90601D52906F6D51D
:10B1D0002046FEF72DFD05F0F0014FF48060394365
:10B1E00000EB0420FCF7F8FC224F56B93E88701C97
:10B1F00080B23880A0F57F41F03902D14FF4404051
:10B20000388040F20440310A00EB0420FCF7E4FCF3
:10B2100040F20540F1B200EB0420FCF7DDFC40F207
:10B22000014000EB042601213046FCF7D5FC3046F6
:10B23000FCF790FC0028FAD101207988A0408143D6
:10B2400005F00102A2400A437A80B9888143B9809F
:10B25000084900200A3121F81400091F085540F25E
:10B26000034000EB04252846FCF774FC0028FAD0C4
:10B2700060B2F8BD4A0000107CB501210846FBF71A
:10B28000C3F9154D052211462846F9F7EDF90522B7
:10B2900006212846F9F7E8F9052207212846F9F79B
:10B2A000E3F902218DF8041000248DF80640E02116
:10B2B000009169462846F9F799F901218DF80410A3
:10B2C0008DF806408DF8074010200090694628460A
:10B2D000F9F78CF97CBD00000000024010B50B4C62
:10B2E00002212046FBF772FC0028F9D000212046FD
:10B2F000FBF775FC01212046FBF768FC0028F9D01C
:10B300002046FBF76AFCC0B210BD000000300140CF
:10B3100070B505460A4C02212046FBF757FC002871
:10B32000F9D029462046FBF75AFC01212046FBF7BD
:10B330004DFC0028F9D02046BDE87040FBF74DBC1D
:10B340000030014010B586B001210803FBF778F901
:10B350000020ADF80400ADF808000221ADF80A1095
:10B360000121ADF80C104902ADF80E100821ADF81E
:10B370001010ADF812000720ADF814004FF48270E1
:10B38000ADF80600054C01A92046FBF72AFC012177
:10B390002046FBF70FFC06B010BD00000030014056
:10B3A00000B52DED048B83B041EC190B00F0D2FFFA
:10B3B00041EC180B18EE100A18EE901A8DED008B68
:10B3C000002818BF0120084320F00040C0F17F6032
:10B3D00000F1E040C00F14D019EE101A19EE900AD7
:10B3E0008DED009B002918BF0121084320F000408B
:10B3F000C0F17F6000F1E040C00F04BF0120F5F70D
:10B40000FAFB51EC180B03B0BDEC048B00BD00003F
:10B4100070B5FF23FF22084D05F5807605E010F892
:10B42000014B54402A5D5A40335D491E89B2F6D221
:10B4300042EA032070BD0000EEC8020810B50121E9
:10B440000807FBF7EFF80120FBF76EF801218804ED
:10B45000FBF7DAF80248416841F40071416010BD21
:10B460000070004070B50C46134D144E40F225514B
:10B47000012811D000223046FCF7D5F810212846CB
:10B48000F9F720F940F22771012C0ED03046BDE8C3
:10B4900070400022FCF7C7B801223046FCF7C3F821
:10B4A00010212846F9F70CF9ECE73046BDE870406A
:10B4B0000122FCF7B8B80000000C02400044004034
:10B4C00010B5064C00212046FBF73DFE2046002229
:10B4D000BDE810400121FBF72CBE0000000C00402D
:10B4E00010B5084C01212046FBF706FE002120463E
:10B4F000FBF729FE20460122BDE810401146FBF76C
:10B5000018BE0000000C00402DE9F74F82B007463E
:10B51000904640F2294000EB072A5046FCF71AFB00
:10B5200004464FF4856000EB072B5846FCF712FBEE
:10B5300004EB00201FFA80F91A20FCF70BFB7D00BA
:10B540000326AE403040E840012181404FF0FF30FB
:10B5500000EB812404EA09043846FFF7FFF8204491
:10B5600080B201901A20FCF7F5FA3040E840012142
:10B57000814088B204EB0801B1EB802F1CD91A205E
:10B58000FCF7E8FA3040E84001218140C4EB81201B
:10B5900084B2224603990198FCF7F8FA039805193A
:10B5A000A8EB040084B23846FFF7D8F880B22246F0
:10B5B0002946FCF7EBFA04E0424603990198FCF7B0
:10B5C000E5FA09EB080084B2210A5846FCF704FBAF
:10B5D00005B0E1B25046BDE8F04FFCF7FDBA2DE9E9
:10B5E000F74F82B00746904640F2254000EB072A0D
:10B5F0005046FCF7AFFA044640F2244000EB072B1C
:10B600005846FCF7A7FA04EB00201FFA80F91B202C
:10B61000FCF7A0FA7D000326AE403040E84001214F
:10B6200081404FF0FF3000EB812404EA09043846E2
:10B63000FFF7D6F8204480B201901B20FCF78AFA6D
:10B640003040E8400121814088B204EB0801B1EBB1
:10B65000802F1CD91B20FCF77DFA3040E8400121E7
:10B660008140C4EB812084B2224603990198FCF703
:10B67000D1FA03980519A8EB040084B23846FFF705
:10B68000AFF880B222462946FCF7C4FA04E04246ED
:10B6900003990198FCF7BEFA09EB080084B2210A6D
:10B6A0005846FCF799FA05B0E1B25046BDE8F04FB4
:10B6B000FCF792BA00787047017070477047704786
:10B6C0007047704700207047704700000249002013
:10B6D000486001207047000000000020024901225C
:10B6E0004A600870012070470000002010B5044631
:10B6F0000248FCF711F82070012010BD0044004002
:10B70000F0B587B001210820FAF77EFF314F1021F4
:10B710003846F8F7D5FF1020059001258DF8185010
:10B7200000248DF81A4003208DF8190002268DF8A8
:10B730001B6005A93846F8F759FF01214804FAF7BC
:10B7400071FF072205213846F8F78EFF07220621F0
:10B750003846F8F789FF602005908DF818608DF85D
:10B7600019608DF81A408DF81B5005A93846F8F776
:10B770003DFF4FF4E1300190ADF80840ADF80A40CC
:10B78000ADF80C40ADF810400C20ADF80E00124E94
:10B7900001A93046FBF762FF26218DF800100A212F
:10B7A0008DF801108DF802408DF803506846F9F7C6
:10B7B00031FF012240F225513046FBF734FF0121D1
:10B7C0003046FBF7FDFE40213046FBF7EDFE07B0AB
:10B7D0000120F0BD000C02400044004070B504465A
:10B7E0000A4D10212846F8F76DFF2146084C2046E7
:10B7F000FBF796FF40212046FBF7EEFE0028F9D02C
:10B8000010212846F8F75CFF012070BD000C0240B3
:10B81000004400407FB501210820FAF703FF1420FF
:10B82000029040F63300ADF804000024ADF80C405F
:10B83000ADF80640134D01A92846FBF787FC01210E
:10B840002846FBF74DFC32218DF800100B218DF8B6
:10B8500001108DF8024001218DF803106846F9F7B8
:10B86000D9FE01212846FBF747FC0022012128468A
:10B87000FBF75FFC01212846FBF741FC04B00120E7
:10B8800070BD0000000C004038B500251C4C20782D
:10B89000002804D0EC221BA122A0F5F74FF868463F
:10B8A000FFF724FF617839B1254801290AD0022920
:10B8B00015D0032921D102E0FFF712FE1DE0FFF7AA
:10B8C0000FFE1AE00021A1809DF80030A1884A1CDB
:10B8D000A280435402206070FFF702FE0DE0A188B1
:10B8E000FF2906D89DF80030A1884A1CA280435445
:10B8F00001E003206070FFF7F3FD284638BD00002B
:10B90000080000202E2E5C2E2E5C4D4F44425553D5
:10B910005C6D6F646275735C7274755C6D62727479
:10B92000752E630065536E645374617465203D3DEC
:10B930002053544154455F54585F49444C450000DE
:10B94000D807002070B50024124D6878002811D067
:10B95000022814D0032816D06878A0B1687802288D
:10B9600011D0687803280ED040F261120AA1124863
:10B97000F4F7E4FF0020FFF7B1FE044603E00120E6
:10B98000FFF7ACFE0446FFF79BFD012068702046E0
:10B9900070BD0000080000202E2E5C2E2E5C4D4F46
:10B9A000444255535C6D6F646275735C7274755C70
:10B9B0006D627274752E630014CD020870B5002597
:10B9C000164C6078012805D040F2271214A11CA063
:10B9D000F4F7B4FF207810B101281CD104E0002155
:10B9E0000120FFF73FFD16E0608850B1A0680078A5
:10B9F000FFF7F4FEA068401CA0606088401E6080D5
:10BA000009E00320FFF76AFE054600210120FFF749
:10BA100029FD00202070284670BD0000080000208D
:10BA20002E2E5C2E2E5C4D4F444255535C6D6F6440
:10BA30006275735C7274755C6D627274752E6300EE
:10BA4000655263765374617465203D3D20535441C3
:10BA500054455F52585F49444C45000010B50029D9
:10BA60000AD00878002807D005487844F6F706FF82
:10BA7000002801D0002010BD0248784410BD00000D
:10BA80003A1400003214000010B500290AD00878DA
:10BA9000002807D005487844F6F7F0FE002801D0CA
:10BAA000002010BD0248784410BD00001E150000A3
:10BAB0001615000081F00041704780F0004070478B
:10BAC00021F00041704720F00040704721F0004213
:10BAD000A2F16052B2F5801F01F0004328BFD2F1FD
:10BAE0007F6C0BD95FEA001C43EAC20242EB507044
:10BAF00018BF704728BF20F001007047B2F5801FC3
:10BB0000BCBF184670474FEA410C1CF5001F02D21B
:10BB1000084600F04BBE70B500F086FB00000089BF
:10BB2000FFF7F6BF4FF00040A0F58000704700001F
:10BB300010B591EA030F48BF83F0004300F1DE84A3
:10BB4000841A71EB030C05D2121943EB0C03001B92
:10BB500061EB0C01DFF824E14FEA1154A4EB135C14
:10BB60001EEA430F18BF9EEA445F73D023EA0E0318
:10BB7000DCF1200E21EA045143F4801332D322FA7F
:10BB80000CFE10EB0E0023FA0CFE41EB0E01CCF183
:10BB9000200E03FA0EFE10EB0E0051F10001B1F57C
:10BBA000801FCCF1200E32D201EB045112FA0EF2BA
:10BBB000BDE8104058BF7047401C38BF5FEA4202E2
:10BBC00018BF7047002814BF20F0010041F10001A8
:10BBD0004FEA410313F5001F38BF7047A1F1C04180
:10BBE00000F070BB012A43EB0302ACF1200CDCF146
:10BBF0001F0E32BF4FF0000E23FA0CF310EB0300C0
:10BC000041EB0451B4EB115FD0D0A1EB045101F52D
:10BC1000801149085FEA300001EB04510ED350F166
:10BC2000000038BF12FA0EFE08D1BDE81040C9E787
:10BC3000401C38BF5FEA4202CAD1C3E7BDE81040EA
:10BC40004FEA410313F5001F38BF7047A1F1C0410F
:10BC500000F038BB9EEA445F08D011EA5E0FBDE8F1
:10BC6000104004BF01F0004100207047BDE81040C3
:10BC700070B500F0D9FA00BF64FBBE3E0000E0FFE3
:10BC800002494FF0000000F09DBD00BF0000F87FAA
:10BC9000491058BFC1F140415B1058BFC3F1404348
:10BCA0008B42EFF3008070472DE9C04130B4DFF8DC
:10BCB000A0C23CEA111418BF3CEA131400F0EC8057
:10BCC00081EA03051CEA111444EAD57418BF1CEA82
:10BCD000131500F0C780A4EB05044FF0004545EABA
:10BCE000C12145EAC32341EA505143EA525304F1CA
:10BCF0007F74994204F500344FEAC0204FEAC22213
:10BD000008BF904200F09C804FEA13650FF2401686
:10BD1000765D4FEA134506FB05F7C7F1807706FB12
:10BD200007F74FEAD737A7FB03687642C8F5803894
:10BD3000A7FB06CE38BFA8F1010807FB08E64FF0C5
:10BD4000000EA6FB028CE6FB03CEDCF1000CCEF16C
:10BD5000004E38BFAEF1010EA6FB0C584FF00007A5
:10BD60004FF00005E6FB0E87A1FB08C6A0FB07CE3F
:10BD700016EB0E0645F10005E1FB076515F1E04EF7
:10BD80007EBFA4F580345FEA46066D4116F1800758
:10BD900045F100054FEA17274FEA066647EA0567AF
:10BDA000A6F1DE46B6F1805F4FEA15251FD9384669
:10BDB00024F0010C05EBC471BCF1FE6F01EB0C111A
:10BDC00002D8F0BCBDE8008124425CBF01F5801EB2
:10BDD0009EEAC47F02D4F0BCBDE80081244238D47E
:10BDE000F0BCA1F1C041BDE8004100F06BBA4FEAE0
:10BDF000D22242EA43524FEAD323A7FB02864FEAFC
:10BE0000D02040EA415007FB03661EEA0E0F4FEABE
:10BE1000D12105FB026658BFA6EB0056B6EB0056D3
:10BE20004FEA520E4EEAC37E18EB0E0E56EB530E3F
:10BE3000BDD518EB02085E417F1C55F10005B6E741
:10BE40004FF480154FF000074FF000064FF0000848
:10BE5000ADE7F0BC4FF0000001F1C04101F000413E
:10BE6000BDE8008111EA0C1F0CEA131500D00CE0AC
:10BE700013EA0C1F00F025804FF00000F0BC81EAAF
:10BE8000030101F00041BDE80081F0BCBDE80041C4
:10BE900081EA030100F016BAF0BCBDE8004170B5BC
:10BEA00000F0C2F9097EFC3E00F007B881EA030108
:10BEB0004FF0000001F00041704781EA030100F0FB
:10BEC00001BAF0BCBDE800414FF0000021497047C5
:10BED000FFFDFBF9F7F5F4F2F0EEEDEBE9E8E6E44F
:10BEE000E3E1E0DEDDDBDAD8D7D5D4D3D1D0CFCDD6
:10BEF000CCCBCAC8C7C6C5C4C2C1C0BFBEBDBCBB0F
:10BF0000BAB9B8B7B6B5B4B3B2B1B0AFAEADACAB09
:10BF1000AAA9A8A8A7A6A5A4A3A3A2A1A09F9F9EE3
:10BF20009D9C9C9B9A999998979796959594939395
:10BF3000929191908F8F8E8E8D8C8C8B8B8A89892C
:10BF400088888787868585848483838282818180AF
:10BF50000000FF070000F87F51EA030C17D41CF51E
:10BF6000801F58BFBCF5801F00F10680994218BFA2
:10BF7000704708BF9042704707D711F5801F58BF20
:10BF800013F5801F19D499427047894270471CF5F8
:10BF9000801F08D5BCF5801FF7D58B4218BF7047AE
:10BFA00008BF824270474FF4001C1CEB410F38BFA2
:10BFB0001CEB430F01D28B42704770B500F034F98F
:10BFC000922449004FF000514FF08053FFF760BEBC
:10BFD0004FEA41034FEA5353A3F58063D3F11E03A5
:10BFE000C8BFD3F1210C0CDD4FF0004242EAC12260
:10BFF00042EA505232FA03FC8CEAE17CACEBE1708D
:10C000007047102BC4BF0020704703F5787CBCF14B
:10C01000FF3F04D06FF0004282EA2100704770B504
:10C0200000F002F94992248000207047F2E710F0F6
:10C03000004248BF4042B0FA80F310FA03F10AD040
:10C04000C3F11D0303F580634FEA415002EB035235
:10C0500002EBD12170474FF00000704751EA030C0A
:10C0600017D41CF5801F58BFBCF5801F00F1068057
:10C07000994218BF704708BF9042704707D711F523
:10C08000801F58BF13F5801F19D499427047894209
:10C0900070471CF5801F08D5BCF5801FF7D58B4273
:10C0A00018BF704708BF824270474FF4001C1CEB5A
:10C0B000410F38BF1CEB430F01D28B42704770B564
:10C0C00000F0B2F8922449004FF000514FF0805335
:10C0D000FFF7DEBDDFF848C170B51CEA111E1EBFB8
:10C0E0001CEA13159EEA0C0F95EA0C0F00F06F8006
:10C0F00081EA030423EA4C134EEAD47E21EA4C1170
:10C1000041F4801143F48013AE44A1FB024CA0FB28
:10C110000365AEF17F7E361955EB0C05A1FB034C90
:10C120004CF10003A0FB021C16EB0C06654153F119
:10C130000003094218BF46F0010613F4007F0BD13B
:10C140004FEA03314FEA0530340341EA155140EA22
:10C1500016506FF003020AE04FEAC3214FEAC520F0
:10C16000F40241EA555140EA56506FF0020202EBE8
:10C170002E4201EB025585EACE710AD05FEA440CEB
:10C1800018BF24F0004450F1000041F1000120EA02
:10C19000D47040F2FE7C624500D270BDA84214BF4C
:10C1A0004FF080444FF04044002E08BF0024BEF101
:10C1B000806FA8BFA1F1C041BDE8704080F28280CD
:10C1C0004FF0000001F1C04101F0004170479EEACC
:10C1D0000C0F0CEA131518BF95EA0C0F06D04FF0A0
:10C1E000000081EA030E0EF0004170BD00F01CF863
:10C1F0008900013E00F007B800F009B84FEA430C8F
:10C200005FEA5C5C08D081EA030100F05BB84FEAAA
:10C21000410C5FEA5C5CF6D14FF0000001497047C9
:10C220000000FF070000F87F0EF1020E2EF0030E53
:10C230005EF8046B364205D4012A43EB030515F57D
:10C24000001F12D8012841EB010C1CF5001F0CD86F
:10C250000ED14FEAD17C15F5001F0CEB4C0C0CF104
:10C26000020C08BF4CEBD37C04E04FF0080C01E05B
:10C270004FEAD37C0CEB4C0526FA05F606F00706D0
:10C28000B6F1040C06D20EEB860CBDE870404CF003
:10C29000010C6047DFE80CF0090B02024FF000418F
:10C2A0004FF00000A1F5002170BD1946104601288D
:10C2B00051EB010418BFD4F5001484BF002001F035
:10C2C000004170BD0808A0F500114FEA3101704728
:10C2D00053EA010C17D41CF5801F58BFBCF5801F12
:10C2E00000F106808B4218BF704708BF824270473A
:10C2F00007D713F5801F58BF11F5801F19D48B4243
:10C3000070479B4270471CF5801F08D5BCF5801F05
:10C31000F7D5994218BF704708BF904270474FF455
:10C32000001C1CEB430F38BF1CEB410F01D299429C
:10C3300070470FB40CBC03BCFFF7C1BE91EA030FFA
:10C3400010B581F000413FF5FBAB83F0004300F0F6
:10C35000D5B800002DE9F04101F5801CBCF5001FA7
:10C36000C0F2A9804FEA115C21EA0C510CF1FD0CDE
:10C3700041F480115FEA5C0C0CF5C07C01D34000F5
:10C38000494130A4890241EA905187028E0E0A0C7D
:10C39000A45D04FB04F602FB06F6C6F14046A4FBCE
:10C3A0000662F60D46EA422606FB06F4A4FB0123CC
:10C3B0005242C3F1404338BF5B1EA6FB0242002439
:10C3C000E6FB0324D20B42EA4446A6FB0623A1FB6C
:10C3D00002E2A3FB07E4E3FB61426442C2F1404E88
:10C3E00038BFAEF1010EA6FB04234FF00002E6FBBE
:10C3F0000E32A2FB03463400E2FB6264A1FB06E6B8
:10C40000A4FB07E8E4FB61687642C8F1405838BFF6
:10C41000A8F10108A2FB06E4A3FB08E5E2FB6854CF
:10C42000A1FB05E6A7FB04E8E1FB648618F1200503
:10C4300056F10006A809A8F11B08B10908F03F0849
:10C44000B8F10A0F40EA86601CD901EB0C51BDE837
:10C45000F08100BFFCF5EEE8E2DDD8D3CFCBC7C357
:10C46000C0BDB9B6B4B1AEACA9A7A5A3A19F9D9B11
:10C470009A9896959392908F8D8C8B8988878685D4
:10C4800084838281A0FB006800FB01F208EB420874
:10C49000B8EB872807D5341858EB0104D5D5401CD4
:10C4A00051F10001D1E7341A78EB0104CDD4401EDC
:10C4B00071F10001C9E75FEA4C0C5FEA9C5C0DD1A9
:10C4C00005D34FF0000001F00041BDE8F081BDE868
:10C4D000F04170B5FFF7A8FE6DDBFFBEBDE8F0418F
:10C4E0004FF00000004970470000F87F10B591EA56
:10C4F000030F48BF83F000433FF522AB841A71EB72
:10C50000030C07D212198CF0004C43EB0C03001BF8
:10C5100061EB0C01DFF8A4E14FEA1154A4EB135CCA
:10C520001EEA430F18BF9EEA445F00F0B08023EA82
:10C530006E03524221EA0451C3EB6E0338BF5B1E07
:10C54000DCF1200E25D322FA0CFE10EB0E0043FA8C
:10C550000CFE41EB0E01CCF1200E03FA0EFE10EBA7
:10C560000E0051F10001CCF1200E29D412FA0EF286
:10C5700001EB0451BDE8104058BF7047401C1CBF80
:10C58000B2F1004F704700280CBF491C20F0010099
:10C59000704712EB020E43EB030218BF4FF0010E7F
:10C5A0004EEA4202ACF1200CDCF11E0E54D943FAE3
:10C5B0000CFE10EB0E0051F1FF31CCF11E0ED5D563
:10C5C0000EF1010E12FA0EFE404141EB010101EBAA
:10C5D000445C5FEA5C5C10D910EBDE7001EB045147
:10C5E00038BFBEF1004FBDE8104018BF70470028AB
:10C5F0000CBF491C20F00100704730D24FEAD42C08
:10C6000011F5001124F400641BD0B1FA81F20B3A49
:10C61000A41AA41ED2F12003914030FA03F3194367
:10C62000904001EBCC71002C01EB0451BDE81040AF
:10C63000A8BF704701F1C0414FF0000001F0004178
:10C640007047B0FA80F310FA03F100D110BDE41A7C
:10C65000173C4805C90AE4E701EB045110BD491035
:10C6600001EB0451BDE810404FEA300002E04FF00A
:10C67000000170474A0008BF0042F8D0B2F5001F21
:10C6800028BF704701F000414FF0000070479EEA5C
:10C69000445F07D011EA5E0FBDE8104004BF0021DF
:10C6A00000207047BDE8104070B5FFF7BDFD00BF2A
:10C6B00040DFF63E83F00041104670470000E0FF87
:10C6C00043004FEAD30C4FEA3C0C43401FBF4007E6
:10C6D0000CF1605113F0FE4F70471CF0006F03D156
:10C6E00000200CF0004170470CF0004343EA50700A
:10C6F00010B540EACC0000F00EF800BF0000009238
:10C700004FEA0001FFF7DEBD4FF000414FF000009F
:10C71000A1F5002170470EF1020E2EF0030E5EF817
:10C72000044B244204D44FEA4102B2F17F4F11D8A6
:10C730004FEA4003B3F17F4F0CD80ED14FEAD07CC3
:10C74000B2F17F4F0CEB4C0C0CF1020C08BF4CEB20
:10C75000D17C04E04FF0080C01E04FEAD17C0CEBF7
:10C760004C0324FA03F404F00704B4F1040C06D2D9
:10C770000EEB840CBDE810404CF0010C6047DFE884
:10C780000CF0070802024FF00040A0F5800010BD39
:10C790000846420018BFD2F1807288BF00F0004006
:10C7A00010BD4FF04070E1EE100A7047FF2141EAE2
:10C7B000D050C00570474FF000007047F5F76BB8D8
:10C7C000F5F7A0B90CF00F03092B08BF082000F003
:10C7D0005F800A2B0BD0082B18BF704708BF1CF0D6
:10C7E000400F0AD04FF000004FF0000170471CF0DE
:10C7F000400F18BF4FF0004070471CF0100F08D0DA
:10C8000020F0704300F07F4242EAD3014FEA4370C8
:10C81000704700F0604021F07F4242EA000201F0E0
:10C820007F4040EA727070474FF0FF0C4CF4E06CB0
:10C830001CEA11531CBF9CEA030C9445C2BFDA42A8
:10C8400001EB02517047002B0DD0BCF1000F0FD04F
:10C85000002A01F00041A4BF41F0E04141F07F61B6
:10C860004FF00000704701F000414FF000007047AA
:10C8700050EA01334FF09B0C18BF4CF0806C7FF4F2
:10C88000FFA97047F4F786BCF5F7A8BDF5F736BFEA
:10C890001CF4801F11D01CF4E02F03D06FEACC31C0
:10C8A000490070474FF04050EFF3008222F0704291
:10C8B00042EA000282F3008870474FF000007047A0
:10C8C000206700100C0000008000000020690010AC
:10C8D0000001000040000000E8030000010000002B
:10C8E000206D00100C00000080000000100000C14E
:10C8F000814001C0804101C0804100C1814001C030
:10C90000804100C1814000C1814001C0804101C01F
:10C91000804100C1814000C1814001C0804100C10F
:10C92000814001C0804101C0804100C1814001C0FF
:10C93000804100C1814000C1814001C0804100C1EF
:10C94000814001C0804101C0804100C1814000C1DF
:10C95000814001C0804101C0804100C1814001C0CF
:10C96000804100C1814000C1814001C0804101C0BF
:10C97000804100C1814000C1814001C0804100C1AF
:10C98000814001C0804101C0804100C1814000C19F
:10C99000814001C0804101C0804100C1814001C08F
:10C9A000804100C1814000C1814001C0804100C17F
:10C9B000814001C0804101C0804100C1814001C06F
:10C9C000804100C1814000C1814001C0804101C05F
:10C9D000804100C1814000C1814001C0804100C14F
:10C9E000814001C0804101C0804100C1814000C040
:10C9F000C101C30302C2C60607C705C5C404CC0CE7
:10CA00000DCD0FCFCE0E0ACACB0BC90908C8D81856
:10CA100019D91BDBDA1A1EDEDF1FDD1D1CDC14D466
:10CA2000D515D71716D6D21213D311D1D010F03096
:10CA300031F133F3F23236F6F737F53534F43CFCA6
:10CA4000FD3DFF3F3EFEFA3A3BFB39F9F83828E856
:10CA5000E929EB2B2AEAEE2E2FEF2DEDEC2CE42426
:10CA600025E527E7E62622E2E323E12120E0A06096
:10CA700061A163A3A26266A6A767A56564A46CAC66
:10CA8000AD6DAF6F6EAEAA6A6BAB69A9A86878B8D6
:10CA9000B979BB7B7ABABE7E7FBF7DBDBC7CB474E6
:10CAA00075B577B7B67672B2B373B17170B0509096
:10CAB00091519353529296565797559594549C5C26
:10CAC0005D9D5F9F9E5E5A9A9B5B995958988848D6
:10CAD00049894B8B8A4A4E8E8F4F8D4D4C8C4484A6
:10CAE0008545874746868242438341818040303175
:10CAF0003233343536373839414243444546403085
:10CB00005800303132333435363738396162636436
:10CB10006566403078000400000800000000000056
:10CB200000020001000010004FBB610567ACDD3F53
:10CB3000182D4454FB21E93F9BF681D20B73EF3F44
:10CB4000182D4454FB21F93FE2652F227F2B7A3CBC
:10CB5000075C143326A6813CBDCBF07A8807703C75
:10CB6000075C143326A6913CC4EB98999999C9BFE8
:10CB7000711623FEC671BCBF6D9A74AFF2B0B3BF1D
:10CB80009AFDDE522DDEADBF2F6C6A2C44B4A2BFDD
:10CB90000D5555555555D53FFF8300922449C23F49
:10CBA0006E204CC5CD45B73F513DD0A0660DB13F7D
:10CBB000EB0D76244B7BA93F11DA22E33AAD903F8F
:10CBC000000000000000F03F000000000000F83FFF
:10CBD00000000000000000000000004003B8E23F39
:10CBE000000000000000000006D0CF43EBFD4C3EEB
:10CBF000033333333333E33FFFAB6FDBB66DDB3FE0
:10CC00004D268F515555D53F01411DA96074D13F27
:10CC100065DBC9934A86CD3FEF4E454A287ECA3F21
:10CC20003E5555555555C53F93BDBE166CC166BFA3
:10CC30002CDE25AF6A56113FF16BD2C541BDBBBE9C
:10CC4000D0A4BE726937663E0000000000000000FC
:10CC50000000000000000000303132333435363738
:10CC6000383961626364656678700030313233341C
:10CC70003536373839414243444546585000000064
:10CC800002400000000000A000000000054000007D
:10CC9000000000C8000000000C4000000000409CA4
:10CCA00000000000194000000020BCBE0000000091
:10CCB00034400000BFC91B8E00000004B5400000D6
:10CCC000504BCFD06607E2CF010000006C4100005E
:10CCD0003E8251AADFEEA73401000000D9420000D5
:10CCE000DCB5A0E23A301F97FFFFFFFFB44500001C
:10CCF000FD25A0C8E9A3C14FFFFFFFFFFF3F0000D4
:10CD00000000008000000000FF3F000000000080E5
:10CD1000000000002820655263765374617465201A
:10CD20003D3D2053544154455F52585F494E49544C
:10CD30002029207C7C2028206552637653746174FE
:10CD400065203D3D2053544154455F52585F524346
:10CD5000562029207C7C20282065526376537461FC
:10CD60007465203D3D2053544154455F52585F4502
:10CD700052524F522029000025645F25645F253000
:10CD80002E32663A3A25643A3A25643A3A25733A9D
:10CD90003A25643A3A253034783A3A25643A3A25C5
:10CDA000643A3A25643A3A25643A3A25643A3A258F
:10CDB000643A3A25643A3A25643A3A252E31665F58
:10CDC000252E31663A3A252E31665F252E31663A98
:10CDD0003A25645F25645F25643A3A25645F2564DB
:10CDE0003A3A25645F25640025645F25645F253039
:10CDF0002E32663A3A25643A3A25643A3A25733A2D
:10CE00003A25643A3A253034783A3A25643A3A2554
:10CE1000643A3A25643A3A25643A3A25643A3A251E
:10CE2000643A3A25643A3A25643A3A252E31665FE7
:10CE3000252E31663A3A252E31665F252E31663A27
:10CE40003A25645F25645F25643A3A25645F25646A
:10CE500000000000D0CF020800000020D80700002A
:10CE6000C401020804D2020800000010A000000063
:10CE70002002020804D20208D80700207015010021
:10CE80003C020208A4D20208A0000010909F0000FB
:10CE90003C020208000000000000F07FFFFFFFFFDF
:10CEA000FFFFEF7F1001000043000000F8FFFFFFCD
:10CEB00000404040404040404040414141414140AD
:10CEC0004040404040404040404040404040404062
:10CED00040050202020202020202020202020202F1
:10CEE00002202020202020202020200202020202F6
:10CEF000020290909090909010101010101010104E
:10CF00001010101010101010101010100202020259
:10CF1000020288888888888808080808080808089D
:10CF20000808080808080808080808080202020299
:10CF300040000000000000000000000000000000B1
:10CF400000000000000000000000000000000000E1
:10CF500000000000000000000000000000000000D1
:10CF600000000000000000000000000000000000C1
:10CF700000000000000000000000000000000000B1
:10CF800000000000000000000000000000000000A1
:10CF90000000000000000000000000000000000091
:10CFA0000000000000000000000000000000000081
:10CFB000000000001C00000043000000F8FFFFFF1D
:10CFC0000C0000000E0000000F0000002E0000000A
:10CFD0000114022B0232112E6DA20208040835A1A1
:10CFE0000208031A0D0832103683A30208061AEB52
:10CFF0002032171AD11832013619A00208051A91E9
:10D0000018320F1A1D2829741A95180135BC2002F0
:10D0100040045A1004DA04040A1118040A110C041A
:10D0200011D95029049A1C040A15084C09155412E8
:10D03000801943111210120219FE19051A800C11E1
:10D040003A801312082A040E4A081C1A800F590A43
:10D050003933392C493C291A39162909A98C290454
:10D0600029B0690469EC0A11140469A0DA100401FA
:10D070001F1A04751A108649061A0197590B124097
:10D080002A800E2280290719A1014205298FC27525
:10D090003C62012009EC51383DEC51B83DA3803F82
:10D0A0000310A041DBE8033971021373021372D03D
:10D0B0000844656661756C740510413030320D119D
:10D0C00042313233140A2234500611727074616393
:10D0D0000B156765160C11766F6C16FB6572BF1920
:10D0E000160C1173706416CA6D80598409114219A7
:10D0F000160D107363616E160914420C1172747070
:10D10000160911B02916EB6D6F441916EA696C39CE
:10D11000160C126C61639ADC746172431916CE743A
:10D12000726176657139B00C105F7468420B1170D2
:10D1300064580D106D6F6465160B12676F9A0C11B1
:10D14000706F7316ED6261636B16F80874706C6132
:10D150007965722CDD616E676C6FF00872656C65C5
:10D160006167760D1063616C6C16EF7365747461A2
:10D17000736E19160D10726F757416041073747037
:10D1800029160B1170641619B30911160C1174725B
:10D190006116EB6D6F9929160C11766D6F840C1169
:10D1A0006C6F63B0DD61766F698629580D107573F9
:10D1B000696342FD61736572160910F1392CFA72C8
:10D1C0001839420A117942E6616E676C650F116485
:10D1D000656C727470581B7463B1BA632EDF727021
:10D1E000746E6F64412916EC6C696E162942F469FD
:10D1F0007073FD7072696EC5110F104465666175BC
:10D200006C18F26600000000000102030401020332
:10D2100004060708090000000000000000000000EC
:10D2200000000000000000000000000000000000FE
:10D2300000000000000000000000000000000000EE
:10D24000000000000000000000000000000000C01E
:10D2500000000000000000000000000000000000CE
:10D260000004F601C0A80064821F00000000000056
:10D27000000000000002573531303053000000003C
:10D28000BDB60208BFB60208C3B60208C1B602089E
:10D29000B5B60208B9B602080000000000000000A0
:04D2A0007F0000000B
:040000050802018963
:00000001FF
